:100000000C94481A0D9467210D943C210D941121F4
:100010000D94E6200D94BB200D9490200D94652046
:100020000D943A200C94791A0C94791A0C94791A3C
:100030000C94791A0C94791A0C94791A0D94233D26
:100040000C94791A0C94791A0C94791A0C94791AE4
:100050000C94791A0C94791A0C94791A0D94C71C83
:100060000C94791A0D9418240D94EE230C94791A9B
:100070000C94791A0C94791A0C94791A0C94791AB4
:100080000C94791A0C94791A0C94791A0C94791AA4
:100090000D94E6280D945C280D949E280C9420263F
:1000A0000C94791A0C94791A0C94791A0C94791A84
:1000B0000C94791A0C94791A0C94791A0C94791A74
:1000C0000C94791A0C94791A0C94791A0D94B8231B
:1000D0000D948E230C94791A0C94791A0C94791A35
:1000E0000C94791A07634236B79BD8A71A39685619
:1000F00018AEBAAB558C1D3CB7CC5763BD6DEDFD4A
:10010000753EF6177231BF000000803F0800000006
:10011000BE922449123EABAAAA2ABECDCCCC4C3EFC
:1001200000000080BEABAAAAAA3E00000000BF00EB
:100130000000803F0000000000084178D3BB4387E7
:10014000D1133D190E3CC3BD4282AD2B3E68EC82FB
:1001500076BED98FE1A93E4C80EFFFBE01C4FF7F80
:100160003F00000000000C9455F80C94D8EA0C9461
:10017000984E0C94E0360C9404350C943B3A0C9455
:100180009C650C94566D0D949C1A0C943F200C9415
:10019000CFEA0C9418730C94A5310C94902E0C9407
:1001A000B5BD0D94373C0C94CCB20C941A200D9430
:1001B00098090C9423C20C9445280C9461AD0C94BE
:1001C0006D3D0C941EB80C9491E70C9494DF0C9444
:1001D000E0B20C9425B80D94900B0C9465720C94BD
:1001E000416C0C9434720C9472A30C9488BD0C94E2
:1001F00049220D94FD340D94161C0C9421700C941E
:1002000059660D9455160C9448AD0C9490DF0C94DF
:100210004F6D0D9411190C94756D0D9400330C9461
:10022000114A0D9479350C94E0210C949A6D0C943C
:10023000D0DF0C9483B40C944AB40C94F81B0C9447
:10024000191C0C94813A0D943A0C0C945C410C945A
:10025000DD300C9470BC0C9495BC0D94251C0C9452
:100260008FBC0C94B8B30C94C1F80C94A21A0C94E3
:10027000A6BD0C9481B20C94E9720C9426C20D9424
:10028000A7310C9422800D94E72B0C94A2BC0D9402
:10029000F7300C9403610C946CBC0C94391C0C94D6
:1002A0005F450C942B380C94E9DF0C94FA1A0C94EB
:1002B0001D810C9488F70D94BB170C9471630D94F9
:1002C000FB160C940C810C9412810D94CD160C9499
:1002D00080570C94FBB70D9422090D94B5090D9429
:1002E000BC1A0C9419FB0C940BF90C949CBD0D9446
:1002F0005E190C94D7370C947DBC0C9418810C9427
:10030000B2E20C942CB80C94E8E70C9406450C94DB
:100310006EBD0D94F80D0D94CA0D0D94DF310C9443
:1003200043A50C9479630C94962A0C9476450C940E
:100330007A720D940C370C949F6E0C94DBA40C9481
:10034000BC510C941B800C9458650C9402720C9454
:100350002FA50C94866C0C94F5710C947C6D0C9408
:10036000E71B0C94B96D0D94421B0C94801C0C94EB
:100370005C710C9414C20D9408180C94D3210D9444
:10038000A7380C9485210C94F4560C941E6A0C9496
:10039000E3F80C947CDF0C94681E0C943D710C9473
:1003A000617E0D944F380D94D8380C94091D0D942E
:1003B000F3220C941A1E0D9412180C94AB640C9436
:1003C00062BC0C9442230C9438B40C94CA660C940E
:1003D000D6B20D94BC360C94CEA40C9405350C9476
:1003E00088E70C9452710C9484DF0D9488180C9457
:1003F00081BC0C948CDF0C947EE70D94D60D0C948C
:10040000221E0C9457E10D9455180C947B6E0C949D
:1004100075630C9425E00D940F090C94B8B20D94FB
:1004200057310C9468630C949FB20D946C190C9422
:1004300014E70C9470350C948BBC0D94623C0C94B6
:10044000CAE70C94D9E20D94C40B0C94C21D0C9411
:10045000E7DF0C948C9D0C94BD720D94AF190D9434
:10046000FE0D0C94E56D0C944FAD0C94C81D0C94CE
:10047000A9B20C94A6AD0C94CD360C9477A40C9430
:1004800088630C94CFB30C94BFBD0C945E570C944E
:10049000CA720D94D00D0C94CBDE0C946E580C9453
:1004A00004720C94CD1A0C94981E0C94D9710D946E
:1004B0003D190C943DE40C948B6D0D94CA090D9478
:1004C000EE0B0D94521A0C94D2420C94AF7F0D9403
:1004D0009A360D9471400D9490350C94431B0D94F5
:1004E0006D0C0C94AE380C94DF430C94F3630C94B5
:1004F00022210C9429E00C94DE6D0D941E170D94AE
:10050000A60C0C94F7720C9481F20D94D6320C94D4
:10051000AC4E0C943A600C9414430C94C96E0C9439
:1005200075E30D945D1A0C942C9C0C9420710C9422
:100530008E450C941C1E0C9407350C94DEEA0C942A
:1005400098640C94EFFA0D940F2C0C9487BC0C94C7
:10055000F2600C949B6F0D94AD220C94A7BC0D948B
:10056000E40C0C94A8630D942C170C94A97F0C94A4
:10057000B2750C94B1DE0C94CF6D0C94156C0C9488
:1005800099BC0C9440460D948D0C0C94826D0D9486
:100590008D090C9494630C94A6A40C9452720C9440
:1005A000A31A0C944D730C9468BC0D9420190D94EF
:1005B000441B0C94D3BD0C9415730C9415C20C946D
:1005C000C01D0C94C2B20C94BB820C94F51B0C940D
:1005D000FB2D0C940F810C9406350C943A710D94FC
:1005E000DE190C94A67F0C94CE8D0C94ED570C94D0
:1005F000A6DF0C9422580C94C9BD0C94A3720C94E1
:100600003A580C94B31A0C9436E00C94E4720C949F
:100610008B6F0D9496190C949DBC0C94401B0D94FB
:10062000D6080C9485630C94681C0C9474BC0D94CF
:10063000040D0C94A5570C94EA6F0D9443360C945A
:10064000C46D0C94C61A0C9409B80C94CCE50C94A7
:100650007E4E0D9493140C94923D0D94D13B0C94CA
:10066000A3BC0D9418180C94BAE20C947C210C9441
:10067000CA570C94D9650C9492BD0D94F3180C9440
:1006800098630C9429F30C949EB30D94FC3B0C944A
:10069000B9630C9488DF0C940FE00C94B39F0D9415
:1006A000B8090D940F180C94E7BD0C9417480C94DE
:1006B0002F6D0C94E3DF0C9480DF0C9402B80C9443
:1006C0006A460C94C61D0C9416960C9424720C94D5
:1006D000F5E70C9444650C9413460D94CE160C94D7
:1006E00090630C9478BD0C9411580C9475E70C949D
:1006F000AFB30C94DDBD0C94476D0D94B7320C94E0
:1007000007F90D94AA090C940CF80D94A1180D94F6
:100710003C1A0C94939D0C94192B0C9483630C94A9
:10072000651C0C9493F80C94DEE70C94EDFA0C9491
:10073000615D0C945ABD0C94F1A40C94C4F70C9414
:10074000C41D0C946B830C9410B80C94128A0C94F6
:100750006FA40C9419E60C9455BD0D94FB080C94F1
:10076000B2F80D946D380C9470AD0C94C6DF0D94F6
:10077000201B0D941D0D0C94386D0C94ED1F0C94E2
:10078000F7600C9405710C9424E80C94D81B0C941D
:100790008FAD0D9438350C949B1D0C9482690C948C
:1007A0005FF30C94C3710C94391D0C94B76E0C94C8
:1007B000E0630C9415810C9477BC0D94F7360D947E
:1007C000A7090D9498310C94A41A0C94ECDE0D94A6
:1007D00096080C94EF430C94B86C0C94D8720C945B
:1007E00080BD0C946D730C94A3430D94261A0C9445
:1007F00026F90C9499720C948BA40C9405700C94AB
:1008000091B20D940A170C94FCDF0C944F600C9479
:100810004A1B0C94BB6C0D9417350C94F3E70C94A5
:100820001E1E0D94CC160C9464BD0D94A13B0D942A
:100830006E170C94201E0C94B6E70D94CB160C94F6
:100840004DBD0C94C64D0C9492F30D9454400C94F1
:10085000BAF20C941E6F0C94B8A40D949B090D94DD
:10086000A8190C94486C0C94BE4E0C94A3E70C94FD
:10087000604E0D94D41A0C946C9F0C94841C0C94B0
:1008800043434E414E494E495459494E46CDCCCC36
:100890003D0AD7233C17B7D13877CC2B329595E654
:1008A000241FB14F0A000020410000C84200401C34
:1008B0004620BCBE4CCA1B0E5AAEC59D746364690B
:1008C0006E6F70737578585B000A282D2943525952
:1008D0005054000A282D2950554C5345206F6E2046
:1008E00050494E3132000A282D2943414E000A2832
:1008F0002D294D455243555259000A282B294D5553
:100900004C544956454E54000A282B2950574D5FE8
:1009100052454C4159000A282B294D444E53000A98
:10092000282D2955415254425249444745000A282E
:100930002B295359534C4F47000A282B295049441F
:10094000000A282D294D43503233303137000A2810
:100950002D294152544E4554000A282B294F544109
:10096000000A282D29535049204C4544000A282BC1
:10097000294D4F544F5220435452000A282D2941EB
:1009800043204841494552000A282D294343533802
:10099000313120262048444331303830000A282B9A
:1009A00029524553544152545F4C414E5F4F4E5F64
:1009B0004D5154545F4552524F5253000A282D292D
:1009C0004841524452455345542C207573696E6713
:1009D00020736F6674000A282B29434F554E5445E7
:1009E00052000A282B29444854000A282B29445332
:1009F000323438322D313030000A282B294F5749F4
:100A00005245000A282D2949504D4F444255530064
:100A10000A282B294D4F4442555320307830362038
:100A200061742053657269616C322073706565640E
:100A30003A39363030000A282B2941444146525574
:100A40004954204C4544000A282B29444D58000A9B
:100A5000282B2957697A6E657435783030000A285A
:100A60002B294672656552616D207072696E7469DA
:100A70006E67000A282B295741544348444F4700CA
:100A80006C617A79686F6D652E7275000A436F6EBE
:100A9000666967207365727665723A00323031316B
:100AA00030334C0020432B2B2076657273696F6EB8
:100AB0003A00343063316663615F323032362D3054
:100AC000312D3130000A4C617A79686F6D652E7274
:100AD00075204C6967687448756220636F6E747224
:100AE0006F6C6C65722000204F464600204F4E0010
:100AF0002042595041535300536176656420746F0E
:100B000020454550524F4D00536176696E67206312
:100B10006F6E66696720746F20454550524F4D2EA9
:100B20002E00556E6B6E6F776E20737566666978F2
:100B30002000556E6B6E6F776E20636D64200043EE
:100B40006F756E7465723A2000444D582D4F757460
:100B500020496E69743A2000444D582D4F75742019
:100B600073746F703A200041737369676E65643AFD
:100B700000444D58206374726C3A2000693136008D
:100B800001693332000275313600037533320004D7
:100B9000693868000569386C0006753868000775A3
:100BA000386C00087831300009313030000A446573
:100BB0006661756C742073657269616C206D6F6419
:100BC00065204E3831207573656400384531002644
:100BD00000384E31000600384532002E00384E32C3
:100BE000000E00384F31003600384F32003E0037DB
:100BF0004531002400374532002C00374F31003496
:100C000000374F32003C00374E31000400374E327F
:100C1000000C00206164646564206279206E756D4B
:100C200020004D4255533A2000416464696E6720AC
:100C300072656773207769746820616374696F6E89
:100C4000733A00416464696E67207265666572720A
:100C5000656420726567733A00416464696E672059
:100C6000707265666574636820726567733A004DDB
:100C70004255533A204D6F646275732074656D70F0
:100C80006C617465206E6F7420666F756E643A20B7
:100C9000004D4255533A20496E76616C6964207468
:100CA000656D706C6174652E002C002C002C002C7E
:100CB000004D4255533A20636F6E66696720666146
:100CC000696C65643A004D4255533A20636F6E6615
:100CD0006967206572726F72004D4255533A206306
:100CE0006F6E666967206C6F6164656420004D42B9
:100CF00055533A204F7574206F66206D656D6F7285
:100D000079004D4255533A20506F6C6C696E6720E4
:100D10006572726F7220004D4255533A204E6F74C7
:100D200020737570706F72746564207265672074CB
:100D30007970650A004D425553443A2049676E6FF9
:100D4000726564202D20657175616C207769746807
:100D5000207365747465642076616C004D42555350
:100D6000443A204D61707065643A004D42555344D9
:100D70003A204E65737465644D61707065643A0025
:100D80004C6173744B6E6F776E2076616C75653A4B
:100D90002000536561726368696E67207265673A07
:100DA0002000206F7574206F662072616E67652069
:100DB0006275666665722C206665746368696E6725
:100DC00000646566207265672320004D42555344D8
:100DD0003A20536561726368696E672072656723A4
:100DE000003A002066726F6D207479706520004DA6
:100DF000425553443A2020676F7420002076616C7E
:100E00003A0020004D425553207265733A2000206D
:100E100076616C206E6F74206368616E6765642E06
:100E200020436F6E74696E7565004D4255533A00EC
:100E30003A20657175616C20746172676572742EF9
:100E4000003D004D4255533A002076616C206368A6
:100E5000616E6765642E004D4255533A00204E6F17
:100E6000773A00204C6173743A002023002070729E
:100E70006566657463682000205265672F636F693B
:100E80006C206D75737420626520696E7400206932
:100E90006E7465726E616C2073656E64206572722B
:100EA0006F72202D206E6F207265672F636F696CE3
:100EB0000020696E7465726E616C2073656E6420CB
:100EC0006572726F72202D206E6F2074656D706C6C
:100ED0006174650020696E7465726E616C20736563
:100EE0006E64206572726F72202D206E6F20737495
:100EF0006F7265004D425553443A20656E64506FE1
:100F00006C6C20004D425553443A20506F6C6C205D
:100F100000206E6F7420666F756E64004D425553ED
:100F20003A2020706172616D20002073656E6469E3
:100F30006E672063616E63656C6C6564004D42553D
:100F4000533A2020706172616D20004D4255533A32
:100F50002020002073656E64206572726F722E20EF
:100F6000004D4255533A2020004164642040563AD7
:100F700020002056616C3A20004D425553443A20DF
:100F80007375666669783A00206F722073756666BD
:100F9000697820004D4255533A204E6F2074656D9C
:100FA000706C61746520666F7220004D6F746F7293
:100FB0003A2074696D656F757400556E6B6E6F774E
:100FC0006E20636D64004D6F746F723A20466F72CD
:100FD00063656420657865637574696F6E00564556
:100FE0004E543A20636F6E666967206661696C656E
:100FF000640056454E543A20696E69740056454E59
:10100000543A2050494420503D0056454E543A2011
:1010100044652D496E69740056454E543A20436824
:10102000616E2062616C616E63653D002073657462
:101030002052455645525345206D6F646500564514
:101040004E543A205049443A20002073657420449D
:101050004952454354206D6F64650056454E543ADD
:10106000205049443A20002073657420524556456B
:10107000525345206D6F64650056454E543A2050DA
:10108000415353205049443A200020736574204452
:101090004952454354206D6F64650056454E543A9D
:1010A0002050415353205049443A2000206F75741A
:1010B0003A00207365743A0020696E3A0056454E36
:1010C000543A2000204F75743A00205265713A005E
:1010D00056454E543A2000206D33002066726F6DE5
:1010E0002000204D6178207265713A002066616EA3
:1010F000253A002061637469766520563A005645AA
:101100004E543A20546F74616C20563A0056454E46
:10111000543A2076616C7565200041432061697204
:1011200020726F6F6D74656D703A200056454E5495
:101130003A004143206D6F64653A200056454E5495
:101140003A004143206169722074656D703A200055
:1011500056454E543A005049443A20616C726561DC
:10116000647920696E697469616C697A656400509C
:1011700049443A20496E76616C69642070617261FD
:101180006D2061727261792E002C002C002C002CD5
:10119000005049443A20636F6E6669672066616952
:1011A0006C65643A005049443A20636F6E66696723
:1011B000206572726F72005049443A20636F6E6608
:1011C0006967206C6F6164656420005049443A206F
:1011D0004F7574206F66206D656D6F727900504990
:1011E000443A2044652D496E69742000203C414CEE
:1011F0004D3E0020443A0020493A0020503A002059
:10120000696E3A00207365743A005049443A2000F0
:101210005049443A20496E76616C6964207061726D
:10122000616D2061727261792E00536574206F7553
:101230007420746F20002050494420616C61726DED
:101240002E20002050494420616C61726D3A206369
:101250006C6F736564005049443A20556E6B6E6F35
:10126000776E2073756666697820005049443A208D
:10127000556E6B6E6F776E20636D64200020536532
:1012800074706F696E743A005049443A20002049E6
:101290006E7075742076616C75653A005049443AF9
:1012A000200020696E697400200050574D2D4F7545
:1012B000742023002073746F7000200050574D2D50
:1012C0004F75742023003D0050696E3A0020696E0E
:1012D00069740070696E230072656C617943747281
:1012E0003A20002073746F700052656C61792D4F45
:1012F000757420230072656C61794374723A200022
:1013000069646C65006F66660068656174696E6724
:101310000066616E00647279696E6700636F6F6C5E
:10132000696E6700616374696F6E002069732000E5
:101330004F7574200072656C61794374723A2000B5
:10134000556E6B6E6F776E207375666669782000D8
:1013500072656C61794374723A2000556E6B6E6FE2
:10136000776E20636D64200072656C6179437472DE
:101370003A2000616374696F6E0072656C61794335
:1013800074723A20005B305D3A2000202D202D2021
:101390002D20EFBBBF003E003E31202D20005B30F2
:1013A0005D3A2000202D202D202D20EFBBBF003ED8
:1013B000003E31202D20005379736C6F67207265D9
:1013C00073756D6564005379736C6F672072657314
:1013D000756D6564005379736C6F672073757370F6
:1013E000656E646564000000000000636D640000C9
:1013F000736574000076616C000064656C000048E1
:1014000053560000524742000066616E00006D6F47
:101410006465006374726C006875650000736174C4
:10142000000074656D7000726177000020002E006E
:10143000696E00735F6F7574006D79686F6D65001C
:101440004354524C2F657865633A204F75744F664C
:101450004D656D6F72793A2000202D3E20004D5170
:1014600054543A2000202D3E2000456D69743A20E6
:101470003C00202D3E20004974656D436D643A2088
:1014800000202D3E20004974656D3A2000315754EC
:101490003A20427573207265736574206572726FAD
:1014A00072003157543A2042757320526573657447
:1014B00020646F6E65003157543A204453323438FB
:1014C000322070726573656E742C2072657365745A
:1014D000004932432052657365740053746174751A
:1014E000732064656666657265640A002D3E00506F
:1014F00075623A20002D3E005075623A20002D3E64
:10150000005075623A20000000000000636D640026
:1015100000736574000076616C000064656C000007
:101520004853560000524742000066616E00006D4D
:101530006F6465006374726C0068756500007361A8
:1015400074000074656D700072617700002D3E00BC
:101550005075623A20002D3E005075623A200053CB
:10156000454E445354415455533A20556E6B6E6F5B
:10157000776E20636D64200A000000000000000008
:101580000000004F4E00000000000000004F4646E3
:10159000000000000000005245535400000000000D
:1015A00000544F47474C450000000048414C540050
:1015B0000000000000584F4E0000000000000058DE
:1015C0004F4646000000000000494E43524541533B
:1015D00045000044454352454153450000454E41B6
:1015E000424C450000000044495341424C45000034
:1015F00000554E465245455A450000465245455A0B
:1016000045000000004155544F0000000000004616
:10161000414E5F4F4E4C590000484947480000007A
:101620000000004D454449554D000000004C4F5707
:1016300000000000000000484541545F434F4F4CFC
:101640000048454154000000000000434F4F4C004B
:101650000000000000445259000000000000005249
:101660004742000000000000004853560000000000
:10167000000000206661696C65643A004D6F646229
:101680007573206F7020004D423A206F6B003D0053
:101690004D423A205643230020636D643D003D00D7
:1016A0004D423A2056435F6865617423004D423ACB
:1016B000204E6F7420737570706F72746564207241
:1016C000656720747970650A002056616C3A30783D
:1016D0000020543A00205265673A3078004D423A73
:1016E00020416464723A00444D580000000000003C
:1016F000444D58524742570000444D58524742000B
:10170000000050574D0000000000004D425553446A
:10171000494D0000544845524D4F00000052454C81
:1017200041590000000047524F555000000000563C
:101730004354454D500000004D4255535643000060
:10174000004143484149455200005350494C4544EB
:101750000000004D4F544F5200000000504944001B
:1017600000000000004D42555300000000005541AC
:101770005254425244470052454C415950574D0033
:10178000444D5852474257570056454E5453000057
:101790000000454C455641544F5200434F554E545E
:1017A0004552000048554D0000000000004D4552D4
:1017B00043555259000020002D3E00436F6E766560
:1017C0007274696E6720002D3E0057726F6E67203D
:1017D00041737369676E6D656E742000524742787D
:1017E0003A200020764C6576656C3A0020436F6E97
:1017F00076563A0020436F6E76533A0020486F7455
:101800003A00436F6C643A0020436F6E76657274E1
:10181000656420563A00436F6E7665727465642085
:10182000533A002D3E0057726F6E67204173736903
:10183000676E6D656E7420002D3E0057726F6E6787
:101840002041737369676E6D656E7420004D415061
:101850003A2076616C206D617070656420746F2031
:1018600020004D41503A2076616C75652061626FB1
:10187000766520726967687420626F756E642000F7
:101880002069732062656C6F77206C6566742062D6
:101890006F756E6420004D41503A2076616C75651D
:1018A00020004D41503A20636D64206D6170706579
:1018B0006420746F200000000000000000000000A1
:1018C0004F4E00000000000000004F4646000000A0
:1018D0000000000052455354000000000000544F27
:1018E00047474C450000000048414C5400000000B0
:1018F0000000584F4E00000000000000584F4646C0
:10190000000000000000494E43524541534500008D
:1019100044454352454153450000454E41424C45E4
:101920000000000044495341424C45000000554E20
:10193000465245455A450000465245455A45000025
:1019400000004155544F00000000000046414E5F2A
:101950004F4E4C5900004849474800000000000025
:101960004D454449554D000000004C4F57000000C4
:1019700000000000484541545F434F4F4C0048452C
:101980004154000000000000434F4F4C0000000095
:10199000000044525900000000000000524742007D
:1019A0000000000000004853560000000000000046
:1019B00020537566663A002041543A0053746F70A4
:1019C00070696E6720496E707574730020697320AA
:1019D0000044656C6574696E6720636F6E662E20C7
:1019E00052414D207761733A0053746F7070656493
:1019F000006E6F7468696E6720746F2073746F7007
:101A00000053746F7070696E67206368616E6E65F5
:101A10006C73202E2E2E0043616E206E6F74206337
:101A20006C65616E202D206C6F636B656400436F85
:101A30006E666967206368616E676564206C6F63BA
:101A4000616C6C792C20706F7274616C20646973A6
:101A500061626C6564002F636F6E6669672E6A73DE
:101A60006F6E007265626F6F742000436D643A2080
:101A7000002F636F6D6D616E642F002F72616D2F8B
:101A8000002F6974656D2F002F6974656D2F00221A
:101A9000687474703A2F2F6C617A79686F6D652E57
:101AA00072752F70776122004C6F636174696F6E7D
:101AB0003A20687474703A2F2F003F6D61633D00C7
:101AC0002669703D0026706F72743D00266E616D50
:101AD000653D002F0020004D5154543A20436F6D56
:101AE000706C6574652E2052656D6F766520746F1D
:101AF000706963200024636F6D6D616E64004D51E9
:101B000054543A20436C65616E557020726574615F
:101B1000696E656420746F70696320002200220082
:101B20004F75744F664D656D6F727921005D2000B1
:101B30003A5B004D5154543A005D00456D70747924
:101B40003A205B000A003A004D41433A00554450A8
:101B5000205379736C6F6720696E697469616C6971
:101B60007A65642E0A005379736C6F672070617216
:101B7000616D733A002E6C6F63616C005365727611
:101B8000696365207265636F72643A20006D444E2C
:101B90005320726573706F6E646572207374617226
:101BA0007465642E004572726F7220736574746977
:101BB0006E67207570204D444E5320726573706FB0
:101BC0006E6465722100476F74204950206164641F
:101BD000726573733A00276970205B69705B2C64CF
:101BE0006E735B2C67775B2C7375626E65745D5DDD
:101BF0005D5D27202D2073657420737461746963A3
:101C00002049500A004661696C656420746F206346
:101C10006F6E6669677572652045746865726E657A
:101C200074207573696E6720444843502E20596FA5
:101C3000752063616E20736574206970206D616E1C
:101C400075616C6C792100204D41534B3A0020475F
:101C5000573A0020444E533A004C6F61646564204B
:101C600066726F6D20666C6173682049503A000A95
:101C70007573657320444843500A0053746172744D
:101C8000696E67206C616E00414243444546474897
:101C9000494A4B4C4D4E4F5051525354555657583C
:101CA000595A6162636465666768696A6B6C6D6ED8
:101CB0006F707172737475767778797A30313233E8
:101CC0003435363738392B2F3D0042617369632034
:101CD000003A004F544120696E697469616C697AF9
:101CE00065640A0044454641554C54207061737345
:101CF000776F726420666F72204F544120415049C3
:101D00002E20557365206F746170776420636F6D4A
:101D10006D616E6420746F207365740070617373FD
:101D2000776F7264004D5154543A20747279697916
:101D30006E67206E656E78742062726F6B657200DC
:101D40004D5154543A20546F6F206D616E79206369
:101D50006F6E6E656374696F6E206572726F7273F9
:101D60002E2052657374617274204C414E002074B1
:101D7000727920616761696E20696E203520736514
:101D8000636F6E6473004D5154543A206661696C00
:101D900065642C2072633D004D5154543A204177C4
:101DA000616974696E6720666F722072657461691B
:101DB0006E656420746F7069637300636F6E6E6527
:101DC000637465642061732000202E2E2E00207520
:101DD0007365723A003A000A4D5154543A204174E6
:101DE00074656D7074696E6720636F6E6E65637481
:101DF000696F6E20746F2000646973636F6E6E6527
:101E000063746564005573696E67204D51545420A6
:101E100070617373776F72642066726F6D20636F89
:101E20006E666967002E6C6F63616C006D444E5383
:101E3000206E616D6520757064617465643A200080
:101E4000446576696365204E616D653A004D515475
:101E5000543A204174206C6561737420646576691E
:101E60006365206E616D6520616E642062726F6BC8
:101E70006572204950206D75737420626520636F10
:101E80006E6669677572656400757074696D652C3E
:101E900066726565686561700034306331666361E0
:101EA0005F323032362D30312D3130004C69676869
:101EB000744875622000246E616D65005265626928
:101EC0006E6420737563636573732E2049502061BF
:101ED0006464726573733A004572726F723A20726D
:101EE0006562696E64206661696C0052656E657733
:101EF000656420737563636573732E204950206198
:101F00006464726573733A004572726F723A20723C
:101F1000656E65776564206661696C000A4E6F20A6
:101F20006C696E6B00436F6E74696E7565207769BE
:101F300074682070726576696F75736C79206C6F48
:101F40006164656420636F6E666967003330732077
:101F5000454550524F4D206973206E6F7420726555
:101F60006C6F616465642E205265626F6F74004D02
:101F70005154543A20416363657074696E672063FD
:101F80006F6D6D616E64732E2E2E0A004E6F204DA4
:101F900051545420636F6E66696775726564004CB6
:101FA0006F6164696E6720636F6E66696720667231
:101FB0006F6D20706F7274616C2064697361626C04
:101FC00065642E2075736520676574204F4E2074FC
:101FD0006F20656E61626C6500436F6E6669672095
:101FE00069732076616C696400436F6E74696E7505
:101FF0006520776974682070726576696F75736C97
:1020000079206C6F6164656420636F6E6669670038
:102010005365747570204F5441004D5154543A200B
:102020007365742066697273742062726F6B657277
:102030000043757272656E74204C414E20636F6E62
:102040006669672869702C646E732C67772C7375CA
:10205000626E6574293A000A557365207468657369
:102060006520636F6D6D616E64733A202768656CDF
:102070007027202D207468697320746578740A278E
:102080006D61632064653A61643A62653A65663AF7
:1020900066653A3030272073657420616E64207362
:1020A000746F7265204D41432D6164647265737372
:1020B00020696E20454550524F4D0A276970205BBC
:1020C00069705B2C646E735B2C67775B2C73756235
:1020D0006E65745D5D5D5D27202D207365742073D2
:1020E00074617469632049500A27736176652720FB
:1020F0002D20736176652063757272656E7420633E
:102100006F6E66696720696E204E5652414D3B20C6
:102110004F4E7C4F4646202D20656E61626C652FC8
:1021200064697361626C65206175746F7361766553
:102130000A2767657427205B636F6E666967206195
:102140006464725D27202D2067657420636F6E665E
:1021500069672066726F6D207072652D636F6E66A1
:102160006967757265642055524C20616E642073F6
:10217000746F726520616464722C204F4E7C4F46F0
:1021800046202D20656E61626C652F646973616203
:102190006C6520646F776E6C6F6164206F6E207366
:1021A0007461727475700A276C6F616427202D202A
:1021B0006C6F616420636F6E6669672066726F6D15
:1021C000204E5652414D0A2770776427202D2064F7
:1021D0006566696E6520616E642073746F72652038
:1021E0004D5154542070617373776F72640A276F76
:1021F000746170776427202D20646566696E6520A0
:10220000616E642073746F7265204854545020418D
:1022100050492070617373776F72640A276C6F671F
:10222000205B73657269616C5F6C6F676C65766566
:102230006C5D205B7564705F6C6F676C6576656C58
:102240005D27202D20646566696E65206C6F6720B0
:102250006C6576656C2028302E2E37290A276B692D
:102260006C6C27202D20746573742077617463680B
:10227000646F670A27636C65617227202D20636C89
:1022800065617220454550524F4D0A277365617252
:10229000636827202D2073656172636820312D7774
:1022A000697265206465760A277265626F6F7427AC
:1022B000202D207265626F6F7420636F6E74726F71
:1022C0006C6C657200536F6674207265626F6F7418
:1022D000696E672E2E2E00206E65770020697320B0
:1022E000003157543A003157543A205365617263B4
:1022F00068696E67206465760052414D3D000A535F
:1023000079736C6F6720000A312D77697265200040
:102310000A6D71747420000A6D6F646275732076A3
:1023200032000A6D6F6462757320763120282B2984
:10233000000A696E7075747320000A6974656D73A4
:1023400020000A436F6E666967757265643A002FF4
:1023500000496E3A2000496E697469616C697A6956
:102360006E6720496E70757473003157543A20734C
:1023700065747570207265736F6C7574696F6E200B
:10238000003157543A204453323438322D313030F2
:10239000206E6F742070726573656E7400315754CF
:1023A0003A204453323438322D31303020493243D0
:1023B00020726573746F726564003157543A20421D
:1023C0007573207265736574206572726F72003167
:1023D00057543A2042757320526573657420646FB8
:1023E0006E65003157543A204453323438322D311F
:1023F00030302070726573656E742C207265736561
:1024000074004572726F7220312D7720696E697485
:10241000003157543A204453323438325F3130302F
:102420005F4932435F544F5F31575F4252494447DF
:102430004520696E697400444D584F75742E2046CE
:102440007265653A00444D58696E2042756666654E
:102450007220616C6C6F632065727200496E6974E2
:1024600020696E2063683A003B003D0050696E3A77
:10247000003B003D4C4F5700546865726D6F3A0049
:102480004F6E6520776972652052656164790A0034
:10249000467265653A00444D58206F757420737418
:1024A00061727465642E204368616E6E656C733A68
:1024B0002000444D5820696E207374617274656405
:1024C0002E204368616E6E656C733A0042726F6BCA
:1024D00065727320636F6E666967757265643A0032
:1024E0004170706C79696E6720636F6E6669670012
:1024F0004C6F6164656420455441473A004E6F203B
:1025000073746F72656420636F6E666967004C6FE9
:10251000616465642066726F6D20454550524F4D71
:10252000006C6F6164206661696C6564004A534F9A
:102530004E206465746563746564004C6F61646902
:102540006E6720436F6E6669672066726F6D204507
:102550004550524F4D00436F6E6669672061757438
:102560006F736176653A000A5379736C6F67206404
:1025700065627567206C6576656C3A0053657269B3
:10258000616C206465627567206C6576656C3A00E5
:1025900053617665640A005365742064796E616DD9
:1025A00069632049500A004F54412050617373778A
:1025B0006F726420757064617465640A004E6F20E8
:1025C00049502061647265737300205361766564BD
:1025D000004C6F6164696E67204854545020636FEB
:1025E0006E666967206F6E20737461727475703ADD
:1025F00000000000000000000000004F4E0000003E
:1026000000000000004F464600000000000000529D
:10261000455354000000000000544F47474C45000C
:1026200000000048414C54000000000000584F4E8C
:1026300000000000000000584F4646000000000067
:1026400000494E43524541534500004445435245DD
:102650004153450000454E41424C450000000044B6
:10266000495341424C45000000554E465245455A9B
:10267000450000465245455A45000000004155546A
:102680004F00000000000046414E5F4F4E4C590085
:1026900000484947480000000000004D45444955A6
:1026A0004D000000004C4F570000000000000048A3
:1026B0004541545F434F4F4C004845415400000092
:1026C000000000434F4F4C000000000000445259EE
:1026D000000000000000005247420000000000001F
:1026E0000048535600000000000000636F756C64E2
:1026F000206E6F742070617273653A2000557064AB
:10270000617465640A00454550524F4D20636C6505
:10271000617265640A004D5154542050617373779F
:102720006F726420757064617465640A002B002DFB
:1027300000455461673A200047657420455441477D
:102740003A2000485454502F312E310025733A203E
:1027500025730D0A0020485454502F312E310D0A94
:10276000486F73743A2025730D0A41636365707472
:102770003A202A2F2A0D0A436F6E6E656374696FC3
:102780006E3A20636C6F73650D0A0025730020009C
:102790000D0A00474554006661696C656420746FDA
:1027A00020636F6E6E6563740A004552524F523A51
:1027B000205365727665722072657475726E6564F9
:1027C0002000436F6E666967206E6F7420636861D6
:1027D0006E6765640A00446F6E652E0A00436F6E73
:1027E0006669672070617273696E67206661696CE3
:1027F00065640A004765742061626F7274656400E5
:10280000676F7420436F6E6669670A00687474703E
:1028100020726574636F64652000667265652000D0
:10282000436F6E666967205552493A206874747028
:102830003A2F2F002044656661756C7420636F6EBB
:102840006669672073657276657220757365643A90
:1028500020006C617A79686F6D652E7275000000DA
:102860002100240027002A002D0030003300010140
:102870000000040107010A010000220025002800D1
:102880002B002E0031003400020100000501080178
:102890000B010505050507050808080802020202E4
:1028A0000A0A0808040404040101010101010101EC
:1028B0000303030303030303040707070C0C0C0CB7
:1028C0000C0C0C0C020202020606060606060606A0
:1028D0000B0B0B0B0B0B0B0B01021020200808102D
:1028E0002040102040800201020108040201010280
:1028F0000408102040808040201008040201800459
:1029000002018040201008040201080402010102B3
:1029100004081020408001020408102040800000BC
:102920000A0B02090C0D0E08070304010000000049
:102930000000000000000000000000000000000097
:102940000000000000000000000012111000000054
:102950000000000000000000000000000000000077
:10296000000000004D4255533A204164642040531A
:102970003A20002F64617461002F736B6574636883
:10298000004163636573732D436F6E74726F6C2DBA
:10299000526571756573742D507269766174652D19
:1029A0004E6574776F726B3A20747275650041637F
:1029B000636573732D436F6E74726F6C2D416C6C15
:1029C0006F772D486561646572733A202A00416310
:1029D000636573732D436F6E74726F6C2D416C6CF5
:1029E0006F772D4D6574686F64733A20504F535460
:1029F0002C4745542C4F5054494F4E53004163636C
:102A00006573732D436F6E74726F6C2D416C6C6FB8
:102A1000772D43726564656E7469616C733A2074D6
:102A2000727565004F5054494F4E530044454C4514
:102A30005445005055540047455400504F535400DE
:102A4000617574686F72697A6174696F6E3A20009B
:102A5000417574686F72697A6174696F6E3A2000AB
:102A6000436F6E74656E742D4C656E6774683A20A2
:102A7000006F637465742F73747265616D00696DA6
:102A80006167652F6A70656700696D6167652F67AB
:102A9000696600746578742F68746D6C006170707D
:102AA0006C69636174696F6E2F6A736F6E00746511
:102AB00078742F706C61696E00436F6E74656E740C
:102AC0002D547970653A2000436F6E6E65637469AA
:102AD0006F6E3A20636C6F73650041636365737357
:102AE0002D436F6E74726F6C2D416C6C6F772D4F30
:102AF000726967696E3A202A00556E6B6E6F776E49
:102B0000004E6F74204D6F646966696564004F4BB9
:102B1000004D6F766564207065726D616E656E74D0
:102B20006C7900496E7465726E616C2053657276C3
:102B30006572204572726F72005061796C6F6164CA
:102B400020546F6F204C61726765004E6F74206671
:102B50006F756E64005757572D41757468656E74B4
:102B600069636174653A20426173696320726561CB
:102B70006C6D3D224163636573732072657374727B
:102B800069637465642200556E617574686F72695B
:102B90007A6564005061796C6F61642073697A654D
:102BA0002077726F6E67004261642072657175658F
:102BB000737400485454502F312E31200020005798
:102BC000726F6E67207061796C6164004D5154546E
:102BD0003A204354524C2F7478743A204F75744FF6
:102BE000664D656D6F72793A2000202D3E2041546C
:102BF0003A004368616E20747970653A004E6F2028
:102C000073746F7265642076616C756573202D2016
:102C100064656661756C743A200053617665642062
:102C2000455441473A0053657420455441473A2082
:102C300000556E6B6E6F776E2073756666697820CF
:102C400000556E6B6E6F776E20636D642000636C51
:102C5000724374723A2000444D58494E3A00454F31
:102C600046003D00494E3A002500C2B04320483D91
:102C70000020444854323220747970652E20543D2F
:102C800000494E3A00204E6F20656D6974206461E2
:102C90007461210020436F756E74657220747970C1
:102CA000652E2076616C3D00494E3A0020436F75D9
:102CB0006E74657220747970652E20494E434F52B0
:102CC0005245435420496E74657272757074206E5B
:102CD000756D626572212121004952513A004163AC
:102CE00074697661746520696E2000416374697649
:102CF00061746520696E20002D3E00200023002DA8
:102D00003E00200050656E6465643A2023002D3E2D
:102D100000456D69743A002D3E00456D69743A00B6
:102D20002D3E00456D69743A002D3E00456D697475
:102D30003A003D004C454741435920494E3A002056
:102D4000666F7220286D73293A004354524C3A2022
:102D50005363686564756C6520636D642000206D45
:102D6000730020666F7220004354524C3A20417227
:102D70006D656420002044697361726D6564004371
:102D800054524C3A20002074696D653A0043545205
:102D90004C3A205265733A004354524C3A206D6FBE
:102DA0006D656E74617279206576656E740020546D
:102DB000533A0020543A00544845524D3A00436C6F
:102DC00065616E696E6720616C61726D20003D0007
:102DD00050696E3A004354524C3A20436F6D6D6116
:102DE0006E6420626C6F636B65642062792064722C
:102DF00069766572004354524C3A204F4E3A416C0A
:102E00007265616479204163746976650A00435490
:102E1000524C3A2048414C543A416C726561647995
:102E200020496E6163746976650A004354524C3AD6
:102E300020584F4E3A2044697361626C65640A0001
:102E40004354524C3A20584F4E3A416C726561647B
:102E500079204163746976650A004354524C3A20E4
:102E6000584F464620736B69707065642E2050720F
:102E7000657620636D643A004354524C3A20547591
:102E8000726E6564206F66662066726F6D3A0043ED
:102E900054524C3A20526573746F726564206672A6
:102EA0006F6D3A004354524C3A2049676E6F726519
:102EB000642C206368616E6E656C20636D643D00F8
:102EC00020457865633A004354524C3A204163747C
:102ED0006976653A004354524C3A2048414C543A82
:102EE000416C726561647920496E616374697665CD
:102EF0000A004354524C3A20584F4E3A20446973CA
:102F000061626C65640A004354524C3A20584F4E3B
:102F10003A416C7265616479204163746976650A2F
:102F2000004354524C3A20584F464620736B697008
:102F30007065642E205072657620636D643A00439C
:102F400054524C3A205475726E6564206F66662048
:102F500066726F6D3A004354524C3A205265737456
:102F60006F7265642066726F6D3A004469736172B6
:102F70006D696E67206E6F7420617574686F726919
:102F80007A6564004354524C3A20636F6D6D616EF4
:102F900064206A75737420666F7220004354524C2B
:102FA0003A204E6F7420656E6F756768206D656D91
:102FB0006F727920666F722067726F7570206F7004
:102FC00065726174696F6E00496E76616C69642028
:102FD00061726700496E76616C6964206172670096
:102FE000496E76616C696420617267004354524C8B
:102FF0003A20556E6B6E6F776E20737566666978D2
:1030000000536B697070696E6720736368656475DF
:103010006C65642067726F75702065786563004326
:1030200054524C3A206368616E6E656C2066726F14
:103030007A656E004354524C3A206368616E6E6547
:103040006C2066726F7A656E00536B697070656490
:1030500020686F6D696520737475666600200020B6
:103060005375623D00204974656D3D004354524CD8
:103070003A2052414D3D004354524C3A204F757412
:103080004F664D656D6F72793A2000282D2920001A
:10309000282B2920002076616C756520697320003B
:1030A00020756E6B6E6F776E0A005D3D005B0020D1
:1030B000696E76616C69640020004143544956454D
:1030C0003A00206F6B003A00206661696C6564000D
:1030D0003A005265747279696E6720564354454DC3
:1030E0005020434D440A005265747279696E67201E
:1030F000564320434D440A005265747279696E67E5
:10310000206D6F6462757320434D440A00526574EC
:103110007279696E6720434D440A00206572726FB0
:10312000723D004D423A20706F6C6C696E672000F2
:103130002056616C3A20004D423A20004D423A2020
:103140004E6F7420737570706F7274656420726551
:103150006720747970650A004D423A20706F6C6C7C
:10316000696E672064696D6D657220004D423A207A
:10317000496C6C6567616C20617267756D656E7412
:10318000730A00206572726F723D004D423A2070E2
:103190006F6C6C696E6720504920002D004D423ADB
:1031A0002050492056616C203A004D423A20706F01
:1031B0006C6C696E6720504920004D423A20706F58
:1031C0006C6C696E6720464D206661756C742000DA
:1031D000206572726F723D004D423A20706F6C6CC8
:1031E000696E6720002D004D423A20464D20566101
:1031F0006C203A004D423A20706F6C6C696E67200B
:10320000464D20004354524C2F706F6C6C3A204F47
:1032100075744F664D656D6F72793A200020736545
:10322000632072656D61696E696E6700005EBCE265
:10323000613FDD83C29C7E20A3FD1F419DC3217F92
:10324000FCA2401E5F01E3BD3E6082DC237D9FC186
:10325000421CFEA0E1BF5D0380DE3C62BEE0025C7A
:10326000DF81633D7C22C09E1D43A1FF4618FAA466
:1032700027799BC584DA3866E5BB5907DB85673952
:10328000BAE406581947A5FB7826C49A653BD98746
:10329000045AB8E6A7F91B45C6987A24F8A6441A3A
:1032A00099C7257B3A6486D85B05E7B98CD2306E26
:1032B000EDB3510F4E10F2AC2F7193CD114FADF312
:1032C000702ECC92D38D6F31B2EC0E50AFF1134D06
:1032D000CE90722C6D33D18F0C52B0EE326C8ED0FA
:1032E000530DEFB1F0AE4C1291CF2D73CA947628E6
:1032F000ABF517490856B4EA6937D58B5709EBB5D2
:1033000036688AD495CB2977F4AA4816E9B7550BC5
:1033100088D6346A2B7597C94A14F6A8742AC896B9
:10332000154BA9F7B6E80A54D7896B353E3E200005
:10333000496E76616C696420636F6D6D616E6400C7
:10334000000020002300260029002C002F0032005E
:10335000000100000301060109013E3E3E004E6FE0
:10336000204D414320636F6E666967757265643AEC
:1033700020736574206669726D77617265277320AA
:103380004D41430A00454550524F4D207369676EC9
:103390006174757265206F6B00496E697469616C48
:1033A000697A696E6720454550524F4D2E00207254
:1033B000656164206572726F7220666F7220003ED4
:1033C0002000203C003157543A003157543A206EC7
:1033D0006F7420696E6974003157543A2042555316
:1033E000592074696D656F7574003157543A2044E3
:1033F00053323438325F4552524F525F434F4E463C
:103400004947003157543A20312D7769726520734E
:10341000686F727465640072656164790024737406
:1034200061746500757074696D65006672656568C4
:10343000656170002473746174730020457870694D
:103440007265640A00202D746172676574207A6F5A
:103450006E652D0020416C61726D20457870697237
:1034600065640A0020636D643A00204375723A0077
:10347000205365743A002054696D65723A00204CFF
:103480006F636B733A0052414D3D000069022504A1
:1034900011241FBECFEFD1E2DEBFCDBF00E00CBFD5
:1034A00019E0A0E0B2E0E6E8FAEB02E00BBF02C0F0
:1034B00007900D92A83AB107D9F721E1A8EAB9E03F
:1034C00001C01D92AD3BB207E1F71AE1C7E4DAE1B2
:1034D00000E006C021970109802FFE010F941355CB
:1034E000C634D10780E00807A9F70F94FC430D9478
:1034F000315D0C94000020913C0A260F3327331FC6
:1035000021323105ECF42091740BFC0190E080E055
:10351000243069F082E00895A0913C0A2191AC0129
:10352000445E554FA40FB52FB11D2C9301968617FD
:1035300098F380913C0A680F60933C0A80E00895FC
:1035400081E0089508950895E091A30B8091A20B66
:10355000E81730F4F0E0E15AF54F808190E00895EB
:103560008FEF9FEF08959091A30B8091A20B2FEF07
:103570003FEF981748F4E92FF0E0E15AF54F20812A
:1035800030E09F5F9093A30BC90108958091A20B37
:103590009091A30B891B990B0895CF92DF92EF9224
:1035A000FF920F931F93CF93DF937C01CB018A018E
:1035B00020917A0B222389F0EB016B01C40ED51EFA
:1035C000CC15DD0569F06991D701ED91FC91019071
:1035D000F081E02DC7011995F3CF642F0E947B1A6B
:1035E000C801DF91CF911F910F91FF90EF90DF9075
:1035F000CF900895CF93DF931F92CDB7DEB7698345
:1036000020917A0B2223F9F02091A00B203258F060
:1036100021E030E0FC013383228390E080E00F90D2
:10362000DF91CF9108958091A10BE82FF0E0E5584C
:10363000F44F998190838F5F8093A10B8093A00BAF
:1036400081E090E0ECCF61E0CE0101960E947B1A10
:10365000F7CF90E0FC01EE56F74DE491F0E0EE0F6D
:10366000FF1FE858F74DA591B4912C918852974DC2
:10367000FC018491822391E009F490E0892F089560
:1036800090E080E00895DC01ED91FC910284F385E7
:10369000E02D1994DF92EF92FF920F931F93CF9337
:1036A000DF93EC010C891D890115110559F01D8A64
:1036B0001C8AC801DF91CF911F910F91FF90EF906D
:1036C000DF900895EC85FD858E859F85DF01A80F2D
:1036D000B91F2C91243209F055C011962C912B372B
:1036E00009F050C00296E80FF91FF12CE12CDF0120
:1036F000D190DD2009F446C08DE7D816E9F08FEFB0
:10370000E81AF80AF4CF198A188A2C853D85211504
:10371000310579F08E859F85280F391FF9012081A9
:10372000222321F001969F878E873EC01D861C862E
:10373000C0CF0FEF1FEFBDCFE114F10419F11C92C0
:103740008E859F8502966C857D85680F791FE8813F
:10375000F9810684F785E02DCE011995998B888B28
:103760001B8A1A8AEC85FD858E859F85E80FF91FD7
:10377000EE0DFF1DD2828E859F850396E80EF91E01
:10378000FF86EE86288939892115310509F4BDCFD8
:103790008A899B89280F391FF9012081222309F486
:1037A000B2CF01969B8B8A8B022F220F110B81CFF8
:1037B000DC011C96ED91FC911D971E968D919C91BC
:1037C000E80FF91F8081082E000C990B0895DC0189
:1037D00015968D919C91009739F0DC01ED91FC914B
:1037E0000680F781E02D1994089583E090E0089514
:1037F000DC011296ED91FC9113973097B9F0169673
:103800008D919C918430910541F08530910541F076
:10381000039749F482E090E0089581E090E00895F4
:1038200081E190E00895828590E0089590E080E045
:10383000089585E090E008951F93CF93DF9300975C
:10384000A1F0FC011085212F2F70223071F4EC01C2
:1038500061857285838594850F94455369877A873E
:103860008B879C87107F13601887DF91CF911F9102
:1038700008958EE090E00895CF93DF93FC01C68118
:10388000D78180858F70853079F08630E1F420977C
:10389000D1F0E881F981309719F080818F7B79F43C
:1038A0000A80DB81C02DF3CF209769F0CE010E9402
:1038B0003C1C811105C00A80DB81C02DF5CF81E061
:1038C000DF91CF91089580E0FBCF84E190E00895EF
:1038D000DC01ED91FC910484F585E02D60E0199503
:1038E00081E090E00895ECEBF0E080818A7B8083BA
:1038F00060E084E10E94ABBC60E085E10C94ABBC6D
:1039000060E08DE00C94ABBC61E08DE00C94ABBC4E
:103910000F931F93CF93DF930097D1F0FC01208585
:103920002F702630A9F48B01EC010E9491AC009716
:1039300089F40E9436B2AC01B801CE010E9473B87E
:10394000B801CE01DF91CF911F910F910C9491ACF2
:1039500090E080E0DF91CF911F910F910895CF9279
:10396000DF92EF92FF92CF93DF9369017A010E9479
:10397000881CEC01892BC9F08885982F9F709230A4
:1039800039F0933071F0911110C0807F8260888788
:10399000C701B6010F94105669877A878B879C8779
:1039A00004C0C986DA86EB86FC86CE01DF91CF9112
:1039B000FF90EF90DF90CF900895CF92DF92EF923B
:1039C000FF9269017A01009791F0FC0120852F7028
:1039D000253069F40E9409ADFC01892B41F09085E6
:1039E0009F70933059F4C184D284E384F484C70176
:1039F000B601FF90EF90DF90CF9008959230B9F725
:103A000061857285838594850F9445536B017C0194
:103A1000EECFCF93DF93EC0165EF72E188E39FE097
:103A20000F94422369EE72E188E39FE00F944223F2
:103A30006C817D8188E39FE00E9422AD63EE72E19C
:103A400088E39FE00F94422388E39FE00F94432292
:103A500060E08C810E94D9BCE881F9810484F585FD
:103A6000E02D60E0CE01199581E090E0DF91CF91EB
:103A70000895CF93DF93EC016CEB72E188E39FE054
:103A80000F9442236C817D8188E39FE00E9422ADE8
:103A90006AEB72E188E39FE00F944223EA81FB81A5
:103AA0000280F381E02D6081718188E39FE00F94B3
:103AB000EB2264EB72E188E39FE00F94422388E3FA
:103AC0009FE00F944322E881F981008CF18DE02D75
:103AD000CE0119958130910529F0029759F060E0E7
:103AE0008C811AC063E070E0CE010F943D1660E057
:103AF0000E94D9BC60E08C810E94D9BC61E070E07A
:103B0000CE010F943D1660E00E94D9BC62E070E0E7
:103B1000CE010F943D1660E00E94D9BCE881F98186
:103B20000484F585E02D60E0CE01199581E090E0F8
:103B3000DF91CF910895CF93DF93EC0168E57BE0AF
:103B400088E39FE00F944223EA81FB810280F381A6
:103B5000E02D6081718188E39FE00F94EB2288E380
:103B60009FE00F944322E881F9810484F585E02DDC
:103B700060E0CE01199581E090E0DF91CF9108954A
:103B80000D94AC4B0D94AC4B0D94AC4B0D94AC4BD5
:103B9000EF92FF920F931F93CF93DF938C016AE014
:103BA00070E188E39FE00F94422388E39FE00F9445
:103BB0004322D8011496ED91FC91309749F1C681CA
:103BC000D781209729F1E881F9813097E9F0808148
:103BD0008823D1F060E375E0CE010E9491AC7C01B6
:103BE000009791F0FC0181859285A385B4850097AB
:103BF000A105B10549F00F94AC4BD70119961D9260
:103C00001D921D921C921C970A80DB81C02DD9CF7A
:103C1000D801ED91FC910484F585E02D60E0C801A8
:103C2000199581E090E0DF91CF911F910F91FF9066
:103C3000EF9008950D94AC4B0D94AC4B0D94AC4BA0
:103C40000D94AC4BEF92FF920F931F93CF93DF93A2
:103C5000EC018B018091B2099091B3090097A9F012
:103C6000FC0120852F70263081F40E9491ACFC016C
:103C700090859F70943049F481859285DF91CF9132
:103C80001F910F91FF90EF900895EE88FF88C70174
:103C900001970D97D0F464E375E0C8010F9474594F
:103CA000892B99F48FE2888F85E08E9DB0018F9DDE
:103CB000700D11246A517C4E46E050E0CE014996C9
:103CC0000F94804DCE014896D9CF90E080E0D6CFBA
:103CD000FC01828193810E9417E821E030E082306C
:103CE00011F430E020E0C90108950F931F93CF93A2
:103CF000DF938C01D0E0C0E001151105B1F0BE01E9
:103D00006458744FC8010F94494D892B51F4FE013A
:103D1000E058F44F849190E0DF91CF911F910F9183
:103D200008952596C233D10539F781E090E0F4CFAC
:103D3000AF92BF92CF92DF92EF92FF920F931F93B9
:103D4000CF93DF93CDB7DEB768970FB6F894DEBF99
:103D50000FBECDBFFC01098B1A8B2B8B3C8B4D8B7F
:103D60005E8B6F8B788F82819381009709F49DC061
:103D700024813581232B09F498C0CC2009F495C007
:103D80006F0170E060E00E94A1E5192FD601ED916E
:103D9000FC91008CF18DE02DC60119955C018230FB
:103DA000910509F476C0039709F445C095E0F1E068
:103DB000AF16B10409F091E019861A861B861C869D
:103DC0001D861E861F86188A8A85807F892B8A8792
:103DD000EE24EA94FE2C09891A892B893C894D89A5
:103DE0005E896F89788DCE0109960E94AC70F1E0F2
:103DF000AF16B10409F44FC082E0A816B10409F06F
:103E000045C06F8570E0D60114968C910E9415BD57
:103E100061E070E0C6010F943D166E8570E00E946F
:103E200015BD62E070E0C6010F943D166D8570E02F
:103E30000E9415BD2BC0612F661F6627661FCE012D
:103E400041960E94F56B5C01BC01D60114968C91E1
:103E50000E9415BD68EC72E188E39FE00F94422355
:103E6000F6016481758188E39FE00E9422AD66ECD3
:103E700072E188E39FE00F944223B50188E39FE05D
:103E80000E9422AD88E39FE00F94432281E090E0FE
:103E90000EC094E091CF63E070E0C6010F943D1630
:103EA000688970E00E9415BDACCF90E080E0689614
:103EB0000FB6F894DEBF0FBECDBFDF91CF911F913B
:103EC0000F91FF90EF90DF90CF90BF90AF9008954B
:103ED000CF92DF92EF92FF920F931F93CF93DC016B
:103EE0001296ED91FC9160E0848195810E9409AD6C
:103EF0008C01009729F0FC0180858F708530D1F00E
:103F000060E172E181E99EE00F94422381E99EE045
:103F10000F944322C12CD12C90E8E92E9FEBF92E6F
:103F2000C701B601CF911F910F91FF90EF90DF90E5
:103F3000CF900895C8010E94ACAD813040F1863029
:103F4000A8F1893020F565E0C8010E9409ADFC01A7
:103F500090859F709330F9F4C184D284E384F48413
:103F6000C1E060E0C8010E9409ADFC0190859F702E
:103F7000933009F5618572858385948520E030E072
:103F8000A9010F943E5387FF1FC0C111C9CFC12C97
:103F9000D12C7601C5CF923049F461857285838535
:103FA00094850F9445536B017C01DACFC0E0C12C9E
:103FB000D12C7601D6CF923039F461857285838514
:103FC00094850F944553DACFC111AACFC12CD12CBF
:103FD0008FE7E82E83E4F82EA3CFCF93DF93EC0195
:103FE0006EED71E188E39FE00F944223EA81FB814B
:103FF0000280F381E02D6081718188E39FE00F945E
:104000004722EC81FD81309721F0808191810F94CE
:10401000AC4B8C819D810F94AC4B70E060E08A8149
:104020009B810E9491E41D821C8281E090E0DF91DF
:10403000CF910895CF93DF93EC0168E375E088E3B7
:104040009FE00F94472240E050E0BA018A819B81B3
:104050000E94D4E4E881F9810484F585E02D60E0D4
:10406000CE0119956D858C810E94ABBC6D858D81CB
:104070000E94ABBC81E090E0DF91CF910895CF9397
:10408000DF93EC0167E475E088E39FE00F94EB2297
:10409000EA81FB810280F381E02D6081718188E3F8
:1040A0009FE00F9447228C819D81009711F00F941F
:1040B000AC4B70E060E08A819B810E9491E41D829C
:1040C0001C8281E090E0DF91CF910895CF92DF9242
:1040D000EF92FF920F931F93CF93DF93009701F11D
:1040E000DC011896EC91EF70E630D1F469017A01A9
:1040F0008B01EC010E9491AC0097A1F4A7019601FD
:10410000B801CE010E94BFB8B801CE01DF91CF91B6
:104110001F910F91FF90EF90DF90CF900C9491AC96
:1041200090E080E0DF91CF911F910F91FF90EF9091
:10413000DF90CF900895CF92DF92EF92FF920F938E
:104140001F93CF93DF93009701F1DC011896EC9158
:10415000EF70E630D1F469017A018B01EC010E9425
:1041600091AC0097A1F4A7019601B801CE010E947D
:104170009BB8B801CE01DF91CF911F910F91FF90B5
:10418000EF90DF90CF900C9491AC90E080E0DF91C5
:10419000CF911F910F91FF90EF90DF90CF900895F6
:1041A0008F929F92AF92BF92CF92DF92EF92FF9247
:1041B0000F931F93CF93DF93CDB7DEB760970FB602
:1041C000F894DEBF0FBECDBFE986FA860B871C8749
:1041D0002D873E874F87588B6115710511F00111AE
:1041E00003C090E080E0CCC07B015C01DB018D90DE
:1041F0009C9019821A821B821C821D821E821F8241
:1042000018868A81807F8A8366E575E0C7010E94EF
:1042100091AC6C016BE575E0C7010E9491AC7C012B
:10422000C114D10451F1F60180858F70843029F5D5
:10423000818592850E94751E182F8930B1F134F462
:104240008130E4F4C12CD12C760168C08A30D1F7DA
:10425000B701CE0109960E94C77829833A834B8320
:104260005C836D837E838F8398873F7009F4B9CF19
:10427000CE0101960E949E6D15C011E0B701CE01DE
:1042800009960E94C77829833A834B835C836D83A8
:104290007E838F8398873F7009F4A3CFCE01019668
:1042A0000E945A6D6B017C0139C0B701CE0109969D
:1042B0000E94C77829833A834B835C836D837E8316
:1042C0008F8398873F7009F48CCF31503B3008F0D2
:1042D000B9CFE32FF0E08827EF58FE4D8F4F0D94B4
:1042E00013558521852122217C217C21E021D321A8
:1042F000D321D3217C217C212D813E814F81588582
:10430000AAE0B0E00F94C954CDCFCD80FAE0CF9EA3
:10431000600111240D2C000CEE08FF0880911E0294
:10432000893020F480911D028930E8F069E77FE050
:1043300088E39FE00F944223B40188E39FE00F9449
:10434000EB2262E77FE088E39FE00F9442232AE0BC
:1043500030E0B701A60188E39FE00F94652288E36F
:104360009FE00F944322D5011296ED91FC9162E0FB
:10437000848195810E9409AD009779F581E090E0F4
:1043800060960FB6F894DEBF0FBECDBFDF91CF9120
:104390001F910F91FF90EF90DF90CF90BF90AF9063
:1043A0009F908F90089520E030E040E251E46D81CD
:1043B0007E818F8198850F94A4530F94105672CFED
:1043C0006D817E818F8198852AE030E040E050E069
:1043D0000F94AA5469017A01A1CFFC0120852F70A6
:1043E000263061F6B4010E9491AC5C01009731F275
:1043F000DC0118968C9118978F709BEF980F923074
:1044000008F0BCCF4501853029F416968C9016979C
:1044100017969C90F5018085806880876FE575E030
:10442000C4010E9491ACFC01892B61F0C186D28647
:10443000E386F486812F8295807F10851F70182B6C
:1044400010879CCF69E67FE088E39FE00F944223CA
:10445000D5016D917C9188E39FE00F94EB2288E376
:104460009FE00F944322A70196016FE575E0C40118
:104470000E949BB86FE575E0C4010E9491ACFC01FD
:10448000892B09F47BCF1295107F90859F70192B93
:10449000D7CF2F923F924F925F927F928F929F92AF
:1044A000AF92BF92CF92DF92EF92FF920F931F9342
:1044B000CF93DF9300D000D01F921F92CDB7DEB70D
:1044C00009831A832B833C834D835E836F837887B4
:1044D000DC011496ED91FC910FEF1FEF3097F9F08E
:1044E00057014C01C288D388E114F10489F1F70126
:1044F0008081882369F1C114D10489F1B701C60113
:104500000E9491ACE980FA800B811C812D813E8153
:104510004F815885BC01C4010E94D0208C01C80184
:1045200028960FB6F894DEBF0FBECDBFDF91CF91B6
:104530001F910F91FF90EF90DF90CF90BF90AF90C1
:104540009F908F907F905F904F903F902F90089515
:10455000C114D10421F0D6011696CD90DC907B8059
:10456000F12C0FEF1FEF272C312C512C412CC114B3
:10457000D10449F161E375E0C6010E9491AC009756
:10458000E9F0FC0120852F702230C1F481859285ED
:10459000A385B48582159305A405B50579F4E98052
:1045A000FA800B811C812D813E814F815885B60197
:1045B000C4010E94D0208C01FF24F394D6011296EE
:1045C000CD90DC90D4CFF110AACF64E97FE081E9EF
:1045D0009EE00F944223B50181E99EE00F94EB2207
:1045E00068E87FE081E99EE00F944223672D70E048
:1045F00081E99EE00E9422AD81E99EE00F94432272
:104600008ECFCF93DF93EC01EC81FD81408151810E
:10461000052E000C660B770B228186EB9BE00F9436
:104620004E2470E060E08A819B810E94A1E5E3EB6B
:10463000FCE0828386EB9BE0918380831092C30D24
:104640001092C50D1092C40DDF91CF910895CF93B4
:10465000DF936115710589F0EB01DC011296ED9194
:10466000FC9162E0848195810E9409ADBE010E94A7
:1046700091ACDF91CF910C9402BB90E080E0DF9190
:10468000CF9108954F925F926F927F928F929F92F7
:10469000AF92BF92CF92DF92EF92FF920F931F9350
:1046A000CF93DF93CDB7DEB768970FB6F894DEBF30
:1046B0000FBECDBF098B1A8B2B8B3C8B4D8B5E8B2A
:1046C0006F8B788FDC0112962D913C911397232BE1
:1046D00009F4DEC0CC2009F4DBC06C01ED91FC9143
:1046E000008CF18DE02D19955C0161E77BE088E39A
:1046F0009FE00F944223CE0141960E942A70A1149C
:10470000B10471F460E0CE0141960E94F56B682F10
:10471000F601848195810F940C3E81E090E0BAC04F
:10472000CE0141960E94E96D4C0194E0F2E0AF1693
:10473000B10459F081E1A816B10409F445C091E033
:10474000A1E0AA16B10409F495E019861A861B8621
:104750001C861D861E861F86188A8A85807F892B67
:104760008A87EE24EA94FE2C09891A892B893C89D0
:104770004D895E896F89788DCE0109960E94AC7053
:1047800067E67BE088E39FE00F944223CE01099621
:104790000E942A70B2E0AB16B10489F0E1E1AE16D6
:1047A000B104B1F0AA94AB2809F0B7CF188963E03F
:1047B00070E0C6010F943D16612F0F940C3E6F857B
:1047C000F6018481958151C0888D8170888FBCCF1E
:1047D0000FE710E08FEF88169806A9F0092C000C5F
:1047E000AA08BB08A50194012959310941095109B9
:1047F000AFEFB0E00F94C9542BE531E040E050E05A
:104800000F94AA54890163E070E0C6010F943D162D
:104810005C01288930E0D8010F942A55412C512C95
:1048200032014A94A30192010F94AA54622FC50148
:104830000F940C3E64E070E0C6010F943D165C01DD
:10484000AFEFB0E0A01BB10B288930E00F942A55E0
:10485000A30192010F94AA54622FC5010F940C3E3C
:104860006F85D60114968D919C910F940C3E1E85F8
:1048700061E070E0C6010F943D16612F0F940C3E6D
:104880001D8562E070E0C6010F943D16612F43CF95
:1048900090E080E068960FB6F894DEBF0FBECDBF03
:1048A000DF91CF911F910F91FF90EF90DF90CF900C
:1048B000BF90AF909F908F907F906F905F904F9040
:1048C0000895FC01818191E090937A0B80939B0B7A
:1048D0001092A10B1092A00B0895CF93C62F0E94A7
:1048E000612461EE8EE79CE00E94FA1A6C2F8EE73D
:1048F0009CE00E94FA1ACF910C941EBFCF93DF93D5
:10490000EC010E94612440E060EFCE010F943A3E3A
:10491000DF91CF910C941EBF0E94612481E00E9420
:104920002EBE91E0811190E0892F08951092740BB2
:1049300081E08093730B10924E0B61E084E10E9442
:10494000ABBC61E085E10E94ABBCE9EBF0E08081AB
:104950008E7F808380818D7F808388E48093B80000
:1049600085E48093BC000895CF93DF9391E090930A
:104970001B0A882361F0C091B800D091BA000E9450
:10498000731C0E949624D093BA00C093B800DF91A4
:10499000CF910895CF92DF92EF92FF920F931F93E2
:1049A000CF93FC01C1810E9409BE6B017C01809103
:1049B000740B811164C081E08093740B8093730B3E
:1049C0009FEF9093720B1092710B1092700B80936B
:1049D0004F0B80914F0BCC0FC82BC0934F0B809186
:1049E0004E0B813009F081C010924E0B0E9409BE1F
:1049F0006B017C0180914F0B8093BB008091760B03
:104A00009091770BA091780BB091790B892B8A2B21
:104A10008B2BA1F00E9409BE0091760B1091770BB1
:104A20002091780B3091790B6C197D098E099F09C3
:104A3000061717072807390708F442C08091BC0001
:104A400083FDD8CF85EC8093BC000E9409BE6B012A
:104A50007C018091740B813009F449C08091710B05
:104A6000811167C08091710BE0E5FBE0AFE5BAE032
:104A700090E0981751F121912D939F5FFACF80918B
:104A8000760B9091770BA091780BB091790B892BD5
:104A90008A2B8B2B09F48BCF0E9409BE0091760BD9
:104AA0001091770B2091780B3091790B6C197D095F
:104AB0008E099F09061717072807390708F077CFCF
:104AC0008091750B0E94B42480E01092A30B809318
:104AD000A20B8EE79CE00E94B31ACF911F910F9119
:104AE000FF90EF90DF90CF90089585EEACCF80914E
:104AF000760B9091770BA091780BB091790B892B65
:104B00008A2B8B2B09F4A5CF0E9409BE0091760B4E
:104B10001091770B2091780B3091790B6C197D09EE
:104B20008E099F09061717072807390708F091CF44
:104B3000C7CF81E099CF8F929F92AF92BF92EF92B1
:104B4000FF921F93CF93DF93EC010E9454BF4B0160
:104B50005C0110E08BE4E82EF12C0E9454BF681930
:104B600079098A099B09683E73408105910510F512
:104B7000ED85FE85309709F0199560EFCE010E9412
:104B80006D24CE010E94CA24182F80FD0FC08A8197
:104B9000813009F41A82812FDF91CF911F91FF900C
:104BA000EF90BF90AF909F908F900895C7010197AD
:104BB000F1F7D3CF81E08A83EECFCF93DF93EC017F
:104BC00063EC0E946D24CE01DF91CF910C94CA2436
:104BD00085ED8093BC008091760B9091770BA0912E
:104BE000780BB091790B0796A11DB11D23E0B69506
:104BF000A795979587952A95D1F72091BC0024FD1C
:104C000003C01092740B08954091760B5091770B6E
:104C10006091780B7091790B452B462B472B69F3EC
:104C20000097A105B10541F02AE22A95F1F700C0ED
:104C30000197A109B109E1CF8091750B0C94B424BF
:104C40001F920F920FB60F9211240BB60F922F9353
:104C50003F934F935F936F937F938F939F93AF9304
:104C6000BF93EF93FF938091B900887F803609F45A
:104C70004DC008F040C0883209F4A9C028F5803141
:104C800009F49DC0C8F4882309F4FBC0883009F4F6
:104C900096C0FF91EF91BF91AF919F918F917F91BE
:104CA0006F915F914F913F912F910F900BBE0F909D
:104CB0000FBE0F901F901895883109F488C080327C
:104CC00041F78093720B14C0803409F49DC040F406
:104CD0008033B9F38833E9F68093720B85ECB0C06A
:104CE000803509F485C0883509F496C0883489F682
:104CF0000E94E825CECF883909F48CC038F5883772
:104D000029F050F4883611F0803719F683E080934B
:104D1000740B10925E0A57C0883809F47BC0803942
:104D200019F0803809F0B5CF80915E0A803208F022
:104D300071C0E0915E0A81E08E0F80935E0A8091DF
:104D4000BB00F0E0E25CF54F80833DC0803B39F072
:104D5000E0F4803A09F479C0883A09F09ACF84E007
:104D60008093740B10923D0A10923C0AE0919E0BC6
:104D7000F0919F0B199580913C0A81110FC081E041
:104D800080933C0A10921C0A09C0803C09F4A6CF0B
:104D9000883C09F4A3CF883B09F07BCFE0913D0A22
:104DA00081E08E0F80933D0AF0E0E45EF54F808154
:104DB0008093BB0090913D0A80913C0A29C080916C
:104DC0004F0B8093BB0085EC8093BC0062CF909129
:104DD000710B8091700B981758F5E091710B81E081
:104DE0008E0F8093710BF0E0E05BF44F8081E9CF90
:104DF000E091710B81E08E0F8093710B8091BB006D
:104E0000F0E0E05BF44F80839091710B8091700B28
:104E10009817C8F285E8D8CFE091710B81E08E0F2A
:104E20008093710B8091BB00F0E0E05BF44F8083D6
:104E30008091730B81115CCF81E080934E0B84EAEB
:104E40008093BC001092740B24CF85EC8093BC003F
:104E50001092740B80915E0A803230F4E0915E0A09
:104E6000F0E0E25CF54F108260915E0A70E0E09144
:104E70009C0BF0919D0B8EE39AE0199510925E0ABF
:104E800008CF1092720B34CFCF93DF93EA01282F13
:104E9000DC01ED91F0E094E0F595E7959A95E1F766
:104EA000ED5AFD4F80818883FD013197E081EF70DD
:104EB000F0E0ED5AFD4F8081898322968A2F821B74
:104EC000861738F3615070E0660F771F460F571F43
:104ED000FA011282DF91CF910895CF92DF92EF9283
:104EE000FF9269017A01009791F0FC0120852F70F3
:104EF000263069F40E9491ACFC01892B41F0908529
:104F00009F709230A1F4C184D284E384F484C701F9
:104F1000B601FF90EF90DF90CF9008956185728584
:104F2000838594850F9410566B017C01F0CF9330EC
:104F3000A9F3913061F7C1840C2C000CDD08EE0858
:104F4000FF08E5CF009789F0FC0120852F70253000
:104F500061F40E9409AD009741F0FC0120852F709B
:104F6000243019F481859285089590E080E00895B9
:104F70000F931F93CF93DF9361ED74E188E39FE07C
:104F80000F94662381E00E942EBE0E94731C61E094
:104F900085E10E94D9BC60E084E10E94D9BCC4E1F3
:104FA000D0E010E001E0612F85E10E94ABBC10274A
:104FB0006AE070E080E090E00E9421BF219799F7BD
:104FC00064E170E080E090E00E9421BF0E9424B97B
:104FD0008091F4109091F510009729F10E948C2493
:104FE000882309F18091F4109091F5100E947E249D
:104FF00066EB74E188E39FE00F946623E091F41080
:10500000F091F51000838091F4109091F5100F94B9
:105010007F3E62EA74E1811102C06DE874E188E3C9
:105020009FE00F94662381E0DF91CF911F910F9154
:105030000895CF92DF92EF92FF920F931F93182F54
:105040006A017B010E9454BF04C0969587957795AD
:1050500067951A95D2F76C217D218E219F218B01B6
:105060009C0101501109210931090E3F1F4F2F4F9B
:105070003F4F20F061E070E080E090E01F910F91E1
:10508000FF90EF90DF90CF9008953F924F925F9204
:105090006F927F928F929F92AF92BF92CF92DF9248
:1050A000EF92FF920F931F93CF93DF9300D000D026
:1050B000CDB7DEB77C01362E8091AF09882309F485
:1050C0000AC1D70114969C9180911D02891708F49A
:1050D00002C18091190A90911A0ABAE06B1312C2A8
:1050E0008C53964FFC011082D70118968D919C919C
:1050F000892B09F4ECC08091C0099091C109A0915D
:10510000C209B091C309892B8A2B8B2B09F0CBC024
:105110000E9454BF2B013C01F70100851185D80185
:1051200019966D917C916115710599F4F80185804E
:105130009680A780B0848091740C9091750CA0919A
:10514000760CB091770C88169906AA06BB0609F46E
:1051500084C0D8011B964D915C911C974115510557
:1051600009F47BC0F701248153968C91539790E00A
:10517000322F377002C0959587953A95E2F780FFF8
:105180006CC0C22ED12CC601887F9370892B39F454
:1051900051968D919C91887F9370C82AD92AD80105
:1051A0008D919C91DC01ED91FC916115710509F4E3
:1051B000C1C00688F789E02D1995019709F04DC007
:1051C0006CE3F801808191810F945E22B601D801D1
:1051D0008D919C910E9467B1F8012281808191811B
:1051E00068E973E1222311F066E973E10F94422329
:1051F000D8011D966D917C911E978D919C910F9475
:10520000EB2260E2F801808191810F945E22D80147
:105210001F966D917C9150978D919C910F94EB22EC
:10522000F8012281808191816BE873E1222311F0E2
:1052300065E873E10F94422364EC79E0D8018D9125
:105240009C910F94EB22F80180819181DC01ED911A
:10525000FC91008CF18DE02D19950E9454BFAB019B
:10526000BC014419550966097709F70185819681C2
:10527000453651056105710508F472C0009721F0AB
:1052800065ED73E10F9466234FEF5FEFBA0180E0A5
:105290000E9419286093C0097093C1098093C209C4
:1052A0009093C30914C00E9454BF0091C00910918B
:1052B000C1092091C2093091C309601B710B820B97
:1052C000930B603375478105910508F021CF10924B
:1052D0001A0A1092190AD70115968D919C9116976A
:1052E000009771F014963C9120911E02231740F014
:1052F000DC01ED91FC910190F081E02D632D199579
:1053000081E090E026960FB6F894DEBF0FBECDBFC9
:10531000DF91CF911F910F91FF90EF90DF90CF9091
:10532000BF90AF909F908F907F906F905F904F90C5
:105330003F9008950488F589E02D26E135E03A8311
:105340002983D80115968D909D90AD90BC901897AB
:105350008B829C82AD82BE82BE016F5F7F4F2CCF5D
:105360004091C0095091C1096091C2097091C3096F
:10537000452B462B472B09F4AACF009721F066EC6A
:1053800073E10F9466231092C0091092C109109224
:10539000C2091092C309D70118960D911C91F8010A
:1053A000618572856115710591F44580568067802D
:1053B00070848091740C9091750CA091760CB091D2
:1053C000770C481659066A067B0609F480CFD80187
:1053D0001B964D915C911C974115510509F477CFAF
:1053E000F701248153968C91539790E0322F3770B8
:1053F00002C0959587953A95E2F780FF68CFC22E57
:10540000D12CC601887F9370892B39F451968D91E8
:105410009C91887F9370C82AD92AD8018D919C913C
:10542000DC01ED91FC916115710509F455C0068808
:10543000F789E02D1995019709F049CF6CE3F80140
:10544000808191810F945E22B601D8018D919C914B
:105450000E9467B1F80122818081918161EB73E143
:10546000222311F06FEA73E10F944223D8011D96B5
:105470006D917C911E978D919C910F94EB2260E22F
:10548000F801808191810F945E22D8011F966D9161
:105490007C9150978D919C910F94EB22F801228181
:1054A0008081918164EA73E1222311F06EE973E156
:1054B0000F94422367EB73E1D8018D919C910F9477
:1054C0004223F80180819181DC01ED91FC91008CF7
:1054D000F18DE02D1995FBCE0488F589E02D26E1AC
:1054E00035E03A832983D80115964D905D906D90F3
:1054F0007C9018974B825C826D827E82BE016F5FCA
:105500007F4F98CF843591050CF0E5CEBDE06B1749
:1055100009F4E1CE9C012F5F3F4F30931A0A20938C
:10552000190A8C53964FFC016083D5CECF92DF923F
:10553000FF920F931F93CF93DF9300D000D01F9261
:105540001F92CDB7DEB76C01F02E1A83022F10E048
:10555000FF2029F00115110511F401E010E040E0F1
:1055600050E061E070E0F601828193810E9474E670
:1055700001301105A9F10230110541F0012BB1F5FF
:1055800066EC7FE088E39FE00F9442238A818F706E
:10559000B9F1F60102811381C8010E9415E5672B5C
:1055A000682B692B89F401E010E0C80128960FB63A
:1055B000F894DEBF0FBECDBFDF91CF911F910F9149
:1055C000FF90DF90CF9008954FEF5FEFBA0180E03A
:1055D0000E941928AB01BC01C8010E94D4E4E3CFAA
:1055E000F1E0FF1681F082E0F81669F06AEB7FE0E7
:1055F00088E39FE00F94422388E39FE00F944322C7
:1056000010E000E0D2CFF601C280D380C6010E9434
:1056100015E5672B682B692B31F24FEF5FEFBA016D
:1056200080E00E941928AB01BC01C6010E94D4E4AD
:10563000BCCF2F923F924F925F926F927F928F9248
:105640009F92AF92BF92EF92FF920F931F93CF93CF
:10565000DF93CDB7DEB72C970FB6F894DEBF0FBE41
:10566000CDBF6130710509F463C18C01FC01E2809A
:10567000F38040E050E061E070E0C7010E949DE6E9
:10568000672B682B692B09F453C140E050E062E0BE
:1056900070E0C7010E949DE6672B682B692B89F497
:1056A00080910002882309F443C140E050E062E0A9
:1056B00070E0C7010E9474E68091000281508093DF
:1056C0000002F801E280F380C7010E9415E54B015A
:1056D0005C0119821A821B821C821D821E821F821B
:1056E00018868A81807F8A8340E050E2B701CE012C
:1056F00001960E94326B60E0CE0101960E94F56B2C
:105700007C01F801828193810E9417E8823011F0B8
:10571000853011F4F12CE12CF80186819AEC980F78
:10572000903108F0B7C121853285A90170E060E0B1
:1057300049875A876B877C8743845484712C612CFA
:105740000E94ECBD9C01990F440B550B241935099F
:1057500046095709AFEFB0E00F94C95429853A853F
:105760004B855C8524193509460957090F94AA54BD
:10577000390137FDB9C15FEF6516710411F00CF006
:10578000B6C181149104A104B10409F08BC1E618DB
:10579000F70856EFE5165FEFF5060CF0F6C0F801D6
:1057A000658585810E94ABBCF801A280B380C501EC
:1057B0000E9415E5672B682B692B59F44FEF5FEFBB
:1057C000BA0180E00E941928AB01BC01C5010E940A
:1057D000D4E4F801B48065858EEF8B0D8C3028F011
:1057E00084ED8B0D833008F070C0AA27BB27AE195B
:1057F000BF09662309F45CC09D01A1E0BFEF0F94CF
:10580000225529E130E040E050E00F94AA54BA015B
:10581000A90141505F4F6F4F7F4F942F852F692F04
:10582000782F6F3F710519F014F06FEF70E0663458
:10583000710514F466E470E08B2D78C06BEA7FE0AC
:1058400088E39FE00F94422388E39FE00F94432274
:1058500062E675E088E39FE00F944722F8016585D2
:1058600084810E94ABBCF801658585810E94ABBC38
:1058700040E050E0BA01F801828193810E94D4E4B3
:1058800040E050E061E070E0F801828193810E9485
:105890004BE640E050E062E070E0F80182819381E5
:1058A0000E944BE6809100028F5F8093000240C00F
:1058B0002FEF30E00F942A5529E130E040E050E02E
:1058C0000F94AA54922F832FAACF858191E0692744
:1058D0009EEF980F9C3020F08C52833008F0D6C099
:1058E0008B2D0E94ABBCAA27BB27AE19BF09F801BC
:1058F00085858823B1F12FEF30E00F942A5529E1F7
:1059000030E040E050E00F94AA54922F832F692F8B
:10591000782F6F3F710519F014F06FEF70E0663467
:10592000710514F466E470E0F80185810E9415BDEC
:1059300090E080E02C960FB6F894DEBF0FBECDBF8E
:10594000DF91CF911F910F91FF90EF90BF90AF909B
:105950009F908F907F906F905F904F903F902F908F
:1059600008959D01A1E0BFEF0F94225529E130E099
:1059700040E050E00F94AA54BA01A90141505F4F92
:105980006F4F7F4F942F852FC2CFFBE0EF16F104AE
:105990000CF45ECFF801658584810E94ABBCF801F0
:1059A000A280B380C5010E9415E5672B682B692B87
:1059B00059F44FEF5FEFBA0180E00E941928AB0164
:1059C000BC01C5010E94D4E4F801B58065858EEF65
:1059D0008B0D8C3020F084ED8B0D8330B0F466237A
:1059E00051F09701A1E0BFEF0F94225523E330E07F
:1059F00040E050E00ACF2FEF30E0D7010F942A5556
:105A000023E330E040E050E05BCF848191E0692700
:105A10009EEF980F9C3018F08C528330B8F58B2D88
:105A20000E94ABBCF80185858823E1F02FEF30E0C0
:105A3000D7010F942A5529E130E040E050E00F945F
:105A4000AA54922F832F692F782F77FF02C070E01E
:105A500060E06F3F710519F014F06FEF70E0F8012E
:105A6000848164CF9701A1E0BFEF0F94225529E113
:105A700030E040E050E00F94AA54BA01A90141502F
:105A80005F4F6F4F7F4F942F852FDDCF8B2D0E945F
:105A9000ABBC4ECF66246A94762C81149104A10489
:105AA000B104F1F0F80127803084032C000C440885
:105AB00055080E9454BF211431044104510409F4D3
:105AC000BDCE681979098A099B0962157305840599
:105AD000950508F0B3CEFFEF6F167F0609F057CE9D
:105AE0004FE7E41AF10855CE712C612C4ACE66249A
:105AF0006A94712C46CE1F93CF93DF9300D000D0D1
:105B0000CDB7DEB76130710509F46BC05CF4672B6B
:105B100009F45DC067E17DE088E39FE00F944223D4
:105B200080E04BC06230710571F06330710591F710
:105B30009093B80C8093B70C55275093BA0C4093B0
:105B4000B90C84E009C09093B80C8093B70C5093C3
:105B5000BA0C4093B90C83E00E94AEC0182F4FEFEF
:105B60005FEFBA0180E00E9419286093BC0970932E
:105B7000BD098093BE099093BF091123D9F062E05B
:105B80007DE081E99EE00F944223812F90E0B0E018
:105B9000A0E089839A83AB83BC8380E190E09E83FD
:105BA0008D83BE016F5F7F4F81E99EE00F945A00A5
:105BB0000F94432281E01111B3CF26960FB6F894CB
:105BC000DEBF0FBECDBFDF91CF911F91089590939F
:105BD000B80C8093B70C5093BA0C4093B90C81E089
:105BE000BBCF9093B80C8093B70C5093BA0C4093F2
:105BF000B90C82E0B1CFCF92EF92FF920F931F9337
:105C0000CF93DF9300D000D01F921F92CDB7DEB7A5
:105C10007C0109831A832B833C834D835E836F83CE
:105C200078876FE37BE088E39FE00F944223CE0107
:105C300001960E942A70898181112CC00B8101304C
:105C400089F128F010E00230F1F5CC2001F160E09C
:105C5000CE0101960E94F56BF70102811381892B19
:105C600081F0C8010E9415E5672B682B692B79F438
:105C70004FEF5FEFBA0180E00E941928AB01BC0131
:105C800003C040E050E0BA01C8010E94D4E481E0C2
:105C900090E02AC08031B0F58E30B8F58130A9F19E
:105CA0008230B9F162E37BE088E39FE00F94422306
:105CB000698188E39FE00E941BAD88E39FE00F9419
:105CC000432201E010E062E27BE088E39FE00F9472
:105CD0004223B80188E39FE00E9422AD88E39FE061
:105CE0000F94432290E080E028960FB6F894DEBF30
:105CF0000FBECDBFDF91CF911F910F91FF90EF901D
:105D0000CF9008958351843068F6F70102811381A2
:105D1000A8CF40E050E0BA01F70182819381B5CF6E
:105D20008F929F92AF92BF92CF92DF92EF92FF92AB
:105D30000F931F93CF93DF9300D000D01F921F9239
:105D4000CDB7DEB76D7F6130710509F4B7C0FC01D6
:105D5000E280F380E114F10409F4B0C08C01C701C2
:105D60000E9415E54B015C0161E070E0C7010E94F3
:105D70005BE581149104A104B10409F49FC020E003
:105D800030E04AE754E40F94A4530F9417566B0184
:105D90007C01C114D104E104F10409F48FC00E9414
:105DA00054BF681979098A099B096C157D058E0510
:105DB0009F0508F483C0F801A280B38070E060E022
:105DC000C5010E945BE520E030E048EC52E40F940E
:105DD000A4530F9417566B017C014FEF5FEFBA018C
:105DE00080E00E941928AB01BC01C5010E94D4E4E7
:105DF00019821A821B821C821D821E821F821886B3
:105E00008A81807F8A83F8016281738140E050E358
:105E1000CE0101960E94326BCE0101960E949E6DCA
:105E20004B015C0160E775E088E39FE00F94EB2293
:105E3000B501A40188E39FE00E9418AD6FE775E00B
:105E400088E39FE00F94EB22B701A60188E39FE06F
:105E50000E9418AD88E39FE00F944322C80CD91C20
:105E6000EA1CFB1C8A81807F86608A83CD82DE8269
:105E7000EF82F886F8016281738140E050E2CE0142
:105E800001960E941F6A63E875E088E39FE00F9423
:105E9000EB22B701A60188E39FE00E9418AD88E3DA
:105EA0009FE00F94432230E020E040E050E260E0C9
:105EB00070E0F801828193810E94408190E080E04F
:105EC00028960FB6F894DEBF0FBECDBFDF91CF91FD
:105ED0001F910F91FF90EF90DF90CF90BF90AF9008
:105EE0009F908F9008958F929F92AF92BF92CF9282
:105EF000DF92EF92FF920F931F93CF93DF937C017A
:105F00004A015901C091B209D091B309062F660F19
:105F1000110B209709F45CC088858F70863009F0DA
:105F200055C068E975E0CE010E9491AC6C0182E039
:105F30008816910449F06DE975E0E3E08E1691044E
:105F400029F0D0E0C0E006C061EA75E0CE010E9411
:105F500091ACEC01C114D104D9F1F60180858F70A8
:105F60008430B1F561857285A801C7010F94A259EB
:105F7000A80166EA75E0C7010F948459209779F16A
:105F800088858F70843059F569857A85A801C701A5
:105F90000F948459A80166EA75E0C7010F948459EB
:105FA000A114B10429F0A801B501C7010F948459C7
:105FB000C701DF91CF911F910F91FF90EF90DF907C
:105FC000CF90BF90AF909F908F900895D0E0C0E0A9
:105FD000A80169E374E1C7010F94804DC9CFF2E0D5
:105FE0008F16910481F083E08816910429F0609166
:105FF000B0097091B109CACFA80163E374E1C70188
:106000000F94624DC7CFA80160E374E1F8CFFF920F
:106010000F931F93CF93DF93CDB7DEB7C455D1094C
:106020000FB6F894DEBF0FBECDBF8C01F62EDC019B
:1060300016966C91FF2011F081E06827F8018481A9
:106040000E94ABBCF80187819085A185B285883E0E
:106050009340A105B10508F49BC065E373E188E3B3
:106060009FE00F94422360E373E188E39FE00F9485
:106070004223D80114966D917C9188E39FE00E94A1
:1060800022AD6BE273E188E39FE00F9442236F2D12
:1060900070E088E39FE00E9422AD88E39FE00F94C8
:1060A0004322FE01E55BFF4F8FE290E081939193E5
:1060B00088E0DF011D928A95E9F764E273E1CE0181
:1060C000855B9F4F0F943E4DF801828193810E9422
:1060D00017E8FF2009F469C06CE173E1853151F0E4
:1060E00065E173E1863131F069E073E18F3011F4DD
:1060F00061E173E1CE018F5B9F4F0F94524D809110
:10610000FD109091FE10059709F442C0D801129637
:10611000ED91FC910280F381E02D00811181011548
:106120001105B1F140E450E0B801CE0101960F94A1
:10613000A2596FE270E0CE0101960F946959892B44
:1061400041F4980143E050E060E4CE0101960E94E2
:10615000732F4FE350E0BE01655B7F4FCE01019688
:106160000F9484590E94AFAC882391F08091FD1068
:106170009091FE10069761F48091F810811108C08B
:1061800041E0BE016F5B7F4FCE0101960E9422C0AD
:10619000CC5ADF4F0FB6F894DEBF0FBECDBFDF91F4
:1061A000CF911F910F91FF90089565E073E18230C8
:1061B00009F4A0CF60E073E19DCFAF92BF92CF9280
:1061C000EF92FF920F931F93CF93DF9300D000D0F5
:1061D0001F921F92CDB7DEB75C0109831A832B8310
:1061E0003C834D835E836F8378876AE773E188E33E
:1061F0009FE00F944223CE0101960E942A70E11481
:10620000F10439F063E773E1C7010F94494D00973A
:1062100049F1F501028113810115110509F1898107
:10622000811163C08B81813009F467C068F18230CD
:1062300049F1082F10E060E573E188E39FE00F94D7
:10624000422360E473E188E39FE00F944223B801A6
:1062500088E39FE00E9422AD88E39FE00F944322F1
:1062600090E080E028960FB6F894DEBF0FBECDBF59
:10627000DF91CF911F910F91FF90EF90CF90BF9042
:10628000AF900895CC20D9F060E0CE0101960E9435
:10629000F56B892B09F44EC0C8010E9415E5672BE8
:1062A000682B692BF9F44FEF5FEFBA0180E00E9491
:1062B0001928AB01BC01C8010E94D4E413C0C80175
:1062C0000E9417E88E3019F050F4813059F460E0E4
:1062D000CE0101960E94F56B892B21F0DDCF835111
:1062E0008430A8F381E090E0BDCF8031F0F48E30AF
:1062F00098F6813089F28230E9F068E673E188E34C
:106300009FE00F9442236BE573E188E39FE00F94D5
:106310004223698188E39FE00E941BAD88E39FE0F0
:106320000F94432201E010E086CF8351843008F4BB
:10633000B3CFE3CF40E050E0BA01C8010E94D4E4FB
:1063400060E0C5010E940730CDCF4F925F926F92FF
:106350007F928F929F92AF92BF92CF92DF92FF92E5
:106360000F931F93CF93DF9300D000D01F921F9203
:10637000CDB7DEB76130710509F482C0FC016281DE
:1063800073816115710509F47BC08C0119821A8231
:106390001B821C821D821E821F8218868A81807F3A
:1063A0008A8340E050E2CE0101960E94326B60E0A9
:1063B000CE0101960E94F56B6C01F80182819381F8
:1063C0000E9415E52B013C01F801278130854185AC
:1063D0005285D6010F94D4542FEF30E040E050E0C6
:1063E0000F94885449015A010E9454BFFF24F3942A
:1063F00081149104A104B10461F06419750986093E
:106400009709FF24F394681579058A059B0508F41C
:10641000F12C411451046104710491F1F801878059
:106420009084A184B2840E9454BFF8018114910425
:10643000A104B10451F0641975098609970968151A
:1064400079058A059B0508F449C0A280B3804FEF07
:106450005FEFBA0180E00E941928AB01BC01C501C1
:106460000E94D4E4CD2861F0F80184810E94291BA8
:10647000F8019681891304C061E0C8010E940730C9
:1064800090E080E028960FB6F894DEBF0FBECDBF37
:10649000DF91CF911F910F91FF90DF90CF90BF9030
:1064A000AF909F908F907F906F905F904F900895E6
:1064B000FF20D9F060E0C8010E940730F801828116
:1064C00093810E943CEA892BD9F640E050E0BA0162
:1064D000F801828193810E94D4E4D2CF84810E940A
:1064E000291BF80196818913E3CFCD2849F2F801E1
:1064F00084810E94291BF80196818913C1CFF11074
:10650000BFCFBACFAF92BF92CF92DF92EF92FF92FE
:106510001F93CF93DF9300D000D0CDB7DEB76C01CF
:106520007C0110E08AE0A82EB12C133061F1F70154
:10653000828190E0B0E0A0E089839A83AB83BC8342
:10654000BE82AD82BE016F5F7F4F87E89EE00F94F1
:106550005A006EE274E10F9442231F5FFFEFEF1ABF
:10656000FF0A143011F726960FB6F894DEBF0FBE5F
:10657000CDBFDF91CF911F91FF90EF90DF90CF9033
:10658000BF90AF900895F601858190E0B0E0A0E063
:1065900089839A83AB83BC83BE82AD82BE016F5F69
:1065A0007F4F87E89EE00F945A006CE274E1D3CFEE
:1065B000FC01DC018D918111FDCF30E020E050E045
:1065C00040E08AE09191992301F1443051055CF556
:1065D0009E3271F42F3F310509F02CF5DB01A40F39
:1065E000B51F12962C934F5F5F4F30E020E0EACF4B
:1065F000829FD001839FB00D1124292F990F330B57
:10660000205331092A0F3B1FDDCF2F3F310509F001
:1066100054F4443051053CF4640F751FFB01228390
:1066200081E090E0089590E080E00895CF93DF93BB
:106630001F921F92CDB7DEB78091B1119091B21128
:10664000009711F48DEB91E1BE016F5F7F4F681BE6
:10665000790B072E000C880B990B0F900F90DF9190
:10666000CF9108954F925F926F927F929F92AF92D7
:10667000BF92CF92DF92EF92FF920F931F93CF932F
:10668000DF93CDB7DEB768970FB6F894DEBF0FBEC5
:10669000CDBFFC01198A1A8A1B8A1C8A1D8A1E8A90
:1066A0001F8A188E8A89807F8A8BA081B18110977A
:1066B00009F47AC08C91882309F476C00081118195
:1066C000D8019C91992309F443C09D3209F4DAC0A2
:1066D00090539A3028F00F5F1F4F11830083EECF45
:1066E000C801912CDC016D01C81AD90A2D91022E26
:1066F000000C330B205331092A303105A0F37F0100
:106700006EE270E0C8010F946959FC01009709F42A
:1067100048C0DC015D01AE1ABF0A11968C91119739
:10672000082E000C990BC09711960A9798F3818157
:10673000282F082E000C330B205331092A30310545
:1067400018F480330CF057C020E030E0A90108C0F5
:10675000912CD12CC12CD3CF29E030E040E050E087
:10676000AAE0B0E00F94C9542B013C012281822F92
:10677000022E000C990BC0978A30910570F42033DB
:106780000CF441C02A330CF042C0092E000CAA0BB5
:10679000BB0B480E591E6A1E7B1EA114B10409F0E2
:1067A00088C0CD2809F073C088E0FE017196DE0133
:1067B000199601900D928A95E1F729853A854B85C6
:1067C0005C856D857E858F85988968960FB6F8946F
:1067D000DEBF0FBECDBFDF91CF911F910F91FF9014
:1067E000EF90DF90CF90BF90AF909F907F906F9091
:1067F0005F904F9008958A330CF0AECF032E000CBB
:10680000440B550BADCF80E090E0DC01C2CF89E0B6
:1068100090E0A0E0B0E0BDCFB8E0CB16D1040CF022
:106820004DC0C8010F94FB4C9B01AC01A4E6B0E045
:106830000F94C954992041F07094609450944094FE
:10684000411C511C611C711C2A89207F26602A8BE7
:10685000460E571E681E791E4D8A5E8A6F8A788E94
:106860006CE270E0F701808191810F946959009783
:1068700021F4D7011D921C9297CF0196F7019183C5
:10688000808392CFC8010196992493942BCFC8019D
:106890000F94FB4CAB01BC01CE0141960E94096BE9
:1068A00029833A834B835C836D837E838F839887B0
:1068B000D7CFF3E0AF16B1040CF4AECFC8010F94FC
:1068C000D94C2A89207F27602A8B6D8B7E8B8F8BFA
:1068D000988FC6CFCF92DF92EF92FF920F931F93C4
:1068E000CF93DF93EC01A881B981109781F18C914E
:1068F000882369F108811981F8019081992351F069
:106900009D3241F090539A3028F00F5F1F4F19834A
:106910000883F0CFC8010F94FB4C6B017C016CE243
:1069200070E0C8010F946959009769F419821882C0
:10693000C701B601DF91CF911F910F91FF90EF90AA
:10694000DF90CF900895019699838883F1CFC12C71
:10695000D12C7601EDCF0097B1F1FC01DB01AC0148
:10696000405F5F4F80E090812FE9290F263098F437
:1069700097559295907F9C9321813FE9320F363055
:10698000B0F42755922B9D933296E417F50759F7EB
:1069900091E0892708952FEB290F263010F49753A3
:1069A000E8CF90539A3028F381E090E0E2CF3FEBBC
:1069B000320F363010F42753E5CF20532A3010F32E
:1069C00081E020E0DFCF80E008950097D1F0DC0186
:1069D0001696ED91FC913097A1F080858F708430F0
:1069E00021F481859285009771F40680F781E02D6E
:1069F000309739F080858F70843019F481859285C5
:106A0000089590E080E00895089508950895089508
:106A10000F931F93CF93DF93EC011D860A811B8197
:106A200070E060E0C8010E94A1E587FD44C08C834E
:106A30008C818150853410F080E28C8361E070E0BD
:106A4000C8010E94A1E587FD3BC08D838D818150E7
:106A5000853410F081E28D8362E070E0C8010E940D
:106A6000A1E5863490F58E8363E070E0C8010E9452
:106A7000A1E59C01215031092115344040F59A8748
:106A8000898764E070E0C8010E94A1E5813024E0BC
:106A9000920700F59C878B8765E070E0C8010E9433
:106AA000A1E518161906CCF498878F83DF91CF9152
:106AB0001F910F91089581958C8381E08D87B8CFC8
:106AC00081958D8381E08D87C1CF1E82CDCF1A86BF
:106AD0001986D7CF80E094E0DDCF80E197E2E4CF64
:106AE0000895CF93DF9300D000D01F921F92CDB7AF
:106AF000DEB7E1E7FEE0128A118A80E090E1958737
:106B0000848784E890E0948B838B81E0868780E0A3
:106B100090E2908B878787E7858B1C821B828DE2B2
:106B200092E09A838983FE83ED838FEF9FEF9887AE
:106B30008F8368E07BE087E89EE00F9442236091BA
:106B4000A8097091A909CE0101960E9475B381E749
:106B50009EE00E9436E068EF7AE087E89EE00F94BE
:106B6000422387E89EE00F9443220E9400CA2896A1
:106B70000FB6F894DEBF0FBECDBFDF91CF91089561
:106B8000EF92FF921F93CF93DF93192F7B01C82FB2
:106B9000D92FD7FF03C0D195C195D10961E08C2FC2
:106BA0000E94D9BC82E0E816F10499F460E08C2FD1
:106BB0000E94ABBC60EF7AE088E39FE00F94422331
:106BC00088E39FE0DF91CF911F91FF90EF900D94AC
:106BD0004322612FEF2851F46095661F6627661FD8
:106BE0008C2F0E94ABBC6CEE7AE0E6CF661F662766
:106BF000661F8C2F0E94ABBC67EE7AE0DDCFBF92A0
:106C0000CF92DF92EF92FF920F931F93CF93DF9378
:106C1000CDB7DEB72E970FB6F894DEBF0FBECDBF4F
:106C20002091FB103091FC10232B09F4A6C0209179
:106C3000FA102111A2C07C018091FA108F5F80931D
:106C4000FA108091F9108F5F8093F9100E9454BF61
:106C50000091B8091091B9092091BA093091BB0986
:106C6000601B710B820B930B6B30710581059105D5
:106C700008F479C083E0E816F104A9F00E9454BF3B
:106C80000091B4091091B5092091B6093091B70966
:106C9000601B710B820B930BBB24B394643671059C
:106CA0008105910508F4B12CE091FB10F091FC10E6
:106CB0000681178101151105C1F1F80180858F70DA
:106CC000863079F51987088770E060E0CE01089674
:106CD0000F944207B701CE0108960F94730A68EA31
:106CE00075E0C8010E9491ACFC01892BD1F0908520
:106CF0009F7095509230A8F4C680D780C114D104FB
:106D000081F0DA82C982B801CE0101960F94420760
:106D1000B701CE0101960F94730AF601C280D380A9
:106D2000EDCFF80102811381C5CFF3E0EF16F10436
:106D300051F00E9454BF6093B8097093B9098093D1
:106D4000BA099093BB09BB2051F00E9454BF6093D5
:106D5000B4097093B5098093B6099093B70910925E
:106D6000A50F1092A60F8091F91081508093F91011
:106D70008091FA1081508093FA102E960FB6F894F5
:106D8000DEBF0FBECDBFDF91CF911F910F91FF905E
:106D9000EF90DF90CF90BF900895A8950F94E529CC
:106DA00082E090E00E94FF350E94C895039734F07E
:106DB0000E9458C50E94C9D90E946ACD0D949614AC
:106DC000A89582E090E00C94FF358091F8108F5FD9
:106DD0008093F810A89583E090E00E94FF350F940F
:106DE000E5298091F81081508093F810089565ECA2
:106DF0007AE087E89EE00F94422362EB7AE087E82E
:106E00009EE00F94422364EA7AE087E89EE00F94C4
:106E100042236CE97AE087E89EE00F94422387E8FA
:106E20009EE00F9443226CE87AE087E89EE00F949E
:106E3000422360E87AE087E89EE00F94422363E70C
:106E40007AE087E89EE00F9442236EE57AE087E8D7
:106E50009EE00F9442236FE47AE087E89EE00F946F
:106E6000422367E47AE087E89EE00F94422366E3DA
:106E70007AE087E89EE00F94422360E17AE087E8B9
:106E80009EE00F94422363E07AE087E89EE00F944F
:106E9000422369EF79E087E89EE00F9442236AEE8F
:106EA00079E087E89EE00F94422362EE79E087E87C
:106EB0009EE00F94422366ED79E087E89EE00F9410
:106EC00042236CEB79E087E89EE00F9442236DE962
:106ED00079E087E89EE00F94422368E879E087E84C
:106EE0009EE00F9442236BE779E087E89EE00F94E1
:106EF00042236DE679E087E89EE00F94422361E645
:106F000079E087E89EE00F94422369E579E087E81D
:106F10009EE00F9442236EE479E087E89EE00F94B0
:106F2000422361E479E087E89EE00F94422369E31D
:106F300079E087E89EE00F9442236EE279E087E8EB
:106F40009EE00F9442236FE179E087E89EE00F9482
:106F5000422366E179E087E89EE00F94422368E0EF
:106F600079E087E89EE00F9442236AEF78E087E8B3
:106F70009EE00F9442236EEE78E087E89EE00F9447
:106F8000422366EE78E087E89EE00F94422363EDAB
:106F900078E087E89EE00F94422369EC78E087E888
:106FA0009EE00F94422387E89EE00D944322CF9306
:106FB000DF93EC0168ED72E188E39FE00F944223D8
:106FC00063ED72E188E39FE00F9442236C817D8141
:106FD00088E39FE00E9422AD6DEC72E188E39FE0C0
:106FE0000F94422388E39FE00F94432261E08C8159
:106FF0000E94D9BC6E818C810E94ABBC8A819B812E
:10700000009729F040E050E0BA010E94D4E4E88102
:10701000F9810484F585E02D62E0CE0119958A811D
:107020009B81009799F00E943CEA1816190674F4A7
:107030000A80DB81C02D4FEF5FEFBA0180E00E9434
:107040001928AB01BC01CE010E94D4E481E090E09C
:10705000DF91CF910895CF93DF93EC016AEA72E15B
:1070600088E39FE00F9442236C817D8188E39FE059
:107070000E9422AD68EA72E188E39FE00F94422308
:10708000EA81FB810280F381E02D6081718188E3D8
:107090009FE00F94EB2262EA72E188E39FE00F9495
:1070A000422388E39FE00F9443228A819B81892BAE
:1070B00009F451C08C819D81892B09F04CC0E88175
:1070C000F981008CF18DE02DCE011995813091056B
:1070D00029F0029759F061E08C811AC063E070E0FA
:1070E000CE010F943D1661E00E94D9BC61E08C8115
:1070F0000E94D9BC61E070E0CE010F943D1661E0C2
:107100000E94D9BC62E070E0CE010F943D1661E0B0
:107110000E94D9BC8091A100887F8093A1008091BA
:107120009100887F809391008091A100826080937C
:10713000A10080919100826080939100E881F981A3
:107140000484F585E02D62E0CE01199581E090E0A0
:10715000DF91CF91089590E080E0FACF2F923F9297
:107160004F925F926F927F928F929F92AF92BF9257
:10717000CF92DF92EF92FF920F931F93CF93DF9303
:10718000CDB7DEB760970FB6F894DEBF0FBECDBFA8
:107190009A838983DC011496ED91FC91309709F470
:1071A0005DC1868097808114910409F41DC1D401CA
:1071B000ED91FC91309709F413C18081882309F483
:1071C0000FC12FEF3FEFA9016CEA75E0C4010E94E7
:1071D0009B2022E030E040E050E069E276E0C4012C
:1071E0000E949B202FEF3FEFA9016DE975E0C401DC
:1071F0000E949B2060E375E0C4010E9491AC988BD3
:107200008F87009709F4ECC0FC0180858F70853072
:1072100009F0E6C0CF010E94ACAD833008F4E0C0B5
:1072200020E030E040EA51E460EB75E0C4010E94E8
:1072300066208C010E941C1C20E030E040EA51E4F2
:1072400064EB75E0C4010E9466206C010E941C1C66
:1072500020E030E040E050EC68EB75E0C4010E94B3
:1072600066207C010E941C1C20E030E040E85FE3C7
:1072700070E060E08F8598890E94DD1C2B013C0145
:1072800020E030E0A9010F943E53B12C87FF06C0E7
:1072900077FA709477F87094BB24B39420E030E0D0
:1072A000A90161E070E08F8598890E94DD1C6B83E5
:1072B0007C838D839E8320E030E0A90162E070E052
:1072C0008F8598890E94DD1C6F83788789879A87CC
:1072D00020E030E040EA50E463E070E08F85988978
:1072E0000E94DD1C6B877C878D879E878CE390E0F6
:1072F0000F94104B1C019801275F3F4FA701475F78
:107300005F4FB601675F7F4F1F92BF92FA85FF9371
:1073100089858F9398859F93AF81AF93AB80BC8015
:10732000CD80DE8083017201C1010F94ED26C10181
:10733000032C000CAA0BBB0BEF85F8898187928781
:10734000A387B48761E070E0C1010F944E2620E06E
:1073500030E04AE754E46B857C858D859E850F94EB
:10736000A4530F941056AF85B88919968D919C91AE
:107370000F94A0266DEF7FE088E39FE00F944223F7
:10738000B301A20188E39FE00E946DB16BEB75E051
:1073900088E39FE00F94EB224B815C816D817E81BD
:1073A00088E39FE00E946DB16FEB75E088E39FE09A
:1073B0000F94EB223F81288599858A85432F522F90
:1073C000692F782F88E39FE00E946DB188E39FE0EA
:1073D0000F9443220F900F900F900F900F900F90EB
:1073E000F40182809380DFCE62EF7FE088E39FE04C
:1073F0000F94422388E39FE00F94432240E050E043
:10740000BA01A981BA8112968D919C910E94D4E40F
:10741000A981BA81ED91FC9111970484F585E02D45
:1074200062E0CD01199581E090E060960FB6F89486
:10743000DEBF0FBECDBFDF91CF911F910F91FF90A7
:10744000EF90DF90CF90BF90AF909F908F907F9004
:107450006F905F904F903F902F9008956EED7FE07A
:1074600088E39FE00F94422388E39FE00F94432238
:1074700090E080E0DACFCF93DF93EC010E940835F3
:1074800063EC75E088E39FE00F94472261E08C8114
:107490000E94D9BC61E08D810E94D9BC6D858C8130
:1074A0000E94ABBC6D858D810E94ABBC60E08E817B
:1074B0000E94D9BC40E050E0BA018A819B810E94C1
:1074C000D4E440E050E061E070E08A819B810E945A
:1074D0004BE640E050E062E070E08A819B810E94D0
:1074E0004BE6E881F9810484F585E02D62E0CE0168
:1074F000199582E08093000281E090E0DF91CF91C6
:1075000008956F927F928F929F92AF92BF92CF9287
:10751000DF92EF92FF920F931F93CF93DF933C0183
:10752000DC0114968D919C911597892B71F412961C
:10753000CD91DC9184E190E00F94104BBC01CE0121
:107540000E9491E4E3019D838C83F301C481D58182
:10755000209769F46EEE7CE081E99EE00F9442236F
:1075600081E99EE00F94432290E080E0A7C24FEFB4
:107570005FEFBA0180E00E9419286E837F838887BD
:107580009987D3011496ED90FC901597E114F104BE
:10759000D1F01296ED91FC913097A9F0C481D5817C
:1075A000209789F088858F70853069F4CE010E941C
:1075B000ACAD823040F00091AB091091AC090115DF
:1075C000110509F08CC061EB7CE081E99EE00F942D
:1075D000422361E070E0E3018C819D81892B11F4ED
:1075E00070E060E081E99EE00E9422AD6FEA7CE0FD
:1075F00081E99EE00F94422361E070E0F301828113
:107600009381892B11F470E060E081E99EE00E9493
:1076100022AD6DEA7CE081E99EE00F944223D30124
:107620001296ED91FC9161E070E084819581892B47
:1076300011F470E060E081E99EE00E9422AD6BEA07
:107640007CE081E99EE00F944223E301EA81FB8123
:107650000480F581E02D80858F7061E070E08530D9
:1076600011F470E060E081E99EE00E9422AD69EAD9
:107670007CE081E99EE00F944223D3011296ED91C4
:10768000FC91848195810E94ACAD61E070E0823014
:1076900010F070E060E081E99EE00E9422AD81E997
:1076A0009EE00F94432266EC7CE081E99EE00F941B
:1076B000422381E99EE00F944322D301ED91FC9196
:1076C0000484F585E02D61E0C3011995E301E881AB
:1076D000F9810084F185E02DC301199545CF61E062
:1076E000CE010E9409ADEC0188858F70843029F4A9
:1076F00069857A856115710539F461E97CE081E974
:107700009EE00F944223CBCFC8010E9491AC8C0124
:10771000009769F46FE67CE081E99EE00F944223D4
:1077200069857A8581E99EE00F94EB22B8CF6FECF2
:1077300075E00E9491AC009709F4D2C0EC01288555
:107740002F70243009F0CCC0C984DA84D0E0C0E0C6
:10775000C114D10409F4B7C0BE016553744FC6010A
:107760000F94494D892B09F0A9C0FE01E153F44F54
:1077700025913491922F832FF7019283838366EDB5
:1077800075E0C8010E9491ACE301EC81FD81009796
:1077900009F4AEC0DC0118962C9118972F70223096
:1077A00009F0A6C019968D919D910D90BC91A02DC8
:1077B0000097A105B10509F49BC0918380834081A6
:1077C0005181052E000C660B770B228186EB9BE026
:1077D0000F944E246BED75E0C8010E9491AC7C01C2
:1077E000F301C481D581009709F488C0DC011896A3
:1077F0008C918F70863009F081C060EE75E0C70112
:107800000E9491AC9B878A8765EE75E0C7010E9454
:1078100091AC9D878C8769EE75E0C7010E9491ACA1
:107820009F878E876FEE75E0C7010E9491AC998BA0
:10783000888B64EF75E0C7010E9491AC009709F452
:107840005AC0FC01818592859D838C836AEF75E027
:10785000C8010E9491AC9B8B8A8B892B09F40CC1C7
:1078600069E57CE088E39FE00F94422388E39FE092
:107870000F944322D3011496ED91FC910288F38971
:10788000E02DC681D781209709F441C06EEF75E0E5
:10789000CE010E9491AC009769F0FC0120852F7009
:1078A000213041F48185882329F068817981C301E1
:1078B0000E9427230A80DB81C02DE5CF2696C8349D
:1078C000D10509F045CF6EEA7BE088E39FE00F9495
:1078D000422388E39FE00F94432296E080E04CCF60
:1078E00086E090E0D70113969C938E93129747CF32
:1078F00080E895E262CF88EE93E0A6CF1B861A86D9
:1079000088EE93E09D838C831D861C869FCF63E465
:107910007CE088E39FE00F94422388E39FE00F948C
:107920004322D3011496ED91FC910288F389E02D56
:10793000E680F780E114F10409F478C06BE575E0A6
:10794000C7010E9491AC009709F465C067E076E03A
:107950000E9491AC8C01009709F45DC0EC01888510
:107960008F70823009F04BC0C984DA84D301149639
:10797000ED91FC910288F389E02D309709F453C012
:10798000C681D78146010D2C000CAA08BB082097A0
:1079900009F449C06BE076E0CE010E9491AC0097FB
:1079A000F1F1FC0120852F702230C9F58185928587
:1079B000A385B48588159905AA05BB0581F562E202
:1079C0007CE088E39FE00F9442236881798188E31B
:1079D0009FE00F94EB2263E17CE088E39FE00F944B
:1079E0004223B60188E39FE00E9422AD88E39FE036
:1079F0000F94432268817981C3010E942723F801F3
:107A000080858F70843039F4D80119966D917C91FE
:107A1000C3010E942723E701EA80FB808BCF0A8005
:107A2000DB81C02DB4CF70E060E0E6CF69E27CE09E
:107A300088E39FE00F94422388E39FE00F94432262
:107A4000D3011296ED91FC9162E0848195810E94B0
:107A500009AD009789F0FC01C681D781209761F0BC
:107A6000CE010E943C1C882319F0CE010E9402BB6B
:107A70000A80DB81C02DF2CF69ED7CE087E89EE0D3
:107A80000F944223D3011296ED91FC910280F38171
:107A9000E02D6081718187E89EE00F94EB2287E8FA
:107AA0009EE00F944322E301E881F9810484F58587
:107AB000E02D62E0C301199581E090E0DF91CF9164
:107AC0001F910F91FF90EF90DF90CF90BF90AF90FC
:107AD0009F908F907F906F900895CF93DF93EC01EC
:107AE00069E47BE088E39FE00F944223EA81FB8115
:107AF0000280F381E02D6081718188E39FE00F9423
:107B0000EB2288E39FE00F944322E881F98104840B
:107B1000F585E02D62E0CE01199581E090E0DF91DE
:107B2000CF910895DC01ED91FC910484F585E02D61
:107B300062E0199581E090E008952F923F924F9274
:107B40005F926F927F928F929F92AF92BF92CF92ED
:107B5000DF92EF92FF920F931F93CF93DF93CDB7F6
:107B6000DEB7CB57D1090FB6F894DEBF0FBECDBF3D
:107B7000E296EFAEE297E396FFAEE397E4960FAF9F
:107B8000E497E5961FAFE597E6962FAFE697E79661
:107B90003FAFE797E8964FAFE897E9965FAFE99771
:107BA0000097B9F124012B2CEC96AFAEEC97EB9635
:107BB000DFAEEB97EA96CFAEEA97362E8C01809136
:107BC0001E02893020F480911D028930C0F0C80166
:107BD0000E94B6B47C01892B91F06FE076E088E3D7
:107BE0009FE00F94EB22B70188E39FE00F94EB2214
:107BF00088E39FE00F944322C7010F94AC4BF80138
:107C000080858F70843009F45FC128F4882309F4DB
:107C100064C180E02FC0853009F446C08630C9F7C2
:107C200068EA75E0C8010E9491AC3C01009709F434
:107C300076C0912C812CB12CA12CD12CC12CE29698
:107C4000EFACE297E396FFACE397E4960FADE497D1
:107C5000E5961FADE597E6962FADE697E7963FAD23
:107C6000E797E8964FADE897E9965FADE997632D02
:107C70000E949D3DC558DF4F0FB6F894DEBF0FBE82
:107C8000CDBFDF91CF911F910F91FF90EF90DF90CB
:107C9000CF90BF90AF909F908F907F906F905F90AC
:107CA0004F903F902F9008958091F9108F5F8093AF
:107CB000F910668077806114710459F14201EC96E5
:107CC000AFACEC97B22CEA96CFACEA97EB96DFAC70
:107CD000EB97E296EFACE297E396FFACE397E4967E
:107CE0000FADE497E5961FADE597E6962FADE697C5
:107CF000E7963FADE797E8964FADE897E9965FAD19
:107D0000E997632DC3010E949D3DF301628073805A
:107D1000D2CF8091F91081508093F9107ACF65E12C
:107D200076E0C8010E9491AC2C016AE176E0C801BE
:107D30000E9491AC7C016FE176E0C8010E9491AC99
:107D4000332039F0F1E03F1609F49FC0D12CC12C4B
:107D50000CC063E276E0C8010E9491AC3C0168E28D
:107D600076E0C8010E9491AC6C016114710409F4C1
:107D70003801C114D10409F468014114510431F4EB
:107D8000EA964FACEA97EB965FACEB97E114F104FF
:107D900021F4EC96EFACEC97F22C6114710409F429
:107DA000A5C0F30180858F70843009F09FC0618485
:107DB0007284C114D10409F49CC0F60180858F70CF
:107DC000843009F096C0C184D28410E000E04114F0
:107DD000510409F4F3C06114710409F4B1C066E8F8
:107DE00074E188E39FE00F944223F201618572857C
:107DF00088E39FE00F94EB2261E874E188E39FE061
:107E00000F944223B30188E39FE00F94EB2288E3B1
:107E10009FE00F944322CE018F589F4F0E942A70FB
:107E2000E114F10409F0D3C0F20180858F70843031
:107E300009F083C14091FF10509100116185728556
:107E4000CE0101960E9463E8CE0101960E9484E46F
:107E50008823B1F00E9416336B01683C71050CF069
:107E600083C060E474E181E99EE00F944223B6018F
:107E700081E99EE00E9422AD81E99EE00F944322B9
:107E8000CE0101960E9400E958C16DE276E0C8017A
:107E90000E9491AC3C0162E376E0C8010E9491AC83
:107EA0006C016114710409F04AC163E276E0C80113
:107EB0000E9491AC3C01C114D10409F450CF892B2C
:107EC00009F05BCF380159CFD12CC12C712C612C1A
:107ED000F12CE12C512C412C48CFD12CC12C712CF0
:107EE000612CF12CE12C512C412C47CF712C612CB1
:107EF00060CF00E020E030E340E150E0BE016F5988
:107F00007F4FCE018F589F4F0E940A6E6C01E496FE
:107F10000FADE49710E00115110509F058CFE29676
:107F20008FADE297811109C0E3968FADE3978F7013
:107F300009F44DCF02E010E04ACF01E010E047CF56
:107F400067E774E188E39FE00F944223F2016185C3
:107F5000728588E39FE00F94EB2262E774E188E387
:107F60009FE00F94422357CF6114710431F0B301A5
:107F7000CE0101960E94F5B483CFA12CC12CF12C27
:107F8000E12CE2960FADE297E3961FADE397E496FE
:107F90002FADE497E5963FADE597E6964FADE697B2
:107FA000E7965FADE797E8966FADE897E9967FAD06
:107FB000E997CE0101960E944CEB62CFE114F104E7
:107FC00009F4BBC0C114D10409F4B7C004C0C11482
:107FD000D10409F429CFF70180858F70843009F02E
:107FE000A8C08185928525961FAE1EAE259748EEC6
:107FF00053E060E070E029964CAF5DAF6EAF7FAFAD
:10800000299723E432E023963FAF2EAF23972F9694
:108010009FAF8EAF2F9761961FAE1EAE619763968E
:108020001FAE1EAE639765961FAE1EAE6597679630
:108030001FAE1EAE679769961FAF0EAF69976A961F
:108040001FAE6A9740E450E0BE016F5F7F4FCE01E4
:108050008F5B9F4F0E9460AE21E030E02C0F3D1FF0
:10806000820F931FFC0110826AE674E188E39FE0AF
:108070000F944223F7016185728588E39FE00F9496
:10808000EB2267E376E088E39FE00F94EB22BE01EA
:108090006F5F7F4F88E39FE00F94EB2265E674E10A
:1080A00088E39FE00F944223B60188E39FE00F949A
:1080B000EB2288E39FE00F9443220E94AFAC882319
:1080C000C1F18091F810811134C06FE270E0CE01EF
:1080D00001960F946959892B51F4F7012185328556
:1080E00043E050E060E4CE0101960E94732F6EE5FC
:1080F00074E188E39FE00F944223BE016F5F7F4FDE
:1081000088E39FE00F94EB2269E574E188E39FE048
:108110000F944223B60188E39FE00F94EB2288E39B
:108120009FE00F94432241E0B601CE0101960E94E8
:1081300022C04114510409F077CE81E09BCD892BF8
:1081400009F01BCE0CCE8F929F92AF92BF92CF922E
:10815000DF92EF92FF920F931F93CF93DF9300D0A4
:1081600000D01F921F92CDB7DEB7DC011296ED91C1
:10817000FC91309709F468C024813581232B09F4E0
:1081800063C08C01662309F472C00E94681FE62E4A
:10819000B72E6C01D8011296ED91FC910280F3810B
:1081A000E02D6081718181E99EE00F94EB2266E30E
:1081B00072E181E99EE00F94422381E99EE00F94F1
:1081C000432220E030E0A9016E2D7B2DC6010F94E3
:1081D000465687FD39C06AE272E181E99EE00F945C
:1081E00042234E2D5B2DB60181E99EE00E946DB1C8
:1081F00081E99EE00F944322D8011296ED91FC9103
:1082000061E0848195810E9409AD19821A821B82E6
:108210001C822A81207F2760F22E2E2D4E2D5B2D71
:10822000B6014D835E836F837887912C812CB12CAE
:10823000A12CD12CC12CE9800B811C813E814F8166
:1082400058856FEF0E949D3D28960FB6F894DEBFCB
:108250000FBECDBFDF91CF911F910F91FF90EF9097
:10826000DF90CF90BF90AF909F908F900895028045
:10827000F381E02D6081718187E89EE00F94EB220D
:1082800063E472E187E89EE00F94422387E89EE072
:1082900028960FB6F894DEBF0FBECDBFDF91CF9109
:1082A0001F910F91FF90EF90DF90CF90BF90AF9014
:1082B0009F908F900D9443224F925F926F927F9286
:1082C0008F929F92AF92BF92CF92DF92EF92FF92E6
:1082D0000F931F93CF93DF93CDB7DEB7E8970FB619
:1082E000F894DEBF0FBECDBF09AB1AAB2BAB3CABD6
:1082F0004DAB5EAB6FAB78AFDC011496ED91FC91AA
:10830000309719F490E080E0C9C020813181232B9F
:10831000C9F33C01DC01ED91FC910284F385E02D71
:108320001995029779F78BA9E82EF12C19A9112339
:1083300021F0E114F10409F431C1823009F4D7C00D
:10834000A8F4882309F4D3C08130A9F066E572E16E
:1083500088E39FE00F944223B70188E39FE00E94E7
:1083600022AD88E39FE00F944322CCCF833009F401
:1083700047C0893059F7D3011296ED91FC9161E025
:10838000848195810E9409AD2C0119A61AA61BA60D
:108390001CA61DA61EA61FA618AA8AA5807F8AA7AE
:1083A00019A761E0CE0189960E94C56A29A33AA364
:1083B0004BA35CA36DA37EA38FA398A71150163186
:1083C00008F0FDC1E12FF0E08827E651FE4B8F4F0A
:1083D0000D9413551443D242DF43DF43DF43DF43A1
:1083E000DF43DF43DF434343A343DF43DF43144320
:1083F0001443DF43DF43DF43144314431443144364
:108400008AA98F7009F47ECFCE01C1960E94146DA7
:10841000D3011496ED91FC916683778380879187D1
:108420006CE972E188E39FE00F944223D301129636
:10843000ED91FC910280F381E02D6081718188E3F0
:108440009FE00F94EB226EE872E188E39FE00F94C7
:108450004223D3011496ED91FC91468157816085AA
:10846000718588E39FE00E946DB188E39FE00F94DF
:108470004322F301E480F5800E9454BFD701529655
:108480006D937D938D939C935597D3011496ED91A5
:10849000FC918689811119C081E090E0E8960FB6C1
:1084A000F894DEBF0FBECDBFDF91CF911F910F912A
:1084B000FF90EF90DF90CF90BF90AF909F908F9004
:1084C0007F906F905F904F900895168A60E0C3018F
:1084D0000E94A340D3011496ED91FC9180E090E0BE
:1084E000A0E0B0EC86879787A08BB18BD5CF8AA907
:1084F0008F7009F407CFCE01C1960E94146DD3018D
:108500001496ED91FC91628773878487958768E85C
:1085100072E188E39FE00F944223D3011296ED911C
:10852000FC910280F381E02D6081718188E39FE0FE
:108530000F94EB226DE772E188E39FE00F944223F2
:10854000D3011496ED91FC91428553856485758520
:1085500088E39FE00E946DB188E39FE00F9443227F
:10856000D3011296ED91FC9162E0848195810E9485
:1085700009AD009709F490CF912C812CB12CA12C3E
:10858000D12CC12CE9A8FAA80BA91CA92DA93EA998
:108590004FA958AD6FEF0E949D3D7ECFEE24E3942E
:1085A000F12CE9CE8091FD109091FE100597F1F02D
:1085B00019821A821B821C821D821E821F821886CB
:1085C0008A81807F8A836BE0CE0101960E94E76AF0
:1085D000912C812CB12CA12CD12CC12C79018A0198
:1085E0009B01AC016FEFC2010E949D3D912C812C3B
:1085F000B12CA12CD12CC12CE9A4FAA40BA51CA54B
:108600002DA53EA54FA558A96FEFC2010E949D3D23
:1086100030E020E040E050E460E070E0F30182816F
:1086200093810E94408138CF19821A821B821C825A
:108630001D821E821F8218868A81807F8A8340E085
:1086400051E060E070E0D30112968D919C910E9400
:108650009DE6672B682B692BA1F06BE0CE0101969C
:108660000E94E76A912C812CB12CA12CD12CC12C19
:1086700079018A019B01AC016FEFC2010E949D3D0F
:10868000BBCF6AE0EBCF8091FD109091FE10059773
:1086900091F061E0D30112968D919C910E94F8E7D0
:1086A00030E020E040E050E160E070E0F3018281E2
:1086B00093810E94408140E050E061E070E0D3018E
:1086C00012968D919C910E9474E6912C812CB12C74
:1086D000A12CD12CC12CE9A4FAA40BA51CA52DA575
:1086E0003EA54FA558A96FEFC2010E949D3DD30141
:1086F000ED91FC910288F389E02DC3011995892B36
:1087000009F4E8CE19821A821B821C821D821E8205
:108710001F8218868A81807F8A8361E0CE0101965C
:108720000E94E76A29873A874B875C876D877E8737
:108730008F87988B79018A019B01AC016FEFC20191
:108740000E949D3DC7CE912C812CB12CA12CD12C07
:10875000C12CE9A4FAA40BA51CA52DA53EA54FA5E7
:1087600058A96FEFC2010E949D3DD301ED91FC918C
:108770000288F389E02DC3011995892B09F08CCE6D
:1087800019861A861B861C861D861E861F86188AD9
:108790008A85807F8A8762E0CE0109960E94E76A17
:1087A00029833A834B835C836D837E838F83988791
:1087B00079018A019B01AC016FEFC201ECCE6BE63F
:1087C00072E188E39FE00F94422369A988E39FE068
:1087D0000E941BAD88E39FE00F944322B7CD2F92F8
:1087E0003F924F925F926F927F928F929F92AF9241
:1087F000BF92CF92DF92EF92FF920F931F93CF938E
:10880000DF93CDB7DEB764970FB6F894DEBF0FBE27
:10881000CDBF1C01DC0114968D919C911597892B7D
:1088200099F41296ED91FC91FA83E98389E190E045
:108830000F94104BBC0189819A810E9491E4D1016F
:1088400015969C938E931497F1010481158101155F
:10885000110569F46BEC71E181E99EE00F9442230C
:1088600081E99EE00F94432290E080E092C3D8011A
:108870001D921C920280F381E02DFC8BEB8B3097D4
:1088800091F0848195819A838983009761F0DC015E
:1088900018968C9118978F70853029F4CD010E941D
:1088A000ACAD811186C061E971E181E99EE00F9470
:1088B000422361E070E0F10184819581892B11F4FC
:1088C00070E060E081E99EE00E9422AD6FE871E116
:1088D00081E99EE00F94422361E070E0D10112969D
:1088E0008D919C91892B11F470E060E081E99EE00C
:1088F0000E9422AD6DE871E181E99EE00F94422370
:10890000D1011296ED91FC9161E070E08481958136
:10891000892B11F470E060E081E99EE00E9422ADB5
:108920006BE871E181E99EE00F944223D101129638
:10893000ED91FC910480F581E02D80858F7061E0E0
:1089400070E0853011F470E060E081E99EE00E9403
:1089500022AD69E871E181E99EE00F944223D101E3
:108960001296ED91FC91848195810E94ACAD61E0FD
:1089700070E0823010F070E060E081E99EE00E94DB
:1089800022AD81E99EE00F94432265EA71E181E91D
:108990009EE00F94422381E99EE00F944322D1018F
:1089A000ED91FC910484F585E02D61E0C1011995FC
:1089B0005BCF60E089819A810E9409AD9F838E839D
:1089C000009729F0FC0180858F70853039F06FE6C3
:1089D00071E181E99EE00F944223D3CF8E819F8184
:1089E0000E94ACAD8150883008F0A3C1E82FF0E0C0
:1089F0008827E250FB4B8F4F0D9413556A46404633
:108A000013468E45764576455F45064567E08E817F
:108A10009F810E9409ADFC0190859F70933009F001
:108A200041C04184528463847484F1E0FD8366E034
:108A30008E819F810E9409ADFC0190859F709330CB
:108A400009F045C081859285A385B48589839A8381
:108A5000AB83BC8391E09D8364E08E819F810E9403
:108A600009ADFC0190859F70933009F050C061857D
:108A70007285838594850F9417564B0163E08E8130
:108A80009F810E9409ADFC0180858F70833009F0C1
:108A900060C081859285A385B4858A879B87AC87D2
:108AA000BD8764C0923059F4618572858385948551
:108AB0000F9445532B013C0181E08D83B8CF412CAD
:108AC000512C8FE7682E83E4782E1D82B0CF923030
:108AD000C9F461857285838594850F9445536983B4
:108AE0007A838B839C83A1E0AD83B6CF412C512C3C
:108AF000BFE76B2EB3E47B2E19821A821B821C8285
:108B00001D82AACF19821A821B821C82A5CF9230A5
:108B1000C1F481849284A384B484B0CFF0EC8F2E0E
:108B2000F7E29F2EF9E0AF2EB12C412C512CAFE78C
:108B30006A2EA3E47A2E19821A821B821C821D825D
:108B40009DCFE0EC8E2EE7E29E2EE9E0AE2EB12C1A
:108B500095CF823009F082C06185728583859485C6
:108B60000F9445536A877B878C879D8762E08E814F
:108B70009F810E9409ADFC0180858F70833009F0D0
:108B800072C091859E87A285AF87B385B88B848597
:108B9000898B61E08E819F810E9409ADFC018085F7
:108BA0008F70833009F08BC0C184D284E384F48455
:108BB00060E08E819F810E9409ADFC0180858F70ED
:108BC000833009F0A9C081859285A385B4858E8301
:108BD0009F83A887B98720E030E0A9016E817F815B
:108BE000888599850F943E5387FFD0C08E819F81E1
:108BF000A885B985B0588E839F83A887B98791E0EF
:108C00009A8BAB89BC891696ED91FC9180858F700B
:108C1000823009F4BDC0833009F4D4C180E090E013
:108C2000A0EAB1E4D3C160EC862E67E2962E69E03B
:108C3000A62EB12C80E090E0A0EAB0E48A879B8762
:108C4000AC87BD87412C512C7FE7672E73E4772ECC
:108C500019821A821B821C821D8288CF80E090E0DC
:108C6000A0EAB0E41ACF823029F561857285838548
:108C700094850F9445536E877F87888B998B89CF16
:108C800040EC842E47E2942E49E0A42EB12C80E0E3
:108C900090E0A0EAB0E48A879B87AC87BD87412C2F
:108CA000512C5FE7652E53E4752E19821A821B82C0
:108CB0001C821D821E861F86188A198A6ACF8230FE
:108CC00039F561857285838594850F9445536B01D1
:108CD0007C016ECF20EC822E27E2922E29E0A22E7C
:108CE000B12C80E090E0A0EAB0E48A879B87AC8753
:108CF000BD87412C512C3FE7632E33E4732E19823C
:108D00001A821B821C821D821E861F86188A198A5F
:108D1000C12CD12C76014CCF823091F561857285C2
:108D2000838594850F9445536E837F8388879987C5
:108D300052CF80EC882E87E2982E89E0A82EB12CA5
:108D400080E090E0A0EAB0E48A879B87AC87BD878B
:108D5000412C512C9FE7692E93E4792E19821A82B7
:108D60001B821C821D821A8A1E861F86188A198AF7
:108D7000C12CD12C7601CE82DF82E886F98641CFE4
:108D80001A8A1E821F82188619863BCF1A8A39CF0B
:108D900061857285838594850F944553F8016287B8
:108DA000738784879587D80116961D921D921D9210
:108DB0001C921997F80112821382148215820E9464
:108DC00054BFD80152966D937D938D939C93559784
:108DD000D1011496ED91FC9181E0868B908E878A6B
:108DE00061E0C1010E94A340F10104811581D80115
:108DF0008D919C9166E571E1892B09F0EACD8CE3B8
:108E000090E00F94104B9C8B8B8B9801265F3F4F0B
:108E1000A8014E5F5F4FB8016A5F7F4F1F92BA890A
:108E2000BF93E989EF93F889FF938F858F939E8590
:108E30009F9356016701EE80FF80088519858B8915
:108E40009C890F94ED26D1011496ED91FC918B89AC
:108E50009C89918380830F900F900F900F900F90BB
:108E60000F90009709F491CD61E070E00F944E26C9
:108E7000D1011496ED90FC90BD81BB2309F44AC04A
:108E8000A301920169817A818B819C810F9446565E
:108E900087FF40C0F7010190F081E02DFF83EE8352
:108EA00089819A81AB81BC8182AB93ABA4ABB5AB1A
:108EB00046AA57AA60AE71AE82AD882359F1068DDD
:108EC000178DF80180809180A280B380A501940164
:108ED000C301B2010F943E5387FF7EC0D8014D926B
:108EE0005D926D927C921397AE81BF8196968D9024
:108EF0009D90AD90BC909997A5019401C301B201DA
:108F00000F943E5387FF7DC0EE81FF8146A257A29A
:108F100060A671A620E030E04AE754E46A857B85CC
:108F20008C859D850F94A4530F941056D7018D9175
:108F30009C910F94A02667EB71E187E89EE00F9467
:108F40004223D1011296ED91FC910280F381E02D34
:108F50006081718187E89EE00F94EB2287E89EE0B4
:108F60000F944322D1011496ED91FC9180E090E0A2
:108F7000A0E0B0EC86879787A08BB18BD101ED91F3
:108F8000FC910484F585E02D62E0C101199581E032
:108F900090E064960FB6F894DEBF0FBECDBFDF91B0
:108FA000CF911F910F91FF90EF90DF90CF90BF90E6
:108FB000AF909F908F907F906F905F904F903F9079
:108FC0002F90089581859285A385B485F8018287C5
:108FD0009387A487B587E7CEA501940169817A813B
:108FE0008B819C810F94465618160CF07DCF898199
:108FF0009A81AB81BC81F80180839183A283B38382
:1090000073CFA501940169817A818B819C810F9432
:10901000465618160CF07ECF89819A81AB81BC81AF
:10902000EE81FF8186A397A3A0A7B1A773CF4F922C
:109030005F926F927F928F929F92AF92BF92CF92E8
:10904000DF92EF92FF920F931F93CF93DF93CDB7F1
:10905000DEB760970FB6F894DEBF0FBECDBF6130AC
:10906000710509F4DBC1DC011496ED91FC91309798
:10907000C9F481E090E060960FB6F894DEBF0FBEB1
:10908000CDBFDF91CF911F910F91FF90EF90DF90B7
:10909000CF90BF90AF909F908F907F906F905F9098
:1090A0004F90089520813181232B19F33C01DC017D
:1090B000ED91FC910284F385E02D19950297C9F694
:1090C000F301E280F380E114F10499F2C7010E94F8
:1090D00017E8823071F240E051E060E070E0C701D3
:1090E0000E949DE6672B682B692B19F6D301149615
:1090F000ED91FC9180819181FC0122AD222309F444
:1091000055C10F94B024882309F450C1D30114969B
:10911000ED91FC9186898823A1F0C3010E94681F0C
:109120006B017C0120E030E0A9010F94465687FDD9
:1091300008C0D3011496ED91FC91C282D382E482DF
:10914000F5826AE072E188E39FE00F944223D30145
:109150001296ED91FC910280F381E02D6081718186
:1091600088E39FE00F94EB2264E072E188E39FE0E4
:109170000F944223D3011496ED91FC9142855385BF
:109180006485758588E39FE00E946DB16FEF71E1A2
:1091900088E39FE00F944223D3011496ED91FC9154
:1091A000468157816085718588E39FE00E946DB19B
:1091B0006AE376E088E39FE00F94EB22D3011496F4
:1091C000ED91FC91428153816481758188E39FE038
:1091D0000E946DB16BEF71E188E39FE00F94422331
:1091E000D3011496ED91FC910190F081E02D408126
:1091F00051816281738188E39FE00E946DB167EFC6
:1092000071E188E39FE00F944223D3011496ED911E
:10921000FC910190F081E02D448155816681778138
:1092200088E39FE00E946DB163EF71E188E39FE006
:109230000F944223D3011496ED91FC910190F0819B
:10924000E02D408551856285738588E39FE00E940B
:109250006DB1D3011496ED91FC918689882331F08C
:109260006CEE71E188E39FE00F94422388E39FE076
:109270000F944322F301E480F580D70156968C9138
:109280008111F7CE0281138161E0F801848195811B
:109290000E9409AD2C0120E030E0A901D7011E9603
:1092A0006D917D918D919C9151970F943E538111B9
:1092B0000CC020E030E0A901F70162817381848154
:1092C00095810F94465618165CF040E050E061E03E
:1092D00070E0C8010E949DE6672B682B692B31F175
:1092E00019861A861B861C861D861E861F86188A6E
:1092F0008A85807F8A8761E0CE0109960E94E76AAD
:1093000029833A834B835C836D837E838F83988725
:10931000912C812CB12CA12CD12CC12C79018A014A
:109320009B01AC016FEFC2010E949D3D40E050E007
:1093300061E070E0D30112968D919C910E944BE602
:10934000D3011496ED91FC91328163815481458162
:1093500019861A861B861C868A85807F8760F82E70
:109360008A87232F832F962FA52FB42F8D879E8733
:10937000AF87B88B912C812CB12CA12CD12CC12C76
:10938000E9840B851C853E854F8558896FEFC201A6
:109390000E949D3DD3011496ED91FC9182819381B1
:1093A000A481B58186879787A08BB18BD301149652
:1093B000ED91FC91868981115CCE8789908D009713
:1093C00009F457CE28EE33E0829F2001839F500C92
:1093D000929F500C11240E9454BFD3011496ED911A
:1093E000FC914114510499F06201F12CE12C0289A5
:1093F000138924893589AB01BC01401B510B620BD9
:10940000730B4C155D056E057F0508F432CE81E0C7
:10941000868B61E0C3010E94A3402BCE90E080E0E8
:109420002ACE2F923F924F925F926F927F928F92AD
:109430009F92AF92BF92CF92DF92EF92FF920F93E3
:109440001F93CF93DF93CDB7DEB7C458D1090FB6C2
:10945000F894DEBF0FBECDBFFC01902FA2960FAFD8
:10946000A297A3961FAFA397A4962FAFA497A596F4
:109470003FAFA597A6964FAFA697A7965FAFA797C2
:10948000A8966FAFA897A9967FAFA99786EF800F90
:10949000823008F492C6EB96FFAEEEAEEB97AD9637
:1094A000FFAFEEAFAD97822F422E512C002309F46F
:1094B00092C64114510409F483C6EB96AEADBFAD1C
:1094C000EB97AB2B09F48EC6873051F5913109F437
:1094D00027C2923109F444C29031F9F46FEF70E081
:1094E000CE018F599F4F0E94C16B6A962FAF6A972A
:1094F0006B963FAF6B976C964FAF6C976D965FAF67
:109500006D976E966FAF6E976F967FAF6F97A096C1
:109510008FAFA097A1969FAFA19767E0462E512CE1
:10952000AD96AEADBFADAD971496ED91FC91309771
:1095300009F472C466807780CF57DF4F1982188292
:10954000C158D040E9961FAE1EAEE997E3961FAE14
:109550001EAEE397312C212CE7961FAE1EAEE79787
:109560006114710409F466C46CEA75E0C3010E94D9
:1095700091ACE1969FAF8EAFE19769E276E0C301CF
:109580000E9491ACAB969FAF8EAFAB976EE476E046
:10959000C3010E9491ACCD57DF4F99838883C35894
:1095A000D04060E375E0C3010E9491ACED969FAF9F
:1095B0008EAFED97E196EEADFFADE197309709F4F0
:1095C000C0C0AB962EAD3FADAB972115310509F468
:1095D000B8C080858F70823009F0B3C0D901189669
:1095E0008C918F70823009F0ACC02CE330E040E009
:1095F00050E060E675E0C3010E946D27C358DF4F5D
:10960000688379838A839B83CD57D040EB96EEADF8
:10961000FFADEB973097F1F1BF01D3018D919C9194
:109620000F947459892BB1F5B2E04B16510409F42B
:10963000A9C30CF09DC1F1E04F16510409F43AC2E0
:10964000CD57DF4FE881F981C358D040309711F1F1
:10965000912C812CB12CA12CD12CC12CA296EFAC39
:10966000A297A396FFACA397A4960FADA497A59637
:109670001FADA597A6962FADA697A7963FADA79726
:10968000A8964FADA897A9965FADA9976FEFCF01A8
:109690000E949D3DAB96EEADFFADAB978185928567
:1096A000A385B48582309105A105B10509F443C0B5
:1096B0008F3F9F4FAF4FBF4FF1F1E196EEADFFAD42
:1096C000E19781859285A385B485EF964EAD5FAD18
:1096D000EF97849F9001859F300D949F300D11244A
:1096E000E796EEADFFADE797E20FF31FE796FFAF0A
:1096F000EEAFE797CF57DF4FE881F981C158D040EF
:10970000AF01FF0F660B770B481759076A077B07F6
:1097100094F4CF57DF4F99838883C158D040E9969E
:109720003FAF2EAFE997EF962EAD3FADEF97E396A3
:109730003FAF2EAFE397EF964EAD5FADEF97240EA0
:10974000351ED30112966D907C900ACFA3968FADF3
:10975000A3978F70E1F481E090E0CC57DF4F0FB614
:10976000F894DEBF0FBECDBFDF91CF911F910F9157
:10977000FF90EF90DF90CF90BF90AF909F908F9031
:109780007F906F905F904F903F902F90089560E58D
:1097900071E188E39FE00F94422362E471E188E382
:1097A0009FE00F944223CE018F599F4F0E94146D6A
:1097B000AB01BC0188E39FE00E946DB188E39FE0AC
:1097C0000F944322AD96AEADBFADAD9712960D91FD
:1097D0001C914FEF5FEFBA0180E00E941928AB01A6
:1097E000BC01C8010E94D4E4CE018F599F4F0E9452
:1097F000146D6B017C016FE479E0AD96EEADFFADC9
:10980000AD97848195810E9491ACA701960164EB8C
:1098100075E00E94AF1C9FCF6CE371E188E39FE08D
:109820000F94422362E371E188E39FE00F944223A7
:10983000A2966FADA29788E39FE00E941BAD88E3DC
:109840009FE00F944322A2960FADA2976FE479E0B8
:10985000AD96AEADBFADAD9714968D919C910E9423
:1098600091AC60E476E00E94881C7C01009709F4CA
:1098700072CFFC018085982F9F70923039F0933021
:1098800081F0911168CF807F8260808710E030E0A6
:1098900020E0D70119960D931D932D933C931C97AF
:1098A0005ACF602F70E090E080E00F944353D701CF
:1098B00019966D937D938D939C931C974CCF6CE27E
:1098C00071E188E39FE00F9442236AE171E188E34C
:1098D0009FE00F944223CE018F599F4F0E94146D39
:1098E000AB01BC0188E39FE00E946DB188E39FE07B
:1098F0000F944322CE018F599F4F0E94146D6B012C
:109900007C016FE479E0AD96EEADFFADAD9784815B
:1099100095810E9491ACA701960165E476E079CF2C
:1099200060E870E0CE018F599F4F0E94C16B629634
:109930002FAF629763963FAF639764964FAF64977C
:1099400065965FAF659766966FAF669767967FAFD0
:10995000679768968FAF689769969FAF6997DDCDD7
:109960006AE070E0CE018F599F4F0E94C16CD5CD47
:1099700023E04216510409F429C237E0431651048A
:1099800009F05ECEA3968FADA3978F7009F48CC0BB
:10999000CE018F599F4F0E945A6DAB96AEADBFADB1
:1099A000AB9719960D911D912D913C911C97672BAA
:1099B000682B692B09F4A6C0023011052105310579
:1099C000B1F562E576E088E39FE00F94EB2288E34F
:1099D0009FE00F94432221E030E040E050E0AB965E
:1099E000AEADBFADAB9719962D933D934D935C9360
:1099F0001C9761E0CE018F599F4F0E94E76A2A961B
:109A00002FAF2A972B963FAF2B972C964FAF2C97C3
:109A10002D965FAF2D972E966FAF2E972F967FAF17
:109A20002F9760968FAF609761969FAF6197CE0139
:109A30008F599F4F0E945A6DE196EEADFFADE197B1
:109A400061877287838794878091FD109091FE10C3
:109A5000059751F1D301AD90BC9088248394C12C1B
:109A600050E3D52EE12CF12CA2960FADA297A39630
:109A70001FADA397A4962FADA497A5963FADA5972C
:109A8000A6964FADA697A7965FADA797A8966FAD80
:109A9000A897A9967FADA997AD96EEADFFADAD970E
:109AA000828193810E94DD7DA2968FADA29788234B
:109AB00009F4C6CDA2969FADA297992309F4C0CD13
:109AC000EFEFE90FE63108F059C1F0E08827E459DB
:109AD000F24B8F4F0D941355C64D604EBE4EBE4E89
:109AE000BE4EBE4EBE4EBE4EBE4E7E4E984EBE4E7C
:109AF000BE4EAC4EAC4EBE4EBE4EBE4EAC4EAC4E4E
:109B0000AC4EAC4E0130110521053105B1F563E6CF
:109B100076E088E39FE00F94EB2288E39FE00F94C8
:109B2000432222E030E040E050E0AB96AEADBFAD66
:109B3000AB9719962D933D934D935C931C9762E0E0
:109B4000CE018F599F4F0E94E76A22962FAF22972E
:109B500023963FAF239724964FAF249725965FAF68
:109B6000259726966FAF269727967FAF279728963B
:109B70008FAF289729969FAF2997E196EEADFFAD5D
:109B8000E19711861286138614865ECFE196AEADFC
:109B9000BFADE19719966D917C91CE018F599F4F82
:109BA0000E94C16B29AF3AAF4BAF5CAF6DAF7EAFD8
:109BB0008FAF21969FAF219767E0CE018F599F4FBE
:109BC0000E94C56A29AB3AAB4BAB5CAB6DAB7EABCD
:109BD0008FAB98AFA2968FADA29790E0B0E0A0E0D7
:109BE000AB96EEADFFADAB9781879287A387B48725
:109BF000C12C40E3D42EE12CF12C8091FD109091EA
:109C0000FE10059779F1AB96EEADFFADAB97818570
:109C10009285A385B4850197A105B10519F5E19653
:109C2000EEADFFADE19781859285A385B48544971C
:109C3000A105B105BCF42EE130E040E050E0218701
:109C40003287438754876EE170E0CE018F599F4F72
:109C50000E94C16B298F3A8F4B8F5C8F6D8F7E8FE7
:109C60008F8F98A38091FD109091FE10059709F4B5
:109C7000E7CCF301A080B18088248394A2960FAD35
:109C8000A297A3961FADA397A4962FADA497A596D0
:109C90003FADA597A6964FADA697A7965FADA797A0
:109CA000A8966FADA897A9967FADA997AD96AEADD2
:109CB000BFADAD9712968D919C910E94DD7DC0CC79
:109CC00070E060E0CE018F599F4F0E94C16B29A7C1
:109CD0003AA74BA75CA76DA77EA78FA798AB67E0B5
:109CE000CE018F599F4F0E94C56A29A33AA34BA367
:109CF0005CA36DA37EA38FA398A76CCFED962EAD2A
:109D00003FADED972115310569F0F9018185928507
:109D1000A385B4850097A105B10521F061E070E04D
:109D20000F944E26C12C20E4D22EE12CF12C65CFCD
:109D3000ED962EAD3FADED972115310599F3F90163
:109D400081859285A385B4850097A105B10551F35E
:109D5000DC01DA961C92E6CF892F90E0B0E0A0E01B
:109D6000AB96EEADFFADAB9781879287A387B487A3
:109D7000C12C30E1D32EE12CF12C3FCFC12CD12CC2
:109D800076013BCFA3968FADA3978F7009F458CC83
:109D9000CE018F599F4F0E94146D9B01AC0160EB67
:109DA00075E0C3010E94AF1C8091FD109091FE10E0
:109DB000059709F445CCF301A080B18088248394F1
:109DC000C12C90E2D92EE12CF12C58CFA3968FAD67
:109DD000A3978F7009F4BFCC6DE071E188E39FE039
:109DE0000F944223CE018F599F4F0E94146DAB01F7
:109DF000BC0188E39FE00E946DB188E39FE00F946F
:109E00004322CE018F599F4F0E94146D9B01AC01DC
:109E100064EB75E0C301FDCCE9961FAE1EAEE99779
:109E2000E3961FAE1EAEE397312C212CE7961FAEB2
:109E30001EAEE7972114310409F4BFC1E7968EAD39
:109E40009FADE797B1010F94FF543B016EEF70E1B6
:109E500088E39FE00F944223B10188E39FE00E94D2
:109E600022AD63EF70E188E39FE00F9442230FEF90
:109E700010E0E7968EAD9FADE797B8010F94FF54C1
:109E800088E39FE00E9422AD6CEE70E188E39FE0E2
:109E90000F944223B30188E39FE00E9422AD62EE5B
:109EA00070E188E39FE00F944223E9968EAD9FAD69
:109EB000E997B8010F94FF5488E39FE00E9422AD18
:109EC0006BED70E188E39FE00F944223E3966EAD63
:109ED0007FADE39788E39FE00E9422AD67ED70E1DC
:109EE00088E39FE00F94422388E39FE00F9443228E
:109EF00019821A821B821C821D821E821F82188672
:109F00008A81807F8A83B301CE0101960E94C16B52
:109F100029873A874B875C876D877E878F87988BE9
:109F200067E0CE0109960E94C56A79018A011B018A
:109F30002C01298BFA8A4B8B1C8B6D8B3E8A8F8B65
:109F4000588E6FE479E0AD96EEADFFADAD978481AC
:109F500095810E9491AC912C812CB12CA12CD12CFB
:109F6000C12C9101A2016FEF0E949D3D672809F469
:109F7000F2CBAD96AEADBFADAD971496ED91FC9121
:109F8000309709F4E8CB66807780E3962EAD3FAD3D
:109F9000E397032E000C440B550BE5962CAF3DAF19
:109FA0004EAF5FAFE597E9968EAD9FADE997092E6D
:109FB000000CAA0BBB0BAF968CAF9DAFAEAFBFAF83
:109FC000AF976114710409F4C6CB2CE330E040E094
:109FD00050E060E675E0C3010E946D276B016DE9FA
:109FE00075E0C3010E9491ACAB969FAF8EAFAB976B
:109FF0006CEA75E0C3010E9491AC8C0169E276E0E5
:10A00000C3010E9491ACAB96AEADBFADAB971097BC
:10A0100009F4CBC00115110509F4C7C0009709F474
:10A02000C4C018962C912F70223009F0BEC0F801E0
:10A0300020852F70223009F0B8C0DC0118962C91D1
:10A0400018972F70223009F0B0C0C114D10409F460
:10A05000ACC019968D919D910D90BC91A02D823030
:10A060009105A105B10509F4A4C08F3F9F4FAF4FE3
:10A07000BF4F09F49EC0E9962EAD3FADE997232B63
:10A0800009F497C0D80119968D919C918C9D8001FF
:10A090008D9D100D9C9D100D11242FEF30E0D801E7
:10A0A0000F942A559601DD0C440B550B0F94AA54BE
:10A0B000E5966CAD7DAD8EAD9FADE5970F94785470
:10A0C000AF962CAD3DAD4EAD5FADAF970F94AA549A
:10A0D00019012A0160ED70E188E39FE00F944223AB
:10A0E000F3016081718188E39FE00F94EB226AECB9
:10A0F00070E188E39FE00F944223C8016FEF70E0A6
:10A100000F94FF5488E39FE00E9422AD64EC70E15D
:10A1100088E39FE00F9442232AE030E0B201A101DE
:10A1200088E39FE00F94652288E39FE00F94432229
:10A13000AB96EEADFFADAB9781859285A385B485D7
:10A1400082159305A405B50581F119861A861B862B
:10A150001C861D861E861F86188A8A85807F8A87B0
:10A16000B101CE0109960E94C16B29833A834B83CA
:10A170005C836D837E838F839887912C812CB12C97
:10A18000A12CD12CC12C79018A019B01AC016FEF6C
:10A19000C3010E949D3DAB96AEADBFADAB97199686
:10A1A0002D923D924D925C921C97F30162807380D8
:10A1B00008CF212C312C2101BBCF90E080E0CDCA0B
:10A1C000EB962EAD3FADEB9744244394512C232BBB
:10A1D00009F0A6C9C0CAEB964EAD5FADEB97452B13
:10A1E00009F09EC9833009F4B1CA20F4813008F423
:10A1F00097C9B1CA883009F40FCB8C3009F45FCB12
:10A20000873009F08DC9A7CA4F925F926F927F92F3
:10A210008F929F92AF92BF92CF92DF92EF92FF9276
:10A220000F931F93CF93DF93CDB7DEB768970FB629
:10A23000F894DEBF0FBECDBF3B016FE479E0FC01B7
:10A24000848195810E9491AC2C01009709F47BC018
:10A2500020E030E0A90165E776E00E946D278B01E0
:10A2600020E030E0A90160E476E0C2010E946D27A1
:10A270000115110541F00617170709F064C006150E
:10A28000170509F460C019861A861B861C861D8670
:10A290001E861F86188A8A85807F8A87662DCE0152
:10A2A00009960E94E76A298B3A8B4B8B5C8B6D8BEE
:10A2B0007E8B8F8B988F61E0CE0141960E94C56A9C
:10A2C00029833A834B835C836D837E838F83988756
:10A2D000912C812CB12CA12CD12CC12C79018A017B
:10A2E0009B01AC016FEFC2010E949D3D65E776E0E6
:10A2F000C2010E94881C8C01009711F1FC0180852D
:10A30000982F9F70923039F0933079F0911118C0E6
:10A31000807F82608087C301770CAA0BBB0BF8019A
:10A3200081879287A387B4870BC0B301770C880B12
:10A33000990B0F944553F80161877287838794873F
:10A3400081E090E002C090E080E068960FB6F8945B
:10A35000DEBF0FBECDBFDF91CF911F910F91FF9058
:10A36000EF90DF90CF90BF90AF909F908F907F90B5
:10A370006F905F904F9008952F923F924F925F920F
:10A380006F927F928F929F92AF92BF92CF92DF9205
:10A39000EF92FF920F931F93CF93DF93CDB7DEB76A
:10A3A000E6970FB6F894DEBF0FBECDBF4C0161300B
:10A3B0007105D9F5DC0112968D919C910E9415E5ED
:10A3C000672B682B692B89F14FEF5FEFBA0180E0B3
:10A3D0000E9419286B017C01F40102811381C801DC
:10A3E0000E9415E5C61AD70AE80AF90AF0E6CF1660
:10A3F000FAEEDF06E104F104C0F040E050E0BA01FB
:10A40000C8010E94D4E46FE479E0D40114968D91E0
:10A410009C910E9491AC64EB75E00E9491AC009716
:10A4200021F0FC012085207F2087D40114960D9116
:10A430001C910115110509F4BEC36FE479E0C80150
:10A440000E9491AC3C01009709F4D8C3FC018085BF
:10A450008F70863009F0D2C364EB75E0C3010E94AF
:10A4600091ACFC01892B09F4C9C390859F7093308E
:10A4700009F0C1C3C184D284E384F48420E030E0D5
:10A48000A90160E476E0C3010E946D277EAB6DAB4D
:10A4900020E030E040EF51E4C701B6010F9446568A
:10A4A00018160CF43FC120E030E040E751E4C7014A
:10A4B000B6010F943E5387FF3AC125E130E03CAB33
:10A4C0002BABF80166807780B12C1AAA19AA611407
:10A4D000710409F450C3D301ED91FC91309709F454
:10A4E00014C18081882309F410C120E030E0A90163
:10A4F00069E276E0C3010E946D278B0120E030E025
:10A50000A90160EB75E0C3010E946D271B012C01BE
:10A5100020E030E0A90164EB75E0C3010E946D27E3
:10A520006B017C010F30110509F434C10CF004C13A
:10A530000230110521F00E30110509F005C160E36C
:10A5400075E0C3010E9491AC6C01009709F4DDC075
:10A55000FC0181859285A385B4850097A105B1058D
:10A5600009F4D3C07C01FC0122AD222309F4CDC043
:10A570000F94B024882309F4C8C068EB75E0C301C8
:10A580000E9491AC2C01009709F4BFC0DC01189621
:10A590008C918F70833009F0B8C06DEB70E188E367
:10A5A0009FE00F944223D4011296ED91FC9102801A
:10A5B000F381E02D6081718188E39FE00F94EB22AD
:10A5C00066EA75E088E39FE00F94EB22F301608177
:10A5D000718188E39FE00F94EB2268EB70E188E3E0
:10A5E0009FE00F944223D7015C96ED91FC9140814E
:10A5F00051816281738188E39FE00E946DB162EBBB
:10A6000070E188E39FE00F944223D7019096ED918B
:10A61000FC91408151816281738188E39FE00E94B7
:10A620006DB16CEA70E188E39FE00F944223D7019B
:10A630005E96ED91FC91408151816281738188E346
:10A640009FE00E946DB16CE876E088E39FE00F9494
:10A65000EB22F701408151816281738188E39FE0A1
:10A660000E946DB160E976E088E39FE00F94EB22F1
:10A67000D70114964D915D916D917C91179788E368
:10A680009FE00E946DB164E976E088E39FE00F945B
:10A69000EB22F701408551856285738588E39FE051
:10A6A0000E946DB1D70158968D919C9164E876E037
:10A6B000892B11F06EE776E088E39FE00F94EB22A0
:10A6C000F70182AD6AE876E0811102C067EB78E0BD
:10A6D00088E39FE00F94EB2288E39FE00F944322EE
:10A6E0000431110509F443C10531110509F4CEC146
:10A6F0000E30110551F42BA93CA92431310509F480
:10A700004CC02531310509F4C2C0F3016280738069
:10A71000DECE61857285838594850F9445536B01E8
:10A720007C01ACCE84E190E09CAB8BABCACEAFE0B9
:10A73000B0E0BCABABABC5CE0331110541F024F0AA
:10A74000063111050CF4FBCE10E000E0F8CEC2019A
:10A75000B1010F9445531B012C01C701B6010F94A1
:10A7600045536B017C01AC019B01C201B1010F9407
:10A77000465604E110E0181614F010E000E0A701BE
:10A780009601C201B1010F943E5387FFD8CE05E177
:10A7900010E0D5CEBB24B394D2CE70E060E0D601F9
:10A7A00019968D919C910F9412266BE970E188E3C4
:10A7B0009FE00F944223D4011296ED91FC91028008
:10A7C000F381E02D6081718188E39FE00F94EB229B
:10A7D00066EA75E088E39FE00F94EB22F301608165
:10A7E000718188E39FE00F94EB226AE870E188E3CF
:10A7F0009FE00F94422388E39FE00F9443222DA90A
:10A800003EA92230310509F480CFD401ED91FC91AD
:10A8100020883188F301E080F18019821A821B823E
:10A820001C821D821E821F8218868A81807F8A83F5
:10A83000D20119966D917D918D919C911C970F94E9
:10A840001056CE0101960E94C16B29873A874B872B
:10A850005C876D877E878F87988B67E0CE0109962E
:10A860000E94C56A022F242F09A73AA74BA75CA70D
:10A870006DA77EA78FA798ABA12CCC24C394132FD0
:10A88000352FAB01BC01C401F10119953ECF61E048
:10A8900070E0D60119968D919C910F94122669E76C
:10A8A00070E188E39FE00F944223D4011296ED916A
:10A8B000FC910280F381E02D6081718188E39FE04B
:10A8C0000F94EB2266EA75E088E39FE00F94EB2299
:10A8D000F3016081718188E39FE00F94EB2267E6CA
:10A8E00070E188E39FE00F94422388E39FE00F9498
:10A8F00043222DA93EA92230310509F406CFD40107
:10A90000ED91FC9120883188F301E080F18019827B
:10A910001A821B821C821D821E821F8218868A81D7
:10A92000807F8A83D20119966D917D918D919C9142
:10A930001C970F941056CE0101960E94C16B298777
:10A940003A874B875C876D877E878F87988B67E018
:10A95000CE0109960E94C56A022F242F09A33AA3AB
:10A960004BA35CA36DA37EA38FA398A785CF70E0B4
:10A9700060E0D60119968D919C910F9412266BE59B
:10A9800070E188E39FE00F944223D4011296ED9189
:10A99000FC910280F381E02D6081718188E39FE06A
:10A9A0000F94EB2266EA75E088E39FE00F94EB22B8
:10A9B000F3016081718188E39FE00F94EB226AE4E8
:10A9C00070E188E39FE00F94422388E39FE00F94B7
:10A9D00043222DA93EA92431310509F041C0D401FB
:10A9E000ED91FC9120883188F301E080F18019829B
:10A9F0001A821B821C821D821E821F8218868A81F7
:10AA0000807F8A83D20119966D917D918D919C9161
:10AA10001C970F941056CE0101960E94C16B298796
:10AA20003A874B875C876D877E878F87988B67E037
:10AA3000CE0109960E94C56A022F242F098F3A8FF2
:10AA40004B8F5C8F6D8F7E8F8F8F98A3A12CCC2422
:10AA5000C394132F352FAB01BC01C401F10119952B
:10AA600029A93AA9B901330F880B990B0F944553C3
:10AA7000D20119962D913D914D915C911C970F94A7
:10AA800032550F9410567AAB69AB3FCE61E070E05F
:10AA9000F601818592850F9412266EE370E188E3BA
:10AAA0009FE00F944223D4011296ED91FC91028015
:10AAB000F381E02D6081718188E39FE00F94EB22A8
:10AAC00066EA75E088E39FE00F94EB22F301608172
:10AAD000718188E39FE00F94EB226CE270E188E3E0
:10AAE0009FE00F94422388E39FE00F9443222DA917
:10AAF0003EA92531310569F519821A821B821C8213
:10AB00001D821E821F8218868A81807F8A83D201DD
:10AB100019966D917D918D919C911C970F94105673
:10AB2000CE0101960E94C16B29873A874B875C87CB
:10AB30006D877E878F87988B67E0CE0109960E948C
:10AB4000C56A298B3A8B4B8B5C8B6D8B7E8B8F8B85
:10AB5000988FE9A9FAA9BF01FF0F880B990B0F94F1
:10AB60004553D20119962D913D914D915C911C97C1
:10AB70000F94315586CF29A93AA9232BB9F168E161
:10AB800070E188E39FE00F94422369A97AA988E3E2
:10AB90009FE00E9422AD88E39FE00F94432289A9A1
:10ABA0009AA964E170E01816190614F065E170E0E6
:10ABB000C4010E94045181E090E0E6960FB6F8943B
:10ABC000DEBF0FBECDBFDF91CF911F910F91FF90E0
:10ABD000EF90DF90CF90BF90AF909F908F907F903D
:10ABE0006F905F904F903F902F900895BB2019F386
:10ABF0006FE070E0DDCF923009F48BCDC12CD12C09
:10AC000080ECE82E8FE7F82E39CC2F923F924F92AE
:10AC10005F926F927F928F929F92AF92BF92CF92EC
:10AC2000DF92EF92FF920F931F93CF93DF93CDB7F5
:10AC3000DEB7CF58D1090FB6F894DEBF0FBECDBF37
:10AC40003C011A01CD57DF4F2883C358D040C45769
:10AC5000DF4F19830883CC58D040C257DF4FF982A9
:10AC6000E882CE58D040C957DF4FC882C758D0407D
:10AC7000CB57DF4FB982A882C558D040DC0114966B
:10AC8000ED91FC910288F389E02D86809780AB28B6
:10AC900049F4FE01EE57FF4FCB57DF4FF983E883AE
:10ACA000C558D04081E0CB57DF4FA881B981C55846
:10ACB000D0408C936B01F12CE12C8114910409F4A8
:10ACC000F0C5CD57DF4FB881C358D040B13009F43B
:10ACD00088C008F47FC0B23041F0B33009F477C0C7
:10ACE000D40112968D909C90E8CF6BE076E0C40181
:10ACF0000E9491AC11E0009799F3FC018185928547
:10AD0000A385B4858C159D05AE05BF0549F761E3A4
:10AD100075E0C4010E9491ACC857DF4F99838883C6
:10AD2000C858D040D3011296ED91FC9162E0848125
:10AD300095810E9409ADC657DF4F99838883CA5811
:10AD4000D040822D0E9433B87C01CF57DF4F18824C
:10AD5000C158D04019AA1AAA1BAA1CAA1DAA1EAA29
:10AD60001FAA18AE8AA9807F8AAB66E575E0C40188
:10AD70000E9491AC6C016BE575E0C4010E9491AC3E
:10AD80005C01C114D10451F0F60180858F708430CC
:10AD900029F4818592850E94751E182FEFEFE10F2F
:10ADA000EB3008F09BC10E2E000CFF0B8827E452FD
:10ADB000F94A8F4F0D941355F45680575E57A55797
:10ADC0006E586E58ED57CA57115822583A5868E9CC
:10ADD00076E08DCF6BE976E0C4010E9491AC1BE078
:10ADE0008ACF60EA76E0F8CF1701512C412CA701F9
:10ADF000FF0C660B770BCE01C1960E94096BEA9699
:10AE00002FAFEA97EB963FAFEB97EC964FAFEC97EF
:10AE1000ED965FAFED97EE966FAFEE97EF967FAF43
:10AE2000EF97C158DF4F8883CF57D040C058DF4FCE
:10AE30009883C058D04080911E02893020F48091C0
:10AE40001D028930A8F16FEE7DE088E39FE00F944A
:10AE5000422300E020E030E340E150E0BE016F5FBC
:10AE60007F4FCE01C1960E940A6EBC0188E39FE02D
:10AE70000F94EB2263EE7DE088E39FE00F94422382
:10AE8000612F110F770B88E39FE00E9422AD61EEE6
:10AE90007DE088E39FE00F944223D4016D917C9183
:10AEA00088E39FE00F94EB2288E39FE00F94432216
:10AEB000A114B10409F016C1D12C6FC31701512C94
:10AEC000412CB201A701CE01C1960E94096BE29606
:10AED0002FAFE297E3963FAFE397E4964FAFE49747
:10AEE000E5965FAFE597E6966FAFE697E7967FAF9B
:10AEF000E797E8968FAFE897E9969FAFE9979BCFE2
:10AF0000FE24EF24FE241701512C412CB201A10193
:10AF1000CE01C1960E94096BAA962FAFAA97AB9655
:10AF20003FAFAB97AC964FAFAC97AD965FAFAD97D9
:10AF3000AE966FAFAE97AF967FAFAF97E0968FAFFD
:10AF4000E097E1969FAFE19776CFFE24EF24FE24B1
:10AF50001701512C412CB201A101CE01C1960E94D2
:10AF6000096BA2962FAFA297A3963FAFA397A49683
:10AF70004FAFA497A5965FAFA597A6966FAFA6977C
:10AF8000A7967FAFA797A8968FAFA897A9969FAFD0
:10AF9000A99751CFFF241701512C412CB201A701D1
:10AFA000CE01C1960E94096B6A962FAF6A976B9685
:10AFB0003FAF6B976C964FAF6C976D965FAF6D9789
:10AFC0006E966FAF6E976F967FAF6F97A0968FAFAD
:10AFD000A097A1969FAFA1972ECFEF2CFF2417012A
:10AFE000512C412CB201A701CE01C1960E94096BE0
:10AFF00062962FAF629763963FAF639764964FAFA9
:10B00000649765965FAF659766966FAF669767962C
:10B010007FAF679768968FAF689769969FAF69977C
:10B020000ACF1701512C412C8AA9807F86608AABF8
:10B030002AE030E0D7010F942A556DAB7EAB8FAB81
:10B0400098AFF9CE1701512C412C8AA9807F8760D7
:10B050008AABB701FF0C880B990B0F94455320E086
:10B0600030E048EC52E40F949E556DAB7EAB8FAB55
:10B0700098AFE1CEC10124E0969587952A95E1F736
:10B080000E9433B8FFE02F22332402C096958795A3
:10B090002A94E2F7817099271C01512C412CB201AE
:10B0A000AC01CE01C1960E94096B2A962FAF2A9758
:10B0B0002B963FAF2B972C964FAF2C972D965FAFCB
:10B0C0002D972E966FAF2E972F967FAF2F97609666
:10B0D0008FAF609761969FAF6197ADCE212C312CD9
:10B0E0002101A9CEF50180858F708550823008F04E
:10B0F000E3CEB501CE01C1960E94587629A33AA3AA
:10B100004BA35CA36DA37EA38FA398A788E0FE0149
:10B11000B196DE01999601900D928A95E1F788E04B
:10B12000FE01B996DE01D19601900D928A95E1F764
:10B1300089A9811103C08AA98F7009F180911E022B
:10B14000893008F4B7C26CE57DE088E39FE00F9496
:10B15000422300E020E030E340E150E0BE016F5FB9
:10B160007F4FCE01C1960E940A6EBC0188E39FE02A
:10B170000F94EB2288E39FE00F9443229DCE67E07B
:10B1800076E0C5010E9491AC7C01009709F494CE51
:10B19000DC0118968C918F70823009F41DC18430C7
:10B1A00009F08ACE80911E02893020F480911D0220
:10B1B000893090F062E97DE088E39FE00F944223BC
:10B1C000D70119966D917C9188E39FE00F94EB2253
:10B1D00088E39FE00F944322C657DF4FE881F9814F
:10B1E000CA58D040309709F46DC380858F7086307F
:10B1F00009F066C3D7011996CD90DC90C114D10433
:10B2000009F45EC3D3011296ED91FC9162E0848152
:10B2100095810E9409ADB6010E9491AC0E9447BB86
:10B220006C01892B09F44CC380911E02893020F4F3
:10B2300080911D028930A8F060E87DE088E39FE0FE
:10B240000F944223F60141855285638574852AE077
:10B2500030E088E39FE00F94652288E39FE00F943D
:10B260004322D70119966D917C91D3011496ED91EB
:10B27000FC91828993890E9491AC7C01009709F42A
:10B280001FC366E575E00E9491AC009749F0FC0190
:10B2900020852F70243021F4818592850E94751EAF
:10B2A000D60119964D915D916D917C911C97CE01BF
:10B2B000C1960E94096B22962FAF229723963FAF2B
:10B2C000239724964FAF249725965FAF2597269610
:10B2D0006FAF269727967FAF279728968FAF28972F
:10B2E00029969FAF29976BE575E0C7010E9491AC45
:10B2F000BC01009721F1FC0190859F709550923020
:10B30000F0F4CE01C1960E945876298B3A8B4B8B74
:10B310005C8B6D8B7E8B8F8B988F88E0FE01719696
:10B32000DE01599601900D928A95E1F788E0FE01C1
:10B330007996DE01D19601900D928A95E1F7809180
:10B340001E02893020F480911D028930D8F06BE60E
:10B350007DE088E39FE00F94422300E020E030E3AB
:10B3600040E150E0BE016F5F7F4FCE01C1960E9469
:10B370000A6EBC0188E39FE00F94EB2288E39FE014
:10B380000F944322D60118968C911897982F929576
:10B390009F7090FD95C221E0CF57DF4F2883C158A1
:10B3A000D04091609295907F8F70892B18968C93E6
:10B3B000DD24D394C957DF4FB881C758D040BB2391
:10B3C00009F404C1C857DF4F48815981C858D0409B
:10B3D000452B09F4FBC088C280911E02893020F4FD
:10B3E00080911D028930A8F06BEC7DE088E39FE03E
:10B3F0000F944223F70141855285638574852AE0C5
:10B4000030E088E39FE00F94652288E39FE00F948B
:10B410004322D70119966D917D918D919C911C9736
:10B42000C457DF4FE881F981CC58D0408F0130E01C
:10B4300020E060177107820793070CF453C0C257CE
:10B44000DF4F48815981CE58D0408A0130E020E05A
:10B4500006171707280739070CF444C0AB014E1B29
:10B460005F0BDE01AF57BF4F5D01C12CC257DF4FED
:10B47000E880F980CE58D0408F01CD57DF4F28812A
:10B48000C358D040C3010E94055629AB3AAB4BAB21
:10B490005CAB6DAB7EAB8FAB98AF80911E028930F9
:10B4A00020F480911D028930D0F064EA76E088E3D0
:10B4B0009FE00F94EB2261EC76E088E39FE00F942D
:10B4C000EB22CF57DF4F6881C158D04070E088E34E
:10B4D0009FE00E9422AD88E39FE00F944322DD2489
:10B4E000D3945BC061EC7DE088E39FE00F9442233E
:10B4F000F70141855285638574852AE030E088E351
:10B500009FE00F94652262EA7DE088E39FE00F945C
:10B51000422388E39FE00F94432281E08093B60C9E
:10B52000CE01419690933C0D80933B0DCD57DF4F5C
:10B53000F881C358D0406F2F70E041E050E0D70150
:10B5400019968D919C910E947B2DD82E8823E1F035
:10B55000F701618572859E012F573F4F5901C12C1C
:10B560007B018B01CD57DF4F2881C358D04050E07D
:10B5700040E0C3010E94055629AB3AAB4BAB5CAB34
:10B580006DAB7EAB8FAB98AF80E48093B60C8BEB4A
:10B590009CE090933C0D80933B0DC957DF4FB881E1
:10B5A000C758D040BB2349F0C857DF4FE881F98125
:10B5B000C858D040EF2B09F097C1C657DF4FE8813C
:10B5C000F981CA58D040EF2B09F447C0C657DF4F66
:10B5D000A881B981CA58D04018968C9118978F705D
:10B5E0008630D9F5F40160817181CD010E9491AC62
:10B5F0003C01009791F10E9447BB7C01009709F440
:10B60000D4C0FC0181859285A385B48582159305FC
:10B61000A405B50509F09CC0C957DF4FF881C7588C
:10B62000D040F11157C0D70118968C911897829588
:10B630008F7080FD4FC091E0CB57DF4FE881F981DB
:10B64000C558D040908381608295807F18969C91E8
:10B6500018979F70892B18968C9388E0FE01F196BD
:10B66000DE01D99601900D928A95E1F729AD3AADA8
:10B670004BAD5CAD6DAD7EAD8FAD21969FAD21978D
:10B68000C157DF4F0FB6F894DEBF0FBECDBFDF91BD
:10B69000CF911F910F91FF90EF90DF90CF90BF90CF
:10B6A000AF909F908F907F906F905F904F903F9062
:10B6B0002F90089580911D02893008F4FDCB43CD71
:10B6C000F3016281738140E050E1CE01C1960E9496
:10B6D0001F6A73CFCB57DF4FA881B981C558D040BF
:10B6E0001C92DD2009F4B9CFC957DF4FB881C75884
:10B6F000D040BB2309F4B1CFCF57DF4F8881C15869
:10B70000D04081110AC0CB57DF4FA881B981C558FD
:10B71000D0408C91882309F4A0CF912C812CB12C9E
:10B72000A12CD12CC12CE9A8FAA80BA91CA92DA9E0
:10B730003EA94FA958AD6FEFC3010E949D3D81E026
:10B74000CB57DF4FE881F981C558D040808385CF42
:10B75000218632864386548680911E02893020F4E9
:10B7600080911D028930E8F066EC76E088E39FE086
:10B770000F94EB22B201A10188E39FE00E9418AD73
:10B7800064ED76E088E39FE00F94EB22D4016D91A5
:10B790007C9188E39FE00F94EB2288E39FE00F9475
:10B7A0004322F70180858F7E8087D1109DCFCB57B4
:10B7B000DF4FA881B981C558D0408C91882309F406
:10B7C0004CCFC957DF4FB881C758D040BB2309F4CD
:10B7D00044CFF30180858F708530D1F586819781C4
:10B7E0006FE575E00E9491ACCD57DF4F9983888358
:10B7F000C358D040009771F1DC0118968C911897CE
:10B800008F70823039F519968D919D910D90BC9174
:10B81000A02D82159305A405B505E1F480911E02C3
:10B82000893020F480911D02893050F065E37DE07D
:10B8300088E39FE00F94422388E39FE00F94432224
:10B84000CB57DF4FE881F981C558D040108205CF32
:10B85000C301C6CF912C812CB12CA12CD12CC12C91
:10B86000E9A8FAA80BA91CA92DA93EA94FA958AD72
:10B870006FEFC3010E949D3DCD57DF4F2881398175
:10B88000C358D0402115310509F4E7CED3011896ED
:10B890008C9187FDE2CEF90121863286438654865B
:10B8A000DCCE19821A821B821C828A81807F8A8365
:10B8B0001D821E821F82188688E0FE013196D0CE3E
:10B8C000D12C78CDC957DF4FE881C758D040EE233F
:10B8D00009F4C3CEC857DF4F28813981C858D040FA
:10B8E000D12C232B09F4B9CEC857DF4FA881B981D9
:10B8F000C858D04018968C9118978F70823009F0F4
:10B900005CCE19968D919D910D90BC91A02D8130AA
:10B910009105A105B10509F4D3CE0297A105B105A2
:10B9200009F04BCED30112966D917C9140E050E22C
:10B93000CCCE2F923F924F925F926F927F928F92D6
:10B940009F92AF92BF92CF92DF92EF92FF920F93AE
:10B950001F93CF93DF93CDB7DEB768970FB6F894F8
:10B96000DEBF0FBECDBF6115710509F491C05E8BBE
:10B97000498B9D8B8C8BFB01868097808114910471
:10B9800009F486C0F40180858F70823031F08530F3
:10B9900031F1F40182809380F1CF6184728441E0BF
:10B9A00050E069897E89C3010E947B2D882389F339
:10B9B000B12CA12CCC24C39473018301298950E0BC
:10B9C00040E0B3018C899D890E94055629873A87FA
:10B9D0004B875C876D877E878F87988BDACFC40112
:10B9E0000E94ACAD8230A9F660E0C4010E9409ADAE
:10B9F000FC01C184D284E384F48461E0C4010E9428
:10BA000009ADFC012184328443845484388E2F8A0A
:10BA1000DB8ACA8AA1014C195D094F5F5F4F6989B2
:10BA20007E89C6010E947B2D882309F4B2CF8091C4
:10BA30001E02893020F480911D02893020F088E3B5
:10BA40009FE00F944322712C612C6A897B89660DDB
:10BA5000771D8F89988D861797070CF49ACFB12C94
:10BA6000A12CCC24C39471010A891B892989A301C3
:10BA70008C899D890E94055629833A834B835C8378
:10BA80006D837E838F8398879FEF691A790ADDCF54
:10BA900068960FB6F894DEBF0FBECDBFDF91CF9191
:10BAA0001F910F91FF90EF90DF90CF90BF90AF90DC
:10BAB0009F908F907F906F905F904F903F902F90CE
:10BAC00008952F923F924F925F926F927F928F9242
:10BAD0009F92AF92BF92CF92DF92EF92FF920F931D
:10BAE0001F93CF93DF9300D01F921F92CDB7DEB785
:10BAF00061307105D1F490E080E00F900F900F90CD
:10BB00000F900F90DF91CF911F910F91FF90EF90C9
:10BB1000DF90CF90BF90AF909F908F907F906F906D
:10BB20005F904F903F902F9008952091AD093091F4
:10BB3000AE09232B01F78C01DC01ED91FC9102840D
:10BB4000F385E02D19950297B1F68091BC0990918B
:10BB5000BD09A091BE09B091BF09892B8A2B8B2BFF
:10BB600079F4D8011296ED91FC9162E0848195817F
:10BB70000E9409AD9C838B83892BB1F4B12C01C445
:10BB80000E9454BFC090BC09D090BD09E090BE098E
:10BB9000F090BF096C197D098E099F09683C7105F9
:10BBA00081059105F0F6A7CFEB81FC8180858F7030
:10BBB000863021F7C680D7801D82B12CC114D104F4
:10BBC00009F4DBC3D60118968C91982F9F702BEF48
:10BBD000290F223008F0D1C3BD81B111CEC3282F67
:10BBE00022952F7087FF70C522FD6EC5953009F034
:10BBF000A7C0F601868197816FE575E00E9491AC40
:10BC00001C01892B09F460C581E090E09093AE0996
:10BC10008093AD09B11003C0C8010E940123D10176
:10BC200019964D905C906FED76E088E39FE00F945D
:10BC3000EB22D8011296ED91FC910280F381E02D68
:10BC40006081718188E39FE00F94EB2266EA75E0E2
:10BC500088E39FE00F94EB22F6016081718188E315
:10BC60009FE00F94EB2261E278E088E39FE00F947D
:10BC7000EB22D10119964D915D916D917C911C97AC
:10BC80002AE030E088E39FE00F94652288E39FE09C
:10BC90000F944322F60180809180D8011496ED9193
:10BCA000FC9164ED7EE0309759F0B401828993896C
:10BCB0000E9491AC7C01009709F044C061EB7EE0EA
:10BCC00081E99EE00F94422381E99EE00F94432294
:10BCD000EE24EA94FE2C4201550CAA08BB08D101BF
:10BCE00019964D905D906D907C901C9784149504EE
:10BCF000A604B70409F49DC48091BC099091BD09C4
:10BD0000A091BE09B091BF09892B8A2B8B2B09F416
:10BD100086CF0E9454BF2091BC093091BD0940914B
:10BD2000BE095091BF09621B730B840B950B683CD5
:10BD300071058105910508F072CF0E94CD36D6CFEE
:10BD4000C6015ACF6BE076E00E9491AC3C01892B92
:10BD500079F46BE976E0C7010E9491AC3C016EE892
:10BD60007EE0892B69F0F10180858F70806B808780
:10BD7000D30118968C918F70823079F068E77EE05D
:10BD800081E99EE00F94422381E99EE00F944322D3
:10BD9000EEEFEE2EFF24FA949ECF6EEF75E0C70112
:10BDA0000E9491AC7C01009709F43CC1FC018085A4
:10BDB0008F70813009F05BC18185882309F457C1F8
:10BDC000D10118968C91807FF12CE12C803B19F0E9
:10BDD00072E0E72EF12C6DE67EE088E39FE00F94A1
:10BDE0004223B40188E39FE00F94EB226AE67EE0F1
:10BDF00088E39FE00F944223F301418552856385D8
:10BE000074852AE030E088E39FE00F9465226BEEB2
:10BE100076E088E39FE00F94EB22B70188E39FE090
:10BE20000E9422AD61E875E088E39FE00F94EB2269
:10BE3000F1E0F093B60C81E090E08C0F9D1F9093A1
:10BE40003C0D80933B0D41E050E0B701D3011996C2
:10BE50008D919C910E947B2DF82E4FEF5FEFBA01E0
:10BE600080E00E9419286093BC097093BD098093FB
:10BE7000BE099093BF09FF2009F4F6C0D8011296BD
:10BE8000ED91FC9162E0848195810E9409AD7C0175
:10BE9000009709F4BEC0FC0180858F70863009F0E0
:10BEA000E3C0B401C7010E9491AC7C01009709F482
:10BEB000B0C00E9447BB7C01892B09F4AAC08091C5
:10BEC0001E02893020F480911D02893018F163E64A
:10BED0007EE088E39FE00F944223D70119964D91AD
:10BEE0005D916D917C911C972AE030E088E39FE0A2
:10BEF0000F9465226DE57EE088E39FE00F94422376
:10BF000069817A8188E39FE00E9467B188E39FE0BE
:10BF10000F944322F7014185528563857485898199
:10BF20009A81B0E0A0E0481759076A077B0719F12A
:10BF300067E57EE088E39FE00F944223B40188E345
:10BF40009FE00F94EB2269E47EE088E39FE00F948A
:10BF5000422388E39FE00F944322F0E4F093B60C71
:10BF60008BEB9CE090933C0D80933B0D6DEFE62EA8
:10BF7000FF24FA94B0CEF10181859285A385B48522
:10BF8000481759076A077B0779F563E47EE088E381
:10BF90009FE00F944223B40188E39FE00F94EB22CB
:10BFA00061E47EE088E39FE00F94422369817A8117
:10BFB00088E39FE00E9467B160E37EE088E39FE052
:10BFC0000F94422388E39FE00F944322F0E4F09320
:10BFD000B60C8BEB9CE090933C0D80933B0D5CEF9B
:10BFE000E52EFF24FA9477CE6AE27EE088E39FE0B4
:10BFF0000F944223B40188E39FE00F94EB226FE09B
:10C000007EE088E39FE00F94422388E39FE00F9453
:10C01000432290E49093B60CABEBBCE0B0933C0DA4
:10C02000A0933B0DD1011896EC91E295EF70E15091
:10C03000AA24AA94BA2CEB3008F066C0F0E0D30131
:10C0400019962D913C918827E75DFF498F4F0D94FC
:10C0500013553A604F603A604F60F760F260F760E6
:10C06000F2603A603A600361F12CE12CD2CFF12CFE
:10C07000E12CD8CFF1018185928530933E0D20933C
:10C080003D0D1092400D10923F0D9093420D809304
:10C09000410D86E00E94AEC0A82EB12C35C0D10162
:10C0A00019968D919C9198278927982730933E0D5A
:10C0B00020933D0D1092400D10923F0D9093420D34
:10C0C0008093410D86E00E94AEC0A82EB12CF101F4
:10C0D00081859285A385B4853A2F2B2FD30119969C
:10C0E0008D919C91019690933E0D80933D0D109201
:10C0F000400D10923F0D3093420D2093410D86E08C
:10C100000E94AEC0A80EB11C4FEF5FEFBA0180E0F5
:10C110000E9419286093BC097093BD098093BE09E1
:10C120009093BF0964E07EE088E39FE00F94422390
:10C13000B50188E39FE00E9422AD62E07EE088E3E3
:10C140009FE00F944223B40188E39FE00F94EB2219
:10C1500062EF76E088E39FE00F94EB22F3014185E4
:10C160005285638574852AE030E088E39FE00F9470
:10C1700065226CEF7DE088E39FE00F944223D101BC
:10C1800019964D915D916D917C911C972AE030E05C
:10C1900088E39FE00F94652288E39FE00F94432299
:10C1A000A114B104B9F4F10180858F70823091F44B
:10C1B000E114F10479F0D70118968C918F708230D8
:10C1C00049F481859285A385B485F701818792879B
:10C1D000A387B48791E080E0AB2809F090E0E92ED6
:10C1E000F82E79CDF10181859285992746CFF1010D
:10C1F00081859285A385B485892F9A2FAB2FBB2784
:10C20000A7FDBA95F2CFD10119968C9130933E0DCE
:10C2100020933D0D882341F080E09FEF9093400DE7
:10C2200080933F0D85E036CF90E080E0F7CFD601D8
:10C2300018968C911897806418968C9361E67FE02D
:10C2400081E99EE00F944223D8011296ED91FC9172
:10C250000280F381E02D6081718181E99EE00F947D
:10C26000EB2266EA75E081E99EE00F94EB22F6018D
:10C270006081718181E99EE00F94EB2263E57FE0AC
:10C2800081E99EE00F944223D60118968C9118976D
:10C29000982F92959F70292F2370233039F09F5F3C
:10C2A0009295907F8F70892B18968C936BE47FE02A
:10C2B00081E99EE00F944223D8011296ED91FC9102
:10C2C0000280F381E02D6081718181E99EE00F940D
:10C2D000EB2266EA75E081E99EE00F94EB22F6011D
:10C2E0006081718181E99EE00F94EB2268EF76E036
:10C2F00081E99EE00F94EB22D60118966C9162952D
:10C30000637070E081E99EE00E9422AD81E99EE0C9
:10C310000F944322D7C16DE37FE081E99EE00F9443
:10C320004223D8011296ED91FC910280F381E02D19
:10C330006081718181E99EE00F94EB2266EA75E0ED
:10C3400081E99EE00F94EB22F6016081718181E921
:10C350009EE00F94EB226AE27FE081E99EE00F9479
:10C36000422381E99EE00F944322D60118968C91D6
:10C3700018978F7018968C93A5C11092AE091092E1
:10C38000AD09D8011496ED91FC91C480D580F12CB3
:10C39000E12C0E9454BFC114D104E104F10491F0D6
:10C3A000D8011496ED91FC91468057806084718489
:10C3B00064197509860997096C157D058E059F0519
:10C3C00008F4C3C08091BC099091BD09A091BE0939
:10C3D000B091BF09892B8A2B8B2B09F0A2C0EB816E
:10C3E000FC81EF2B09F0B8C0D8011496ED91FC91B7
:10C3F00082859385892B69F484859585892B49F4F9
:10C4000086859785892B29F480899189892B09F460
:10C41000FFC080911E02893020F480911D02893076
:10C42000B8F064E07FE088E39FE00F944223D801F6
:10C430001296ED91FC910280F381E02D6081718173
:10C4400088E39FE00F94EB2288E39FE00F94432260
:10C4500081E090E09093AE098093AD09B11003C0E4
:10C46000C8010E940123D8011496ED91FC916285C8
:10C47000738542E050E0C8010E94995CD80114968F
:10C48000ED91FC916485758543E050E0C8010E9400
:10C49000995CD8011496ED91FC916685778550E002
:10C4A00040E0C8010E94995CD8011496ED91FC917E
:10C4B0006089718941E050E0C8010E94995C8091D7
:10C4C0001E02893020F480911D028930B8F064EF9B
:10C4D0007EE088E39FE00F944223D8011296ED910D
:10C4E000FC910280F381E02D6081718188E39FE0FF
:10C4F0000F94EB2288E39FE00F9443220E9454BFE5
:10C500006B017C010E9454BF6C197D098E099F0943
:10C51000623371058105910508F076C00E94CD3621
:10C52000F1CF0E9454BFC090BC09D090BD09E090EB
:10C53000BE09F090BF096C197D098E099F09683CFE
:10C5400071058105910508F04ACFD8011496ED9147
:10C55000FC9184819581D1CAAB81BC8118968C9164
:10C5600018978F70863009F03FCF1696ED90FC90AB
:10C57000E114F10409F438CFF7018085982F9F70FA
:10C580002BEF290F223008F02FCF82958F7082FF7A
:10C5900005C08B708295807F892B8087D701189684
:10C5A0008C9182958370833059F563E077E081E95F
:10C5B0009EE00F94EB22D8011296ED91FC9102803F
:10C5C000F381E02D6081718181E99EE00F94EB227F
:10C5D00066EA75E081E99EE00F94EB22F701608145
:10C5E000718181E99EE00F94EB2281E99EE00F9436
:10C5F0004322D70118968C9118978F7018968C93B8
:10C60000F701E280F380B4CF1092AE091092AD0929
:10C61000F801E480F5804FEF5FEFBA0180E00E94FF
:10C620001928D70116966D937D938D939C93199736
:10C630008CCFBDEFEB16BFEFFB0609F46CCEACF56B
:10C64000FCEFEF16FFEFFF06B9F16CE17FE081E947
:10C650009EE00F944223D8011296ED91FC91028046
:10C66000F381E02D6081718181E99EE00F94EB22DE
:10C6700066EA75E081E99EE00F94EB22F6016081A5
:10C68000718181E99EE00F94EB2261E17FE081E915
:10C690009EE00F94422381E99EE00F944322D6014D
:10C6A00018968C9118978F7765CEE114F10409F4F0
:10C6B000BECDEA94EF2849F6F60180858F70808719
:10C6C000F1E0FD83BB24B394F601C280D38076CA27
:10C6D0008FE090E09093FE108093FD1088EC90E046
:10C6E0000895FC01848195810895FC017687658712
:10C6F0000895DC01ED91FC9102A0F3A1E02D1995C4
:10C7000091E089270895862F089581E0862708956E
:10C7100021E0FC018485883008F020E0822F089514
:10C72000FC01848595850895FC0184899589089587
:10C7300026E135E0FC0131832083FB0140895189EA
:10C7400062897389FC0142835383648375830895EE
:10C75000DC01ED91FC91048CF58DE02D19946DE2D6
:10C7600077E2811102C06FE277E287E89EE00D94E4
:10C77000422365EC72E287E89EE00F944223F0E0EA
:10C78000E0E0199584EF91E008958091F90A8823FB
:10C79000B1F0E091FA0AF091FB0A309731F086810E
:10C7A00097819093F80A8093F70A6AE170E287E82C
:10C7B0009EE00F94422387E89EE00D944322089563
:10C7C000892B71F0FB01828193810E948AAE66E120
:10C7D00077E287E89EE00F94422388EC90E008958A
:10C7E00090E080E0F2CF0F931F93CF93DF93EB01A4
:10C7F00002970CF483C00A811B816BEF75E2C801BC
:10C800000F942B4D892B51F481E00E9418B188ECD4
:10C8100090E0DF91CF911F910F91089565E076E24E
:10C82000C8010F942B4D892B11F480E0EECF61ED00
:10C8300075E287E89EE00F9442230E947AB0672F4A
:10C840006095617070E087E89EE00E9422AD87E805
:10C850009EE00F9443228091630E9091640E892B89
:10C86000E9F10A811B810E941BAE8823B9F1F8010E
:10C8700001900020E9F73197E01BF10BB09770F5BC
:10C8800082E70E9406AE8091630E9091640EDC01F7
:10C89000ED91FC910088F189E02D60E270E019953E
:10C8A000B8018091630E9091640E0F94EB228091F9
:10C8B000630E9091640EDC01ED91FC910190F0818A
:10C8C000E02D60E019958091630E9091640EDC017B
:10C8D000ED91FC910488F589E02D19956A817B81A1
:10C8E00087E89EE00F94EB226AEC75E287E89EE011
:10C8F0000F94422387E89EE00F9443228091FD101D
:10C900009091FE1002973CF080EF9FEF9093FE1005
:10C910008093FD107CCF6DEB75E281E99EE00F9472
:10C92000422381E99EE00F94432284EF91E071CF8E
:10C93000892B71F0FB01828193810E94D8AE67EA56
:10C9400075E287E89EE00F94422388EC90E008951A
:10C9500090E080E0F2CFEF92FF920F931F93CF937E
:10C96000DF93CDB7DEB72C970FB6F894DEBF0FBEBE
:10C97000CDBF8C017B0186E195E09A8389831B8280
:10C980001C821D821E8298878F8319861A861B86B9
:10C990001C8605301105ECF0BE01695F7F4FF70181
:10C9A000808591850E94D832892B99F0CE01079617
:10C9B0000E947BAFBE01695F7F4FF701868197813F
:10C9C0000E94D832892B61F0CE0107960E9425B0D3
:10C9D0000EC0CE0101960E947BAF0430110554F7C2
:10C9E000CE0101960E9425B003301105A4F1BE01CD
:10C9F000695F7F4FF701848195810E94D832892B2E
:10CA000051F1CE0107960E94D0AFBE01695F7F4F02
:10CA1000F701828193810E94D832892B19F1CE01CE
:10CA200007960E9426AF60E975E287E89EE00F94C2
:10CA3000422380E00E940FB188EC90E02C960FB664
:10CA4000F894DEBF0FBECDBFDF91CF911F910F9144
:10CA5000FF90EF900895CE0101960E94D0AF023072
:10CA600011059CF6CE0101960E9426AF01301105FA
:10CA7000D1F6CE0101960E9426AF67E975E287E8FC
:10CA80009EE00F944223CFCFCF93C1E068EE73E0D6
:10CA900080E090E00E9421BF6C2F87E89EE00E941A
:10CAA0001BADCF5FC43191F784EF91E0CF91089532
:10CAB0000F931F93CF93DF938C01EB010297C4F088
:10CAC0008A819B810F94DD4C80931E0299270E94DE
:10CAD00022B10230110549F08C819D810F94DD4C0B
:10CAE00080931D0299270E942CB1C8ECD0E002C0AF
:10CAF000C0E9D1E06CE775E287E89EE00F9442233D
:10CB000060911E0287E89EE00E941BAD67E675E219
:10CB100087E89EE00F94422360911D0287E89EE023
:10CB20000E941BAD87E89EE00F944322CE01DF9167
:10CB3000CF911F910F910895CF93DF93EB0102974F
:10CB4000ACF16BEF75E28A819B810F942B4D892BA1
:10CB500029F40E947AB07D7F0E94BFB065E076E242
:10CB60008A819B810F942B4D892B29F40E947AB0E6
:10CB700072600E94BFB066E575E287E89EE00F94A0
:10CB800042230E947AB071FB662760F971E0672743
:10CB900070E087E89EE00E9422AD87E89EE00F9457
:10CBA000432288EC90E0DF91CF9108950E94713587
:10CBB000F8CF0F931F93CF93DF93CDB7DEB769976D
:10CBC0000FB6F894DEBF0FBECDBFE091F410F09128
:10CBD000F510309709F460C0809101119091021115
:10CBE000892B09F459C08FEF83871486138214822E
:10CBF00015821682178210861186128666EE72E200
:10CC000087E89EE00F94422387E89EE00F9443223A
:10CC1000BE016E5E7F4F8091F4109091F5100F94DD
:10CC2000593F1816CCF5A895AE014F5F5F4F68E0ED
:10CC3000CE0142960E944427198ABE016F5F7F4F42
:10CC400080910111909102110E9491AC8C0161EED2
:10CC500072E287E89EE00F944223BE016F5F7F4F30
:10CC600087E89EE00F94EB220115110591F0C801B1
:10CC70000E94E5348C01892B59F26CED72E287E851
:10CC80009EE00F944223B80187E89EE00F94EB22C8
:10CC9000BBCF67ED72E2B4CF88EC90E069960FB637
:10CCA000F894DEBF0FBECDBFDF91CF911F910F91E2
:10CCB00008950F931F93CF93DF9300D000D0CDB78B
:10CCC000DEB70E94F73661E370E287E89EE00F94DA
:10CCD0004223CE0101960F94E03CCE0101960E94C2
:10CCE000823206E115E01A83098380917A0C9091D3
:10CCF0007B0CA0917C0CB0917D0C8B839C83AD83CD
:10CD0000BE83CE0101960E9482321A8309831B8260
:10CD10001C821D821E8280E591E00E94E3B844E0FF
:10CD200050E0BE016D5F7F4F81E090E00F94C52C15
:10CD30000F94D32FCE0101960E9482321A83098369
:10CD40001B821C821D821E8280E591E00E94E3B856
:10CD500044E050E0BE016D5F7F4F85E090E00F94AE
:10CD6000C52C0F94D32FCE0101960E94823267E525
:10CD700070E287E89EE00F94422388EC90E02696CC
:10CD80000FB6F894DEBF0FBECDBFDF91CF911F91DC
:10CD90000F9108950D94AC4BCF92DF92EF92FF92DA
:10CDA0000F931F93CF93DF9300D000D0CDB7DEB7A2
:10CDB0008091AF0981119AC08091FD109091FE1071
:10CDC00002970CF493C08091A8099091A90900974B
:10CDD00009F48CC068E177E00E9491AC8C01009767
:10CDE00009F484C00E94ACADE82EF12CE114F104EA
:10CDF00009F47CC070E060E0C8010E94A2276C01C9
:10CE0000EA94EF2809F481C061E0C8010E9409ADED
:10CE1000FC0101851285CE0101960F94E03CCE0104
:10CE200001960E94E6B866E67BE187E89EE00F94F3
:10CE30004223B60187E89EE00F94EB2266E976E094
:10CE400087E89EE00F94EB22B80187E89EE00E94FD
:10CE500022AD66E976E087E89EE00F94EB2264EA73
:10CE60007BE087E89EE00F94EB2287E89EE00F943A
:10CE7000432262E072E086E59FE00F944F38D09243
:10CE80004C0FC0924B0F10934E0F00934D0F84EA3E
:10CE90009BE0892BE9F586E197E09093500F809312
:10CEA0004F0F8091F70A9091F80A009741F070E0D7
:10CEB00060E00E94A2279093B1098093B00980910D
:10CEC000B0099091B109009731F19093520F80937E
:10CED000510F1092540F1092530F81E08093AF09BD
:10CEE0006DE47BE187E89EE00F94422326960FB61F
:10CEF000F894DEBF0FBECDBFDF91CF911F910F9190
:10CF0000FF90EF90DF90CF90089502E012E083CF82
:10CF100084EA9BE0C2CF8BEA92E0D7CFEF92FF92F8
:10CF20000F931F93CF93DF9300D000D0CDB7DEB720
:10CF30007C018B016CE776E188E39FE00F9442234C
:10CF4000D7011296ED91FC916081718188E39FE099
:10CF50000F94EB2263E776E188E39FE00F9442238E
:10CF6000012E000C220B330B09831A832B833C8385
:10CF700080E190E09E838D83BE016F5F7F4F88E3E9
:10CF80009FE00F945A000F94432240E050E860E085
:10CF900070E0C7010E9474E626960FB6F894DEBFD3
:10CFA0000FBECDBFDF91CF911F910F91FF90EF90FA
:10CFB0000895CF92DF92EF92FF920F931F93CF933A
:10CFC000DF93CDB7DEB7C154D1090FB6F894DEBFF9
:10CFD0000FBECDBF6C01AB0130E020E060E4CE01BC
:10CFE00001967C010E94732FF70101900020E9F760
:10CFF00031978F010E191F09A801B701C6010F94BF
:10D000009459892B11F010E000E0C801CF5BDF4F8D
:10D010000FB6F894DEBF0FBECDBFDF91CF911F9149
:10D020000F91FF90EF90DF90CF9008953F924F9235
:10D030005F926F927F928F929F92AF92BF92CF92A8
:10D04000DF92EF92FF920F931F93CF93DF93CDB7B1
:10D05000DEB72C970FB6F894DEBF0FBECDBF5C01D4
:10D06000362E972E3A0169016DED76E188E39FE057
:10D070000F944223632D792D88E39FE00E9422AD17
:10D0800065ED76E188E39FE00F944223C301B0E0B1
:10D09000A0E08F839887A987BA8730E1432E512C6F
:10D0A0005C864B86BE01695F7F4F88E39FE00F94EB
:10D0B0005A004C0161ED76E10F944223B601C401A0
:10D0C0000E9422AD69EC76E1C4010F944223C701AE
:10D0D000B0E0A0E089839A83AB83BC835E824D82FB
:10D0E000BE016F5F7F4FC4010F945A000F9443221B
:10D0F0008091AD099091AE0970E060E0892B09F054
:10D1000047C081E090E09093AE098093AD0926E09E
:10D1100040E855E260E070E086EB9BE00F944E241F
:10D120003092B50C86EB9BE09093B40C8093B30CDB
:10D130001092C30D1092C50D1092C40D013011054F
:10D1400009F44EC00CF041C0012B09F44EC0C114CB
:10D15000D10409F457C082E0C816D10409F062C0B6
:10D1600070923E0D60923D0D1092400D10923F0D59
:10D17000F092420DE092410D86E00E94AEC0109206
:10D18000AE091092AD09882309F456C0682F70E0EB
:10D19000C5010E948E6790E080E02C960FB6F8944F
:10D1A000DEBF0FBECDBFDF91CF911F910F91FF90DA
:10D1B000EF90DF90CF90BF90AF909F908F907F9037
:10D1C0006F905F904F903F9008950330110581F06C
:10D1D0000430110509F0BBCFFE24EF24FE24B7CFA5
:10D1E000FE2CEE24EE24EA94B2CFFF24FA94AFCFC3
:10D1F000EF2821F492E0E92EF12CEECFEE24E39417
:10D20000F12CEACF70923E0D60923D0D90E080E0EF
:10D21000EE2011F080E09FEF9093400D80933F0D42
:10D2200085E0ABCF6DEA76E188E39FE00F9442237F
:10D230001092AE091092AD0981E090E0AECFCF928E
:10D24000DF92EF92FF921F93CF93DF9300D000D035
:10D25000CDB7DEB768E47BE187E89EE00F94422318
:10D260008BE6E82E8EE0F82E10E090E1C92ED12C4E
:10D27000F70181917F01803130F46FE177E087E839
:10D280009EE00F94EB22153041F1F7013197808138
:10D2900090E0B0E0A0E089839A83AB83BC83DE8218
:10D2A000CD82BE016F5F7F4F87E89EE00F945A00EA
:10D2B00066E47BE10F9442231F5F1630C9F6269681
:10D2C0000FB6F894DEBF0FBECDBFDF91CF911F9197
:10D2D000FF90EF90DF90CF9008958091700E90E0D6
:10D2E000B0E0A0E089839A83AB83BC83DE82CD82E9
:10D2F000BE016F5F7F4F87E89EE00F945A000F9446
:10D300004322DACFEF92FF920F931F93CF93DF93D5
:10D3100000D000D01F92CDB7DEB77B01CE010796BB
:10D320009F938F9301979F938F9301979F938F93D1
:10D3300001979F938F9301979F938F9301979F934B
:10D340008F938E010F5F1F4F1F930F9381E297E022
:10D350009F938F93DB0113968C9113978F93129663
:10D360008C918F930F94295A0FB6F894DEBF0FBE9D
:10D37000CDBF0697ECF46BEE76E281E99EE00F9468
:10D380004223D70112966D917C9181E99EE00F9422
:10D39000EB2280E991E027960FB6F894DEBF0FBE2E
:10D3A000CDBFDF91CF911F910F91FF90EF90089526
:10D3B0008091630E9091640E892BA9F10E941BAE9F
:10D3C000882389F182E70E9406AE8091630E9091D6
:10D3D000640EDC01ED91FC910088F189E02D64E0A0
:10D3E00070E019958091630E9091640EDC01ED91CF
:10D3F000FC910280F381E02D46E050E0B8011995E0
:10D4000086E0F801ABE6BEE001900D928A95E1F767
:10D410008091630E9091640EDC01ED91FC91048883
:10D42000F589E02D19950E941F696DEF76E287E876
:10D430009EE00F94422388EC90E0ADCF0895CF9208
:10D44000DF92FF920F931F93CF93DF93F12C61151F
:10D45000710509F48DC06A01EB018C01CB010E94BA
:10D4600084E4F82E882309F483C0D6FE0EC0D801C8
:10D470008C918B3009F450C008F041C040E051E07D
:10D4800060E070E08A3009F450C0D4FE09C0F801B1
:10D49000608186EF860F843018F0CE010E94F8E795
:10D4A000D5FE66C0D80114964D915D916D917C9129
:10D4B000179711968C918F70873030F08930C8F1B2
:10D4C0008A50823008F45DC0CE010E9431E5EE81C1
:10D4D000FF81309709F44CC080858F709EEF980FC4
:10D4E000923010F0811144C0D80111968C91982F80
:10D4F0009295907F80858F70892B808739C08C3082
:10D5000081F040E056E060E070E08D3009F0BDCF82
:10D51000CE010E9474E6B9CF40E051E060E070E0D7
:10D52000F7CF40E056E060E070E0CE010E944BE6AD
:10D53000ACCFEE81FF813097D9F080858F709EEF60
:10D54000980F923010F0811113C041875287638782
:10D550007487EE81FF818085807F83608087EE8184
:10D56000FF818085982F907F8F708067903629F299
:10D570008F2DDF91CF911F910F91FF90DF90CF9072
:10D580000895CE010E9431E5F3CFCF93DF9300D011
:10D5900000D01F921F92CDB7DEB7FC01628398E0E6
:10D5A000DE01119601900D929A95E1F729813A8159
:10D5B0004B815C816D817E818F81988528960FB625
:10D5C000F894DEBF0FBECDBFDF91CF910895CF930A
:10D5D000DF9300D000D01F921F92CDB7DEB7FC01C1
:10D5E000608398E0DE01119601900D929A95E1F723
:10D5F00029813A814B815C816D817E818F81988503
:10D6000028960FB6F894DEBF0FBECDBFDF91CF9145
:10D610000895CF93DF9300D000D01F921F92CDB713
:10D62000DEB7FC019181907F9A609183448355839A
:10D630006683778388E0DE01119601900D928A95CA
:10D64000E1F729813A814B815C816D817E818F81F7
:10D65000988528960FB6F894DEBF0FBECDBFDF9138
:10D66000CF910895AF92BF92CF92DF92EF92FF9247
:10D670000F931F93CF93DF9300D000D01F921F9280
:10D68000CDB7DEB76115710509F45FC05A016B01B2
:10D690007C01CB010E9484E4082F882369F1D60124
:10D6A00016968D919C91009709F443C0FC0110855A
:10D6B000212F2F703EEF320F323010F021112EC08B
:10D6C00012951F70B4FE59C0C6010E9417E8F701F9
:10D6D0008083112381F18181807F182B1183D601F2
:10D6E0001696ED91FC9181859285A385B485F7010D
:10D6F00084839583A683B783802F28960FB6F894EA
:10D70000DEBF0FBECDBFDF91CF911F910F91FF9074
:10D71000EF90DF90CF90BF90AF900895253049F4FF
:10D7200060E00E9409AD009721F0DC0118961C9181
:10D73000C7CF10E0C7CFD6011696ED91FC9180853A
:10D740008F70823021F0833051F000E0D5CF4185D9
:10D75000528563857485C7010E94096BCDCF4185D1
:10D76000528563857485F7018181807F876081831D
:10D770004483558366837783BFCF1123E1F2F7019A
:10D78000AACFCF93DF9300D000D01F921F92CDB7C6
:10D79000DEB7FC016F3F710519F014F06FEF70E018
:10D7A00077FD60E09181892F8F7081508230C8F4BD
:10D7B000648388E0DE01119601900D928A95E1F76D
:10D7C00029813A814B815C816D817E818F81988531
:10D7D00028960FB6F894DEBF0FBECDBFDF91CF9174
:10D7E0000895907F91609183E3CFCF92DF92EF9283
:10D7F000FF92DC01362F1196EC911197EF70EC300F
:10D8000008F0B6C0F0E08827E75FF3498F4F0D942A
:10D810001355BB6C416C416CB86CB86CB86C866CC1
:10D82000486CB86CB86C156C156C14968D919D9104
:10D830000D90BC91A02D662399F0B7FD9FC08F3F3E
:10D840009105A105B10529F024F08FEF90E0A0E04B
:10D85000B0E02FEF30E0A901481B590BCA010CC002
:10D86000B7FD89C08F3F9105A105B10529F024F0CE
:10D870008FEF90E0A0E0B0E0FF90EF90DF90CF90CE
:10D88000089514962C91822F90E06623A9F3E1CF9E
:10D890001496CD90DD90ED90FC901797662301F1E2
:10D8A00020E030E0A901C701B6010F943E5387FD87
:10D8B00065C020E030E04FE753E4C701B6010F94A4
:10D8C000465618160CF457C0A701960160E070E0A8
:10D8D0008FE793E40F9431550F941056CB01CCCFC2
:10D8E00020E030E0A901C701B6010F943E5387FD47
:10D8F00042C020E030E04FE753E4C701B6010F9487
:10D9000046561816DCF1C701B601E6CF14966D91A4
:10D910007D918D919C9117973323B1F06D395FEF15
:10D9200075078507950754F1611524E6720781058F
:10D9300091050CF52CE93FEF4FEF5FEF0F94AA54E0
:10D94000C90181509F4F98CF6D394FEF74078407FD
:10D9500094078CF0611554E675078105910574F400
:10D9600024E630E040E050E00F94AA54C90184CF8F
:10D970008FEF9FEF81CF90E080E07ECF8FEF90E040
:10D980007BCFCF93DF93EC01DB0189818F708630F1
:10D99000E1F128F481508230C8F080E014C0873073
:10D9A00009F18A508230C8F72FEF30E00F942A55E2
:10D9B00024E630E040E050E00F94AA542C833D83ED
:10D9C0004E835F8381E0DF91CF9108952FEF30E0A8
:10D9D0000F942A5524E630E040E050E00F94AA541A
:10D9E0002C83F0CF2FEF30E00F942A5524E630E05F
:10D9F00040E050E00F94AA54CA01B9010F94455376
:10DA00006C837D838E839F83DDCF2CE933E60F9477
:10DA10002A5524E630E040E050E00F94AA542C83CD
:10DA20003D834E835F83B9CFDC011196EC91119752
:10DA3000EF70E150EB3008F039C0F0E08827EC5D82
:10DA4000F2498F4F0D941355476D476D566D2F6DED
:10DA50002F6D386D4F6D4F6D4F6D2F6D2F6D14966F
:10DA60006D917D918D919C9117970F9445530895D9
:10DA700014966D917D918D919C91179724E630E0DD
:10DA800040E050E00F94AA54CA01B901EECF1496B9
:10DA90006C9170E090E080E00F94435308951496E9
:10DAA0006D917D918D919C911797089560E070E044
:10DAB000CB010895DC011196EC911197EF70E150C4
:10DAC000EB3008F037C0F0E08827E659F2498F4F75
:10DAD0000D9413557C6D7C6D9A6D756D756D8B6DA8
:10DAE000826D826D826D756D756D14966D917D91EF
:10DAF0008D919C911797089514966C9170E090E029
:10DB000080E0089514966D917D918D919C91179769
:10DB10000F941056089514966D917D918D919C915E
:10DB2000179724E630E040E050E00F94AA54CA0171
:10DB3000B901089560E070E0CB010895DC01119611
:10DB4000EC911197EF70E150EB3008F03EC0F0E03F
:10DB50008827E255F2498F4F0D941355C46DC46D5B
:10DB6000E56DB96DB96DDE6DCF6DCF6DCF6DB96DF2
:10DB7000B96D14962D913D914D915C911797A4E646
:10DB8000B0E00F94C954089514966C9184E6689F90
:10DB9000B0011124072E000C880B990B089520E08A
:10DBA00030E048EC52E414966D917D918D919C91FA
:10DBB00017970F94A4530F941056089514966D91CF
:10DBC0007D918D919C911797089560E070E0CB0155
:10DBD0000895FC01A7812A2F2E7FC9F081818F70C3
:10DBE00081508330A0F4A695A150BB0B2BE531E00A
:10DBF0000F942A5524E630E040E050E00F94AA54F8
:10DC0000DA01C90187569F4FAF4FBF4F08958FEF7D
:10DC10009FEF08952F923F924F925F926F927F9263
:10DC20008F929F92AF92BF92CF92DF92EF92FF922C
:10DC30000F93CF93DF9300D01F92CDB7DEB77C0157
:10DC40007A8369835C834B83DB011C92FC016081D6
:10DC50008FEF860F883108F04BC034FF49C0FAE0DF
:10DC60006F9FB00111246A54774ECD010F94804DFF
:10DC7000D70111968C918F7041F04B815C8161E8E6
:10DC800075E089819A810F948459E981FA81019024
:10DC90000020E9F7319729813A81E21BF30B190142
:10DCA0002E0E3F1E4B815C814E1B5F0B4150510974
:10DCB0005C834B83D7011196EC911197EF7009F4B7
:10DCC000F5C0E150EC3008F0F1C0F0E08827E459ED
:10DCD000F1498F4F0D9413557B6E1E6F8B6FEA6F5A
:10DCE0000570C96E9B6F9B6F9B6FB76E9F6E2170A7
:10DCF00029803A80DFCFF7018481282F30E050E07F
:10DD000040E0002359F030E0A4E6B0E00F94DC548A
:10DD10002FEF30E040E050E00F94AA545F934F9310
:10DD20003F932F9385E397E09F938F93FC81FF931D
:10DD30002B812F933F922F920F94BC59B2C017960C
:10DD40008C9117978F9316968C9116978F931596A3
:10DD50008C9115978F9314968C918F9388E397E00D
:10DD60009F938F93BC81BF93EB81EF93E3CF179683
:10DD70008C9117978F9316968C9116978F93159673
:10DD80008C9115978F9314968C918F938CE397E0D9
:10DD9000E7CF1496CD90DD90ED90FC901797F7FEAD
:10DDA00034C084E6882E912CA12CB12CC701B60179
:10DDB000A50194010F94AA549B01AC0188279927CF
:10DDC000DC01821B930BA40BB50BBF93AF939F9306
:10DDD0008F9366277727CB016C197D098E099F09E0
:10DDE000A50194010F94AA545F934F933F932F93EF
:10DDF00080E497E09F938F933C813F934B814F93B7
:10DE00003F922F920F94BC594CC0C701B60124E633
:10DE100030E040E050E00F94AA549F938F937F939B
:10DE20006F935F934F933F932F9381E497E09F937A
:10DE30008F939C819F93AB81AF93E2CFC7010E94E8
:10DE4000E96DBC01D7011696CC9016971796DC9019
:10DE50001797D0FADD24D0F814969C911497159654
:10DE6000FC90EB80BC80292F30E050E040E077FD53
:10DE700035C0011135C07F936F931F921F921F927F
:10DE80009F931F92FF92DF92CF928AE497E09F9335
:10DE90008F93FC81FF932B812F933F922F920F94AE
:10DEA000BC590FB6F894DEBF0FBECDBF89819A81F1
:10DEB0000F900F900F900F90DF91CF910F91FF90E7
:10DEC000EF90DF90CF90BF90AF909F908F907F901A
:10DED0006F905F904F903F902F900895002361F0D6
:10DEE000292F30E0A4E6B0E00F94DC542FEF30E0AF
:10DEF00040E050E00F94AA545F934F933F932F93C9
:10DF00001F92FF92DF92CF928DE497E09F938F93C1
:10DF1000BF92EF9275CF15968C9115971F928F93A4
:10DF200016969C91169717968C9181708F939F935C
:10DF300080E597E015CF14968D909D90AD90BC90A4
:10DF4000179720E030E0A901C501B4010F943E53BA
:10DF50002401350187FF04C077FA709477F8709434
:10DF6000C301B2010F9410566B01072E000C880BF1
:10DF7000990B0F9445539B01AC01C301B2010F945F
:10DF8000315520E030E04AE754E40F94A4530F9455
:10DF90009B560F941056062F772E20E030E0A901F3
:10DFA000C501B4010F943E5387FF07C07F920F93C2
:10DFB000DF92CF9286E597E0D3CE7F920F93DF92E8
:10DFC000CF9287E597E09F938F933C813F934B815E
:10DFD0004F93B0CE14968C9114971F928F931596F1
:10DFE0008C9115971F928F9316968C911F928F93F9
:10DFF0008DE497E09F938F93BC81BF93EB81EF9368
:10E000003F922F920F94BC594CCF17968C91179733
:10E010001F928F9314968C9114971F928F9315963D
:10E020008C9115971F928F9316968C911F928F93B8
:10E030008AE497E09F938F93BC81BF93EB81EF932A
:10E04000DFCE14966D917C914B815C81C1010F9460
:10E05000A2592CCFEF92FF920F93CF93DF93CDB7BE
:10E06000DEB7A0970FB6F894DEBF0FBECDBF7C0120
:10E0700000E020E030E340E250E0BE016F5F7F4F00
:10E080000E940A6EBE016F5F7F4F88E39FE00F948E
:10E09000EB2267EB79E188E39FE00F944223F701DD
:10E0A00061816F7088E39FE00E941BAD60EB79E1B6
:10E0B00088E39FE00F944223F701628188E39FE0A9
:10E0C0000E941BAD88E39FE00F944322A0960FB6F9
:10E0D000F894DEBF0FBECDBFDF91CF910F91FF90BF
:10E0E000EF900895CF93DF93EC016115710539F43A
:10E0F0008F8181708F8381E0DF91CF910895898135
:10E10000982F9F7029F180E09430B0F79B01770F32
:10E11000440B550B2959310941095109A4E6B0E0D6
:10E120000F94C9542BE531E040E050E00F94AA541D
:10E1300037FF02C030E020E02536310514F024E638
:10E1400030E02F5F220F8F818170282B2F83D3CF58
:10E15000807F82608983DACF2F923F924F925F92C5
:10E160006F927F928F929F92AF92BF92CF92DF92E7
:10E17000EF92FF920F931F93CF93DF93CDB7DEB74C
:10E1800068970FB6F894DEBF0FBECDBF6C0109874C
:10E190001A872B873C874D875E876F87788B22E1B4
:10E1A000E216F10480F5F701E75EFC4F3081398B10
:10E1B000CE0109960E94E96D97FD04C0BC01C6011D
:10E1C0000E9472708B85D60112968C931297898566
:10E1D0008C931196EC911197EF70EC3008F06CC0B5
:10E1E000F0E08827E950FF488F4F0D941355527285
:10E1F000207120719972057115736572A372A372F3
:10E20000A37265726572198AD3CFF12C9A859F70BB
:10E210009D3008F0A7C4E92FF0E08827ED5EFE48A6
:10E220008F4F0D9413555C714D736D734D7318734F
:10E2300018734D734D73B275B2754D734D7324726F
:10E240009A859F709D3008F00FC1E92FF0E0882774
:10E25000E35DFE488F4F0D9413555C710272F571AA
:10E2600052713D713A71D971047234723472C37152
:10E27000C37124728889F60187838F85D60116962B
:10E280008C9316978E8515968C9315978D8514967D
:10E290008C93149711968C911197807F892B1196EE
:10E2A0008C930AC08F859889F6018683878190FBBD
:10E2B00080F987838E858583B989BB2309F460C083
:10E2C000F60181818F702B2F30E08217130609F43D
:10E2D00057C06BEB77E188E39FE00F944223D601B0
:10E2E00011966C916F7088E39FE00E941BAD68EB04
:10E2F00077E188E39FE00F944223698988E39FE0F8
:10E300000E941BAD66EB77E188E39FE00F94422308
:10E31000F601008119821A821B821C821D821E82D4
:10E320001F82188689898F709A81907F892B8A83B2
:10E330000983EE24EA94FE2C1181228133814481E9
:10E34000558166817781CE0101960E94AC70D6011D
:10E350002C9311963C93119712964C931297139607
:10E360005C93139714966C93149715967C9315975A
:10E3700016968C93169717969C93C6010E942A7046
:10E3800088E0F60163C18D859E85AF85B889B7FDAC
:10E390000EC08F3F9105A105B10529F024F08FEF44
:10E3A00090E0A0E0B0E0D60114968C9385CF80E099
:10E3B000FACF6D857E858F85988920E06D39BFEF16
:10E3C0007B078B079B076CF02FEF6115E4E67E0758
:10E3D0008105910534F424E630E040E050E00F94EC
:10E3E000AA54D60114962C9367CF8F859889F6018D
:10E3F0008683878190FB80F987838E8585838D85D1
:10E4000084835ACF8D85CFCF8D849E84AF84B88886
:10E4100020E030E0A901C501B4010F943E5360E053
:10E4200087FD0FC020E030E04FE753E4C501B401A1
:10E430000F9446566FEF181624F0C501B4010F94DF
:10E440001756F601648338CFD60111968C91119737
:10E45000807F8C6011968C9311978D859E85159683
:10E460009C938E93149728CF6BE378E188E39FE029
:10E470000F9442236A856F7088E39FE00E941BAD72
:10E4800068E378E188E39FE00F944223F60161811D
:10E490006F7088E39FE00E941BAD88E39FE00F94BC
:10E4A00043220ACF9A859F7011968C911197807F95
:10E4B000892B11968C938D859E85AF85B889F60141
:10E4C00084839583A683B783F7CE9A859F70933014
:10E4D00089F09C3009F4B8CF4D855E856F857889C9
:10E4E000F60144835583668377838181807F892BFE
:10E4F0008183E2CE60E0C6010E94F56BD6011496DE
:10E500008C9314978F85988916968C9316971796E7
:10E510008C91179790FB80F917968C9317978E859F
:10E5200015968C93159711968C911197807F826028
:10E53000B6CE60E0CE0109960E94F56BD601149626
:10E540008C931497F0CF9A859F709D3008F057C038
:10E55000E92FF0E08827E055FD488F4F0D941355C3
:10E560005C71CA72F7727A72F772F772BD72E972F1
:10E57000E972E972D872E47224728D859E85AF8546
:10E58000B889F60184839583A683B7838181807FD0
:10E590008660AECF6D8570E090E080E00F944353CD
:10E5A000D60114966D937D938D939C93179784CE8B
:10E5B0006D857E858F8598890F944553F601648318
:10E5C00075838683978378CE6D857E858F859889C0
:10E5D000E5CFF6018181807F982B91838D859E8583
:10E5E000AF85B88984839583A683B78365CE11965A
:10E5F0008C911197807F982B11969C935CCF66E24B
:10E6000078E188E39FE00F9442236A856F7088E386
:10E610009FE00E941BAD63E278E188E39FE00F94E6
:10E620004223D60111966C9133CFFF24F394EECDA3
:10E630004D855E856F857889F601448355836683B1
:10E6400077838181807F982B918388E0DE0111960A
:10E6500001900D928A95E1F729813A814B815C8185
:10E660006D817E818F81988568960FB6F894DEBFA4
:10E670000FBECDBFDF91CF911F910F91FF90EF9013
:10E68000DF90CF90BF90AF909F908F907F906F90D2
:10E690005F904F903F902F900895963009F437C1C6
:10E6A00048F46D85913071F06FEF70E0933051F068
:10E6B00060E008C0973009F436C19A506D857E85B8
:10E6C0009230B0F784E68F8788898E7F888B1E868C
:10E6D0008A85807F82608A876D872E8530E0AFEFE4
:10E6E000B0E00F94DC54812C912C54018A94611574
:10E6F000F4E67F078105910544F424E630E040E02C
:10E7000050E00F94AA5449015A0114012D852A8B17
:10E71000022F10E0FF2009F470C088898695A82F89
:10E72000A150BB0B7D01BFEFEB16FB0609F01BC12F
:10E73000E0E88E1691040CF0FDC08FE790E0881998
:10E740009909809FD001819FB00D909FB00D112439
:10E750002FEF30E00F942A5521E83EE740E050E0EB
:10E760000F94AA54D60117962C93ABE9B0E0A501FB
:10E7700094010F94C9543FE7432E512C612C712C06
:10E78000A30192010F94AA542C593F4F4F4F5F4F52
:10E790001901AEEFB1E0A50194010F94C954A30192
:10E7A00092010F94AA54D8010F94C9542FEF30E06E
:10E7B00040E050E00F94AA5489012F3F310519F031
:10E7C00014F00FEF10E066E178E188E39FE00F942A
:10E7D0004223B10188E39FE00E9422AD68E078E126
:10E7E00088E39FE00F944223B80188E39FE00E94F2
:10E7F00022AD88E39FE00F944322E2E9F8E2E4913E
:10E80000F0E0EE0FFF1FE858F74D85919491E8ED89
:10E81000F8E2E4912F8538893170AFEFBFEF0F94A4
:10E82000DC542DE631E040E050E00F94AA54442738
:10E830005527AAEFB5E00F94C954DC01CB019058DD
:10E84000AF4FBF4FCD01BB2797FDB095AB2F8E3F8C
:10E85000E1E09E0708F05FC1382F8F3F910508F473
:10E860007CC14EEF481B50E03FEF0F5F1F4FF1019F
:10E87000FF2731962094312C3E9FC0013F9F900D81
:10E880001124292F3327220D331DD8010F942A5527
:10E890004B015C018824AA24BB245E9F90015F9FEA
:10E8A000300D1124232F3327220D331D0F942A55A9
:10E8B000BB27A92F982F872F882A992AAA2A4E9FEB
:10E8C00090014F9F300D1124232F3327220D331D2C
:10E8D000D8010F942A55B82FA72F962F882788275D
:10E8E0009927BB2788299929AA29F601A683958308
:10E8F00084836CED77E188E39FE00F944223C601A7
:10E900000E942A7060E080E00E94D9BCD5CC6D8561
:10E910007E858F85988924E630E040E050E00F94B2
:10E92000AA54B901CFCE6D857E858F8598890F94C5
:10E930001056C8CEA501940120583109410951094A
:10E94000ABE9B0E00F94C9542FE730E040E050E06D
:10E950000F94AA542C593F4F4F4F5F4F1901D601C6
:10E9600017961C9230CF9701AAEBBFEF0F94225558
:10E9700024E630E040E050E00F94AA5429013A0127
:10E98000B4E64B0E511C611C711C26E430E0D7012B
:10E990000F942A5524E630E040E050E00F94AA544A
:10E9A000DA01C9014E96A11DB11D8D8B9E8BAF8BD7
:10E9B000B88F90E8891691040CF092C08FE790E030
:10E9C00088199909809FD001819FB00D909FB00D4B
:10E9D00011242D893E894F89588D0F94D4549B0161
:10E9E000AC01AFEFB0E00F94C95424E63AE640E042
:10E9F00050E00F94AA54D60117962C93A5019401C8
:10EA0000240D351D461D571DAEEFB1E00F94C954BE
:10EA100023EE30E040E050E00F94AA5479018A01DF
:10EA20003C8B2B8BAFEFB0E0A50194010F94C95440
:10EA30002FE730E040E050E00F94AA541901EA8932
:10EA4000AE2FB0E0A80197010F94C9542FEF30E02A
:10EA500040E050E00F94AA5489012F3F310519F08E
:10EA600014F00FEF10E062E078E188E39FE00F948C
:10EA700042232AE030E0B301A20188E39FE00F9433
:10EA800065226CEF77E188E39FE00F9442232AE050
:10EA900030E04D895E896F89788D88E39FE00F941F
:10EAA000652264EF77E188E39FE00F944223B10190
:10EAB00088E39FE00E9422AD6CEE77E188E39FE05F
:10EAC0000F944223B80188E39FE00E9422AD63EED9
:10EAD00077E188E39FE00F9442236B897C8985CEA0
:10EAE000A50194012058310941095109ABE9B0E071
:10EAF0000F94C9542FE730E040E050E00F94AA543F
:10EB00002C593F4F4F4F5F4F1901D60117961C925A
:10EB10001C8A1B8AA8CF8C3FF3E09F0768F48D3FC7
:10EB200022E0920728F452E0580F3FEF40E09DCEDC
:10EB30003CEF381B5FEFFACF8A3F35E0930781F057
:10EB40008B3FE4E09E0728F444E0480F5FEF30E09D
:10EB50008CCE5AEF581B30E001C050E04FEF85CE0D
:10EB600050E0F9CF6AEC77E188E39FE00F9442230D
:10EB70006A856F7088E39FE00E941BAD67EC77E1C8
:10EB80004CCDFC019181892F8F7021F0823029F0CA
:10EB900080E00895907F926091839B0177FF02C08F
:10EBA00030E020E02E3681E0380714F02DE631E029
:10EBB0002683878130FB80F9878381E00895EF9277
:10EBC000FF920F931F93CF93DF93FC01892B69F181
:10EBD0009081992351F19D3291F180ED890F8A3016
:10EBE00070F1C8E0D0E0953211F1CEEFDFEF9B3746
:10EBF000F1F0C7E1D0E09332D1F08F0180ECE82E44
:10EC000088E1F82EC1E0D0E0C7010F94594DAC0166
:10EC1000B701C8010F94724D892B49F021968AE003
:10EC2000E80EF11CC931D10579F7CFEFDFEFCE0146
:10EC3000DF91CF911F910F91FF90EF900895D0E059
:10EC4000C0E0F5CFEF92FF920F931F93CF93DF9326
:10EC5000EC01892B51F188858F70843009F5E984A6
:10EC6000FA84C7010E94DF758C0118161906ECF4AE
:10EC7000C7010F942B2AC801012E000CAA0BBB0B55
:10EC800089879A87AB87BC878885807F82608887E1
:10EC9000C801DF91CF911F910F91FF90EF900895E0
:10ECA000823019F409851A85F3CF10E000E0F0CF27
:10ECB0002F923F924F925F926F927F928F929F928C
:10ECC000AF92BF92CF92DF92EF92FF920F931F937A
:10ECD000CF93DF93CDB7DEB7A4970FB6F894DEBF1E
:10ECE0000FBECDBF7C016B0169E276E0C6010E94D8
:10ECF00091ACFC01892B09F422C180858F7084308E
:10ED000009F455C0853009F01AC106811781011533
:10ED1000110509F414C1D80118968C9118978F70B9
:10ED2000823019F412960D911C910115110509F408
:10ED300006C1F80180858F70853011F0D801F2CFBF
:10ED4000C8010E94ACAD8230C9F760E0C8010E94E2
:10ED500009AD5C010E94227661E0C8010E9409AD04
:10ED60004C01FC0180858F70823041F7C7010E9401
:10ED70005A6DD40119964D905D906D907C901C97C2
:10ED80006415750586059705C9F6A114B10409F443
:10ED9000D6C019861A861B861C861D861E861F866F
:10EDA000188A8A85807F8A87F50161854DC06CEA63
:10EDB00075E0818592850F947459892B09F0BFC045
:10EDC000C7010E945A6D611571058105910509F40D
:10EDD0009CC0660F771F881F991F2FEF30E040E01F
:10EDE00050E00F94AA5457FD16C023303105410559
:10EDF00051050CF070C0DA01C9010196A11DB11DC9
:10EE000082309105A105B10509F44BC00397A10516
:10EE1000B10509F460C0198A1A8A1B8A1C8A1D8AE6
:10EE20001E8A1F8A188E8A89807F8A8B67E0CE01AE
:10EE300041960E94C56A29873A874B875C876D8710
:10EE40007E878F87988B62E1CE0109960E94E76AE0
:10EE500029833A834B835C836D837E838F8398877A
:10EE600029813A814B815C816D817E818F8198857A
:10EE7000A4960FB6F894DEBF0FBECDBFDF91CF9141
:10EE80001F910F91FF90EF90DF90CF90BF90AF90C8
:10EE90009F908F907F906F905F904F903F902F90BA
:10EEA0000895198A1A8A1B8A1C8A1D8A1E8A1F8A3B
:10EEB000188E8A89807F8A8B67E0CE0141960E94F6
:10EEC000C56A29873A874B875C876D877E878F87DE
:10EED000988B61E1B9CF198A1A8A1B8A1C8A1D8A0C
:10EEE0001E8A1F8A188E8A89807F8A8B67E0CE01EE
:10EEF00041960E94C56A29873A874B875C876D8750
:10EF00007E878F87988B60E19FCF198A1A8A1B8A28
:10EF10001C8A1D8A1E8A1F8A188E8A89807F8A8B86
:10EF200067E0CE0141960E94C56A29873A874B87E0
:10EF30005C876D877E878F87988B62E085CF64EBD7
:10EF400075E0C6010E9491AC8C01009709F41CC1C8
:10EF5000DC0118968C918F70853009F0FEC0C801D5
:10EF60000E94ACAD843008F40FC160E0C8010E947B
:10EF700009AD5C0161E0C8010E9409AD3C0162E09D
:10EF8000C8010E9409ADDC0119962D913D914D916A
:10EF90005C911C97298F3A8F4B8F5C8F63E0C8017F
:10EFA0000E9409AD4C0165E0C8010E9409AD6C01E9
:10EFB00067E0C8010E9409AD8C01C7010E945A6D2B
:10EFC000298D3A8D4B8D5C8D6217730784079507E9
:10EFD00014F5C114D10409F4C2C0D60118968C915D
:10EFE00018978F70823009F0BAC019861A861B866E
:10EFF0001C861D861E861F86188A8A85807F8A87C2
:10F0000019964D915D916D917C911C97CE01099659
:10F010000E94096B1DCFD40119962D913D914D9100
:10F020005C911C972D8F3E8F4F8F58A32617370763
:10F0300048075907D4F40115110509F490C0F801E7
:10F0400080858F70823009F08AC019861A861B86E7
:10F050001C861D861E861F86188A8A85807F8A8761
:10F060004185528563857485D1CFD5011996CD90A0
:10F07000DC90F3012184328419861A861B861C8653
:10F080001D861E861F86188A8A85807F8A872101B1
:10F09000032C000C6608770846010D2C000CAA080A
:10F0A000BB08098D1A8D012E000C220B330B09A30E
:10F0B0001AA32BA33CA3C7010E945A6D9B01AC016C
:10F0C000E9A0FAA00BA11CA12E193F09400B510B7E
:10F0D000C301B201681979098A099B090F94785410
:10F0E0000D8D1E8D9801110F440B550BE9A0FAA050
:10F0F0000BA11CA12E193F09400B510B0F94AA54D0
:10F10000820E931EA41EB51EC1018C199D096D8D22
:10F110007E8D098D1A8D601B710B0F94FF5477FF44
:10F1200002C06F5F7F4F75956795CB01770FAA0B74
:10F13000BB0B880D991DAA1DBB1D40E050E0BA0114
:10F14000B7FD64CFB301A20184179507A607B707DF
:10F150000CF05CCFAC01BD0159CF811115C01986EF
:10F160001A861B861C868A85807F8A871D861E8656
:10F170001F86188A88E0FE013996DE0111960190FB
:10F180000D928A95E1F76CCE88E0F701F6CF2F92C9
:10F190003F924F925F926F927F928F929F92AF9227
:10F1A000BF92CF92DF92EF92FF920F931F93CF9374
:10F1B000DF93CDB7DEB765970FB6F894DEBF0FBE0D
:10F1C000CDBF6115710549F528E0FC01DE011196FE
:10F1D00001900D922A95E1F729813A814B815C815A
:10F1E0006D817E818F81988565960FB6F894DEBF1C
:10F1F0000FBECDBFDF91CF911F910F91FF90EF9088
:10F20000DF90CF90BF90AF909F908F907F906F9046
:10F210005F904F903F902F9008953B018C0169E2E1
:10F2200076E0C3010E9491AC6C01D801FC90FF20F4
:10F2300009F45AC0009709F457C0FC0180858F700B
:10F24000843009F4DEC0853009F04EC080911E0282
:10F25000893020F480911D02893050F06FE577E00D
:10F2600088E39FE00F94EB2288E39FE00F94432212
:10F27000D6011696ED90FC90E114F104A9F1F70186
:10F2800080858F705701823069F0B12CA12CE11478
:10F29000F10409F436C1D70118968C918F7085302E
:10F2A00021F0F701E280F380F2CFC7010E94ACADFC
:10F2B0008230B9F760E0C7010E9409AD0E94227652
:10F2C0004C0161E0C7010E9409AD6C01D8018C912D
:10F2D0008815190431F7F60180858F70823009F79F
:10F2E000C114D10409F017C164EB75E0C3010E9499
:10F2F00091AC7C01D80111968C918F7009F43BC1BF
:10F30000E114F10409F43BC1F70180858F70853069
:10F3100009F0D0C1C7010E94ACAD843008F4CAC165
:10F3200064E0C7010E9409AD6C0166E0C7010E945C
:10F3300009AD1C01C8010E945A6D4B015C0160E0DF
:10F34000C7010E9409ADDC0119964D905D906D904A
:10F350007C901C97B0911E02B98B84149504A6046E
:10F36000B7040CF016C1B93020F480911D02893029
:10F3700050F166E978E188E39FE00F944223C801E9
:10F380000E945A6DAB01BC012AE030E088E39FE0A7
:10F390000F94652260E878E188E39FE00F944223B0
:10F3A00060E0C7010E9409ADFC014185528563857B
:10F3B00074852AE030E088E39FE00F94652288E3BB
:10F3C0009FE00F944322C114D10409F479C1D601FE
:10F3D00018968C9118978F70823009F071C119823C
:10F3E0001A821B821C821D821E821F8218868A81BD
:10F3F000807F8A8319964D915D916D917C911C97C8
:10F4000043C06CEA75E0818592850F947459892B0D
:10F4100009F06ACFB0E1FB1609F463C0BF1580F0B4
:10F42000E2E0FE1619F1D8014D915D916D917C914C
:10F43000139714968D919D910D90BC91A02D38C07D
:10F44000F1E1FF16F1F122E1F212EDCF19821A82F9
:10F450001B821C821D821E821F8218868A81807FE9
:10F460008A8344E150E060E070E00EC019821A82A5
:10F470001B821C821D821E821F8218868A81807FC9
:10F480008A8340E050E0BA01CE0101960E94096BE8
:10F4900029873A874B875C876D877E878F87988B14
:10F4A00049855A856B857C858D859E85AF85B88914
:10F4B00049835A836B837C838D839E83AF83B88714
:10F4C0008BCE19821A821B821C821D821E821F8291
:10F4D00018868A81807F8A8340E850E060E070E08F
:10F4E000D3CF19821A821B821C821D821E821F8228
:10F4F00018868A81807F8A834FEF50E060E070E059
:10F50000C3CFA114B10409F4EFCEF50180858F704B
:10F5100009F4EACE650180911E02893020F48091C1
:10F520001D028930B8F062EA78E188E39FE00F9429
:10F530004223D60119964D915D916D917C911C9756
:10F540002AE030E088E39FE00F94652288E39FE0A3
:10F550000F94432219821A821B821C821D821E82F2
:10F560001F8218868A81807F8A83F60141855285B1
:10F570006385748589CFE114F10409F09BC0F8011B
:10F58000408151816281738184819581A681B78197
:10F590008FCF61E0C7010E9409ADDC0119962D9162
:10F5A0003D914D915C911C972A8B3B8B4C8B5D8BD5
:10F5B000281539054A055B053CF5B989B93020F4B1
:10F5C00080911D02893050F062E678E188E39FE087
:10F5D0000F94422388E39FE00F94432221143104C7
:10F5E00009F46EC0F10180858F70823009F068C027
:10F5F00019821A821B821C821D821E821F8218861B
:10F600008A81807F8A83B2CF63E0C7010E9409ADFF
:10F610008C0162E0C7010E9409ADDC011996CD9012
:10F62000DD90ED90FC901C97F80121853285438593
:10F6300054852C193D094E095F09C501B4016419AF
:10F640007509860997090F9478542A893B894C8952
:10F650005D8924193509460957090F94AA54C20E29
:10F66000D31EE41EF51EF989F93020F480911D02A5
:10F67000893090F06DE478E188E39FE00F944223B5
:10F680002AE030E0B701A60188E39FE00F946522ED
:10F6900088E39FE00F94432219821A821B821C8206
:10F6A0001D821E821F8218868A81807F8A83B7010D
:10F6B000A601EACED70118968C918F7009F05FCF22
:10F6C00019821A821B821C828A81807F8A834981E7
:10F6D0005A816B817C8180E090E0DC01E9CE8F92E1
:10F6E0009F92AF92BF92CF92DF92FF920F931F93A0
:10F6F000CF93DF93EC018A819B810E94ACAD082FF0
:10F7000010E00430110554F40E9436B2BC018A8125
:10F710009B810E9443B20F5F1F4FF3CFEA81FB81B1
:10F72000068117810115110531F0D80112968D91CE
:10F730009C919D838C83EC81FD81309721F08281A7
:10F7400093819F838E83EE81FF81309749F0028001
:10F75000F381E02D309721F082819381998788870A
:10F760000115110541F0F80180858F70843059F141
:10F7700028F4823071F0FF24FA940CC0853001F136
:10F780008630C9F766E575E0C8010E9491AC8C012E
:10F79000E7CFF184FA86CE010E9484E4811138C05B
:10F7A00010E000E01C870B87DF91CF911F910F9134
:10F7B000FF90DF90CF90BF90AF909F908F90089573
:10F7C00006811781CDCFC184D284C114D10499F2AE
:10F7D000F6018081882379F297EE892E96E1992EA1
:10F7E000B12CA12CFA2CC4010F94594DAC01B401D9
:10F7F000C6010F94724D892BB9F1FFEFAF1ABF0A02
:10F8000089E0880E911CA7E1AA16B10459F7B3CF7D
:10F81000CE010E9449B18C010097B1F0FC018281B8
:10F820009381892B39F08F2D0E9461B28C01892B35
:10F8300009F4B6CFD801ED91FC910684F785E02D4F
:10F84000BE01C8011995AECF8F2D0E9461B28C0107
:10F85000892B09F4A5CFEA85F0E0EE0FFF1FE958E8
:10F86000F04F11830083E6CFC6010F942B2A8A2D17
:10F8700090E0B0E0A0E0F80181879287A387B48789
:10F880008085807F8260808785CFCF92DF92EF92E4
:10F89000FF920F931F93CF93DF9300D000D01F925E
:10F8A0001F92CDB7DEB77C0109831A832B833C837B
:10F8B0004D835E836F837887CE0101960E942AADC7
:10F8C0008C018981882351F09B81923008F0B6C069
:10F8D000823011F0853011F410E000E070E060E05B
:10F8E000C7010E94A1E5D82EC92E60E976E188E320
:10F8F0009FE00F9442236D2D7C2D88E39FE00E94B2
:10F9000022AD6EE876E188E39FE00F944223B801D0
:10F9100088E39FE00E9422AD88E39FE00F9443229A
:10F920008091AD099091AE09892BE9F040E050E358
:10F93000B701CE0101960E941F6A70E060E0C70126
:10F940000E948E6790E080E028960FB6F894DEBFA4
:10F950000FBECDBFDF91CF911F910F91FF90EF9020
:10F96000DF90CF90089581E090E09093AE0980936E
:10F97000AD0926E040E855E260E070E086EB9BE0F0
:10F980000F944E24D092B50C86EB9BE09093B40C70
:10F990008093B30C1092C30D1092C50D1092C40D3C
:10F9A00080ED97E090933E0D80933D0D1092400DB9
:10F9B00010923F0D01151105E1F185E090E0909363
:10F9C000420D8093410D86E00E94AEC0D82E64E6C1
:10F9D00070E080E090E00E9421BFD1100AC067E88B
:10F9E00076E188E39FE00F94422388E39FE00F9441
:10F9F000432282ED97E090933E0D80933D0D10924F
:10FA0000400D10923F0D24E6209FC001219F900DD4
:10FA100011249093420D8093410D86E00E94AEC068
:10FA20001092AE091092AD09882359F0682F70E04A
:10FA300086CF1092420D1092410DC5CF8FEF9FEFF0
:10FA400083CF81E090E080CF2F923F924F925F92E0
:10FA50006F927F928F929F92AF92BF92CF92DF92DE
:10FA6000EF92FF920F931F93CF93DF93CDB7DEB743
:10FA70002C970FB6F894DEBF0FBECDBF5C01098393
:10FA80001A832B833C834D835E836F837887CE01FB
:10FA900001960E942AAD1C01023011F0053011F4CC
:10FAA000312C212CF50104811581F80180858F709E
:10FAB000853009F07FC0C8010E94ACADE82EF12C62
:10FAC000F2E0EF16F1040CF475C060E0C8010E948A
:10FAD00009ADFC01818592859C878B8761E0C80117
:10FAE0000E9409ADFC01418452846384748488249B
:10FAF0008A94982CF2E0EF16F10459F062E0C80104
:10FB00000E9409ADFC0181849284F3E0EF16F104B8
:10FB1000A1F48FE390E09A87898792E0C92ED12CD7
:10FB200029853A85D1010F94225524E630E040E042
:10FB300050E00F94AA5479011CC063E0C8010E94F0
:10FB400009ADFC01818592859A87898782E0C82E5C
:10FB5000D12CF4E0EF16F10439F064E0C8010E9402
:10FB600009ADFC01C184D28489859A857101892BF4
:10FB7000B9F684019601A2016B857C85C5010E94BE
:10FB800016682C960FB6F894DEBF0FBECDBFDF917E
:10FB9000CF911F910F91FF90EF90DF90CF90BF908A
:10FBA000AF909F908F907F906F905F904F903F901D
:10FBB0002F90089590E080E0E4CF2F923F924F92F3
:10FBC0005F926F927F928F92AF92BF92CF92DF92AD
:10FBD000EF92FF920F931F93CF93DF93CDB7DEB7D2
:10FBE000C457D1090FB6F894DEBF0FBECDBF3C019C
:10FBF000AE960FAFAE97AF961FAFAF97E0962FAF11
:10FC0000E097E1963FAFE197E2964FAFE297E39638
:10FC10005FAFE397E4966FAFE497E5967FAFE59724
:10FC200023961FAE1EAE2397FE01ED5BFF4F82E1D0
:10FC3000DF011D928A95E9F77296119211928EE07A
:10FC4000DF011D928A95E9F76DE677E088E39FE092
:10FC50000F94EB22B50188E39FE00F94EB2261E85B
:10FC600075E088E39FE00F94EB22CE0183599F4F0C
:10FC70000E942A70D4FE2CC0AE96EFADAE97E8314C
:10FC800008F067C1F0E08827E75BF1488F4F0D94DB
:10FC90001355AF7F617EA67FA97FA97FA67F617E76
:10FCA000A97FA97FA97FA97FA97FA97FA97F617E5D
:10FCB000617EA97FA97FA97F617E617E617E617E71
:10FCC000AF7F63E875E1CE018B5A9F4F0F94524D81
:10FCD0000E94AFAC882309F419C18091F8108111FA
:10FCE00015C1A114B10409F05FC030E020E043E089
:10FCF00050E060E4CE0101960E94732FD30112966A
:10FD0000ED91FC91608171814FE350E0CE0101964D
:10FD10000F948459D5FE26C1AE968FADAE97823032
:10FD200009F420C1853009F41DC1AF968FADAF979E
:10FD30008F709FE0980F9F70923018F0883009F014
:10FD400011C101E020E030E244E150E0BE016F5B10
:10FD50007F4FCE0183599F4F0E940A6E482DBE01EE
:10FD60006F5B7F4FCE0101960E9422C069E575E16D
:10FD700088E39FE00F944223BE016F5F7F4F88E3CB
:10FD80009FE00F94EB2266E575E188E39FE00F9416
:10FD90004223BE016F5B7F4F88E39FE00F94EB220D
:10FDA00088E39FE00F944322AF968FADAF978F709B
:10FDB0001601270122243324B0E14B225524882345
:10FDC00011F0D5FC06C0211431044104510409F49A
:10FDD00009C130E020E043E050E060E4CE0101964C
:10FDE0000E94732FD3011296ED91FC916081718175
:10FDF0004FE350E0CE0101960F948459A114B10451
:10FE000069F066EA75E0CE0101960F945E594FE302
:10FE100050E0B501CE0101960F94845966EA75E071
:10FE2000CE0101960F945E594FE350E06BE175E10E
:10FE3000211431044104510459F4E0968FADE09748
:10FE40004FE350E06AE275E1873011F061E175E15E
:10FE5000CE0101960F94624DAF968FADAF978F7024
:10FE60008450823008F0A5C067E1CE0183599F4FCE
:10FE70000E94E76AA6962FAFA697A7963FAFA797CF
:10FE8000A8964FAFA897A9965FAFA997AA966FAF0C
:10FE9000AA97AB967FAFAB97AC968FAFAC97AD966A
:10FEA0009FAFAD9700E020E030E344E150E0BE01B9
:10FEB0006F5B7F4FCE0183599F4F0E940A6E61E0B6
:10FEC00075E188E39FE00F944223BE016F5F7F4F8F
:10FED00088E39FE00F94EB226EEF74E188E39FE0EC
:10FEE0000F944223BE016F5B7F4F88E39FE00F9426
:10FEF000EB2288E39FE00F9443220E94AFAC88235B
:10FF000029F08091F810882309F45DC0B701A6019B
:10FF1000C3010E9474E690E080E0CC58DF4F0FB63A
:10FF2000F894DEBF0FBECDBFDF91CF911F910F912F
:10FF3000FF90EF90DF90CF90BF90AF908F907F9029
:10FF40006F905F904F903F902F9008956DE875E10E
:10FF5000BACE6FE575E188E39FE00F944223E89401
:10FF6000D4F8B6CED4FE20CF66968FAD66978823A0
:10FF700009F41ACF482DBE016B5A7F4FCE0101966E
:10FF80000E9422C060E575E188E39FE00F94422360
:10FF9000BE016F5F7F4F88E39FE00F94EB226DE41B
:10FFA00075E188E39FE00F944223BE016B5A7F4FB7
:10FFB000F3CE20E030E323282428252811F420E084
:10FFC00030E200E072CF482DBE016F5B7F4FCE0163
:10FFD00001960E9422C040E050E260E070E0C30160
:10FFE0000E944BE6D4FE97C0A114B10409F028C1C9
:10FFF000AE96EFADAE97E150E63120F5F0E0882700
:020000021000EC
:10000000EB5FFF478F4F0D9413551881228022809C
:1000100022802280188122802280228022802280D9
:10002000228022801D8115812280228022801B80D7
:100030000C810F81128167E376E1CE018B5A9F4FCD
:100040000F94524D30E020E043E050E060E4CE01F8
:1000500001960E94732FD3011296ED91FC9160815D
:1000600071814FE350E0CE0101960F948459A114A1
:10007000B10469F066EA75E0CE0101960F945E590D
:100080004FE350E0B501CE0101960F94845966EA22
:1000900075E0CE0101960F945E594FE350E06CE09D
:1000A00075E1CE0101960F94624D68EF74E188E32B
:1000B0009FE00F944223BE016F5F7F4F88E39FE074
:1000C0000F94EB2265EF74E188E39FE00F944223E5
:1000D000BE016B5A7F4F88E39FE00F94EB2288E3C9
:1000E0009FE00F9443220E94AFAC882309F40ECF07
:1000F0008091F81081110ACF482DBE016B5A7F4FB5
:10010000CE0101960E9422C040E050E160E070E024
:10011000C3010E944BE6D6FE7CC040E051E060E0A7
:1001200070E0C3010E949DE6672B682B692B09F4E0
:1001300095C067EE75E1CE018B5A9F4F0F94524DDB
:1001400030E020E043E050E060E4CE0101960E9400
:10015000732FD3011296ED91FC91608171814FE371
:1001600050E0CE0101960F948459A114B10469F0B6
:1001700066EA75E0CE0101960F945E594FE350E0B8
:10018000B501CE0101960F94845966EA75E0CE015F
:1001900001960F945E594FE350E064E375E1CE01A0
:1001A00001960F94624D6FEE74E188E39FE00F9427
:1001B0004223BE016F5F7F4F88E39FE00F94EB22E5
:1001C0006CEE74E188E39FE00F944223BE016B5A0A
:1001D0007F4F88E39FE00F94EB2288E39FE00F942A
:1001E00043220E94AFAC882309F490CE8091F8108E
:1001F00081118CCE482DBE016B5A7F4FCE010196E6
:100200000E9422C040E050E460E070E0C3010E9420
:100210004BE681E090E081CE61E476E10ECF6BE4C5
:1002200076E10BCF65E576E108CF6FE076E105CFAB
:10023000F3018285853009F005CF65E076E1FDCEDA
:1002400000E020E030E340E150E0BE016B5A7F4F18
:10025000CE0183599F4F0E940A6EF4CE40E056E0D3
:1002600060E070E0C3010E949DE661157640810563
:10027000910519F46BEF75E15ECF6DED75E15BCF24
:100280006F927F928F92AF92BF92CF92DF92EF9256
:10029000FF920F931F93CF93DF9300D000D01F9254
:1002A0001F92CDB7DEB73C016A017B01590140FFC7
:1002B00003C0E894C0F8D3F8D3FC0DC00E941633F5
:1002C000663971058105910530F08091FD1090919E
:1002D000FE10059729F5B701A60144275077662738
:1002E0007727C3010E9474E66BED74E188E39FE019
:1002F0000F9442238FEF9FEF28960FB6F894DEBF3E
:100300000FBECDBFDF91CF911F910F91FF90EF9066
:10031000DF90CF90BF90AF908F907F906F900895B7
:1003200019821A821B821C821D821E821F821886DD
:100330008A81807F8A8340E050E3B301CE01019639
:100340000E94326B40E050E760E070E0C3010E9421
:100350009DE6C62AD72AE82AF92A882483940981A7
:100360001A812B813C814D815E816F817885C3012B
:100370000E94DD7DC1CF8F929F92AF92BF92CF92AC
:10038000DF92EF92FF920F931F93CF93DF93CDB73E
:10039000DEB760970FB6F894DEBF0FBECDBF8C01FD
:1003A0007B0140E050E860E070E00E949DE6672B32
:1003B000682B692B09F0B5C062E070E0C8010E94AB
:1003C000A1E56C0119861A861B861C861D861E8671
:1003D0001F86188A8A85807F8A87D7FCA2C040E062
:1003E00050E2B801CE0109960E94326B63E070E0E2
:1003F000C8010E94A1E5AC011816190614F04FE3DC
:1004000050E081E0C816D10429F4EF2CFF0CFF085E
:10041000FF2404C082E0C816D104D4F32FEF30E0EB
:10042000D7010F942A559A01550F440B550B0F9481
:10043000AA5449016901C8010E9417E8E82EF12C6D
:1004400060E0CE0109960E94F56B88169906F9F4D2
:10045000CD2841F082E0E816F10419F185E0E816B4
:10046000F104F9F081E090E060960FB6F894DEBFF9
:100470000FBECDBFDF91CF911F910F91FF90EF90F5
:10048000DF90CF90BF90AF909F908F900895CD2830
:1004900099F186E0E816F10441F081E0E816F104F4
:1004A00021F061E0C8010E94F8E7B401CE0109968D
:1004B0000E94C16B40E050E2B801CE0109960E9453
:1004C0001F6A82E0E816F10421F085E0E816F104E5
:1004D00049F430E020E040E050E160E070E0C80125
:1004E0000E94408130E020E040E050E260E070E0B7
:1004F000C8010E944081B6CF85E0E816F10409F4F6
:10050000B1CF82E0E816F10409F4ACCF62E0C80193
:100510000E94F8E730E020E040E050E160E070E069
:10052000E7CF90E080E0A0CFCF93DF93EC0140E0F5
:1005300050E360E070E00E949DE6AB01BC01411514
:10054000510561057105A1F08091FD109091FE109B
:10055000069771F430E020E0CE010E94408140E037
:1005600050E360E070E0CE01DF91CF910C944BE658
:10057000DF91CF910895EF92FF920F931F93CF9346
:10058000DF9300D000D0CDB7DEB78091630E90919D
:10059000640E892B09F46CC087E70E9406AE809137
:1005A000630E9091640EDC01ED91FC910088F1895D
:1005B000E02D70E060E0199510E000E08091630E9E
:1005C0009091640EDC01ED91FC9111971C962D9198
:1005D0003C910217130740F40190F081E02D60E098
:1005E00019950F5F1F4FEACF0088F189E02D70E069
:1005F00060E019950FE114E083E2E82E84E0F82E24
:100600008091630E9091640EF80161918F01DC017D
:10061000ED91FC910190F081E02D1995E016F10625
:1006200079F78091630E9091640EDC01ED91FC915D
:100630000488F589E02D19956FE479E0CE010196E3
:100640000F94E31FCE0101960E9491C9CE0101963D
:100650000F94A41F87E090E00E9422B187E090E011
:100660000E942CB166E077E287E89EE00F94422377
:100670001092830E1092820E80E090E190937E0E95
:1006800080937D0E84E890E09093850E8093840E95
:1006900081E080937F0E80E090E29093810E8093C2
:1006A000800E82E78093860E81E79EE00E94D0DF75
:1006B00081E79EE00E9436E088EC90E026960FB637
:1006C000F894DEBF0FBECDBFDF91CF911F910F9188
:1006D000FF90EF900895FF920F931F93CF93DF93B6
:1006E00000D000D0CDB7DEB78C01BC01CE010196A1
:1006F0000F94DA1FBE016F5F7F4F88E39FE00F9476
:10070000342388E39FE00F944322CE0101960F9497
:10071000A41F61E377E2CE0101960F94AC1FBE01E6
:100720006F5F7F4FC8010F94E21DF82ECE01019636
:100730000F94A41FFF2069F0B801CE0101960F9419
:10074000DA1FCE0101960E9491C9CE0101960F9445
:10075000A41F26960FB6F894DEBF0FBECDBFDF9163
:10076000CF911F910F91FF9008958F929F92BF920A
:10077000CF92DF92EF92FF920F931F93CF93DF936D
:10078000CDB7DEB7AE970FB6F894DEBF0FBECDBFC4
:100790008091A8099091A909892B09F43CC6809100
:1007A000F910811138C68091F9108F5F8093F9108C
:1007B00060EE74E287E89EE00F94422387E89EE0B3
:1007C0000F9443220091A8091091A9096AE777E0E4
:1007D000C8010E9491AC909300118093FF1060E8D3
:1007E00077E0C8010E9491AC9093B3098093B2095D
:1007F0006AE479E0C8010E9491AC9093FC10809368
:10080000FB1067E877E0C8010E9491AC9093FB0A67
:100810008093FA0A009739F1DC011696ED91FC916C
:10082000309709F120852F702530E9F46CEC74E2E3
:1008300087E89EE00F9442238091FA0A9091FB0A88
:100840000E94ACAD8093F90A682F87E89EE00E9471
:100850001BAD87E89EE00F944322E091FA0AF091E5
:10086000FB0A868197819093F80A8093F70A0E9489
:10087000CC666CE877E08091A8099091A9090E9464
:1008800091AC9093840A8093830A009709F4B0C0D6
:100890000E94ACAD082F10E00115110509F4A8C0A5
:1008A000000F111F000F111F8091810A9091820A81
:1008B000892B09F08EC07801013811051CF020E861
:1008C000E22EF12CC7010F94104B9093820A809373
:1008D000810AE092800A1092ED101092EC101092B2
:1008E000F60A1092F50A1092EB101092EF10109287
:1008F000EE10C70101960F94104B9093F110809366
:10090000F0109093EA108093E9108E0D9F1D909344
:10091000E4108093E3100E9454BF6093E51070933D
:10092000E6108093E7109093E81090E080E0E0916B
:10093000F010F091F110E80FF91F10820196E816FF
:10094000F906ACF782E090E09093ED108093EC1004
:100950008091F50A9091F60A009741F061E00E94BB
:10096000D9BC60E08091F50A0E94ABBC80E980931D
:10097000C9001092C8001092CD0083E08093CC0093
:100980008EE08093CA00F0921C02E0921B0220913C
:10099000F0103091F11080911B0290911C02820F97
:1009A000931F9093E4108093E310232B09F45DC010
:1009B0006CE574E288E39FE00F944223B70188E37B
:1009C0009FE00E9437B185E793EE9093E210809309
:1009D000E11062EB74E287E89EE00F944223B801D5
:1009E00087E89EE00E9422AD87E89EE00F944322B4
:1009F00062E977E08091A8099091A9090E9491ACE1
:100A00008C01009709F46BC00E94ACAD882309F4F7
:100A100066C06FEF680FC8010E9409ADFC01E18458
:100A2000F2849091E010992359F0809170008E7FAC
:100A3000809370001092E010109219021092180228
:100A400082E18093170291110F94B03DC7010F947A
:100A5000D83D01E010E0E016F10674F060E0C80156
:100A60000F940C3E0F5F1F4FF6CF65E474E288E3EE
:100A70009FE00F946623A7CF67E374E288E39FE0CB
:100A80000F9442230E941633AB01BC0188E39FE020
:100A90000E9418AD88E39FE00F94432266E974E258
:100AA00087E89EE00F944223B70187E89EE00E940A
:100AB00022AD87E89EE00F94432260E974E288E368
:100AC0009FE00F9442230E941633AB01BC0188E3E0
:100AD0009FE00E9418AD88E39FE00F9443220091AD
:100AE000A8091091A90966E977E0C8010E9491ACB4
:100AF0009093AC098093AB096DE977E0C8010E943F
:100B000091AC9093021180930111892B09F448C094
:100B100080910311811144C08091F4109091F510DF
:100B2000892B09F0D8C161E174E288E39FE00F945A
:100B3000422388E39FE00F9443228FE090E00F94DC
:100B4000104B8C0188E1D80111968C931197129665
:100B50001C9212971C921E961C921E921D970E9428
:100B600024B91093F5100093F410012B09F08CC0F8
:100B700062E074E281E99EE00F94422381E99EE005
:100B80000F94432280E081708093031180910311C0
:100B9000882331F060E874E287E89EE00F944223F6
:100BA0001092F7101092F610E091FF10F0910011E2
:100BB000309709F4BFC2C680D7800091FF10109112
:100BC00000110115110509F4AEC2C114D10409F4D4
:100BD000AAC2F60180858F70853099F7C6010E9400
:100BE000ACAD823070F3A801B601CE0101960E942F
:100BF00033E9CE0101960E9484E48823E1F18C85DB
:100C00009D85009709F406C2DC01ED91FC910284F8
:100C1000F385E02D1995892B49F08C859D85DC01A4
:100C2000ED91FC910084F185E02D19958C859D85D1
:100C3000DC01ED91FC910680F781E02D1995892B5F
:100C4000D1F0CE0101960E9417E8882341F040E0E0
:100C500050E160E070E0CE0101960E9474E68F8161
:100C60009885892B41F040E050E260E070E0CE01D1
:100C700001960E9474E6D6011296CD90DC90CE01CA
:100C800001960E9400E999CF0E9424B98091F41046
:100C90009091F5100E948C24882309F489C063EE9A
:100CA00073E287E89EE00F9466238091F4109091A0
:100CB000F5100E947E24E091F410F091F51081E08F
:100CC00080838091F4109091F5100F947F3E6FEC2B
:100CD00073E2811102C06AEB73E288E39FE00F9434
:100CE00066238091011190910211892B09F44ACF5A
:100CF0008091F2109091F310892B09F0DEC083E10E
:100D000090E00F94104B8C018091F4109091F510AD
:100D10002DE134E0F801328B218B96838583148298
:100D2000108289E0818381E0828383831093F310B2
:100D30000093F2100E9454BF6B017C01F0E1CF0ED2
:100D4000F7E2DF1EE11CF11CD8011596ED91FC9134
:100D500016978FEF8387148613821482158216826A
:100D6000178210861186128614961C92BB24B394A7
:100D7000BE01605E7F4FF801858196810F94593FD7
:100D800018160CF095C00E9454BF6C157D058E0599
:100D90009F0508F08DC0DE01909698E080E09150AC
:100DA00019F1ED91E827F0E0E45DFD4C8491F7CF77
:100DB0000E94B8278091F4109091F5100E948C2425
:100DC000882359F06DE973E287E89EE00F9442238F
:100DD00087E89EE00F94432284CF61E873E281E9C3
:100DE0009EE00F946623CECE9FA19813C1CFD80169
:100DF0008C91811138C015968D919C910F947F3EF6
:100E0000BE01605E7F4FF801858196810F94603E40
:100E100040E064EBD80115968D919C910F943A3E79
:100E2000F80185809680C4010E949B25C4010E9420
:100E3000612467E88EE79CE00E94FA1A60E88EE77A
:100E40009CE00E94FA1A0E941EBFC4010E949B25CA
:100E5000982ED80115968D919C910F947F3E95FC0C
:100E600002C0F801B082AE014F5F5F4FBE01605E0D
:100E70007F4FC8010F94C03ED80111969C9088A165
:100E8000803109F4CAC2BE01605E7F4FC8010F9471
:100E90002F3F891510F5F8018181D80111968C93A7
:100EA000119714968C9114978F5F14968C9360CF42
:100EB000E091F210F091F3101282E0910111F091A3
:100EC0000211E680F7809FE7D92E80910111909161
:100ED0000211892B71F481E056CE88A1803111F482
:100EE0008CE0DBCFBE01605E7F4FC8010F942F3FC7
:100EF000D4CFE114F10479F3BE01605E7F4FF701B6
:100F0000808191810E94AB34882329F36AE673E2E1
:100F100088E39FE00F944223D7016D917C9188E391
:100F20009FE00F94EB2288E39FE00F94432200910F
:100F3000F2101091F310AE014F5F5F4FBE01605E83
:100F40007F4FC8010F94153F882309F45EC088A124
:100F5000803109F45AC0DD82F801858196810F94B1
:100F60007F3EBE01605E7F4FD80115968D919C91AA
:100F70000F94603E40E06EE4F801858196810F9405
:100F80003A3E40E06B81D80115968D919C910F946B
:100F90003A3E40E06C81F801858196810F943A3E9B
:100FA00088A1803141F040E06D81D80115968D9186
:100FB0009C910F943A3EF801858196810F947F3E73
:100FC000BE01605E7F4FD80115968D919C910F9464
:100FD000603EF801408168E4858196810F943A3E35
:100FE00064E170E080E090E00E9421BFD8018C9124
:100FF000882331F06AE070E080E090E00E9421BF39
:10100000F801858196810F947F3ED7011296ED906D
:10101000FC905BCF70E060E0CE0101960E94A1E5FC
:101020008C01912C812C97FF06C011950195110917
:1010300088248394912CCE0101960E9417E8E82E13
:10104000F12C8B85853091F0863009F014CEB02ECE
:1010500061E0802F0E94D9BC61E0892809F441C079
:10106000EA94EF2809F041C060E03FC0EF2829F47E
:1010700062E0CE0101960E94F8E740E050E160E0B6
:1010800070E0CE0101960E9474E68F819885892BCD
:1010900041F040E050E260E070E0CE0101960E9435
:1010A00074E661E0802F0E94D9BC60E0802F0E942E
:1010B000ABBC68E774E288E39FE00F944223B80179
:1010C00088E39FE00E9422AD63E774E288E39FE03B
:1010D0000F94422361E774E288E39FE00F94422378
:1010E000CACDEA94EF2809F0BFCFE62EF12C8B2D64
:1010F0000E94ABBC6CE674E288E39FE00F9442234D
:10110000B80188E39FE00E9422AD6AE674E288E3BA
:101110009FE00F944223B70188E39FE00E9422AD35
:1011200068E674E2D9CFF801868197819093F71031
:101130008093F61088E39FE00F94432266E573E204
:1011400087E89EE00F94422387E89EE00F944322B5
:10115000E091FB10F091FC10309709F4A8C0809149
:10116000F9108F5F8093F910E680F780E114F104A5
:1011700009F498C0D70118968C918F70863009F0C9
:101180007EC0F9A6E8A670E060E0CE0188960F94D4
:1011900042078DA59EA5892B09F471C08091A809ED
:1011A0009091A909892B09F46AC0C8A4D9A4C114D3
:1011B000D104B9F1F60180858F70863091F5D9A2FE
:1011C000C8A270E060E0CE0180960F944207EDA1C6
:1011D000FEA1108211821282138268EA75E0C601B4
:1011E0000E9491ACFC01892BE1F090859F70955095
:1011F0009230B8F4068117810115110591F01A8318
:101200000983B601CE0101960F944207EE81FF815A
:101210001082118212821382D80112960D911C91B4
:10122000EBCF61E573E288E39FE00F9442236BA567
:1012300088E39FE00E941BAD6FE473E288E39FE0C8
:101240000F9442236AA588E39FE00E941BAD88E3C8
:101250009FE00F944322EDA5FEA510821182128219
:1012600013828AA5843078F4823098F060E08BA5F0
:101270000E94D9BCEDA5FEA58181807F8183F70105
:10128000E280F38073CF803459F0823421F08032D1
:10129000B1F762E0ECCF60E08BA50E94D9BCEFCF44
:1012A00062E0FACF8091F91081508093F91062E4E6
:1012B00073E287E89EE00F9442236AE373E287E8D3
:1012C0009EE00F94422381E02091FF1030910011A5
:1012D000232B09F480E00E94AF6361E373E287E8A7
:1012E0009EE00F94422381E02091FB103091FC108E
:1012F000232B09F480E00E94AF6362E273E287E887
:101300009EE00F94422367E173E287E89EE00F942A
:10131000422381E02091AB093091AC09232B09F4E1
:1013200080E00E94AF6360E173E287E89EE00F9483
:10133000422381E02091F70A3091F80A232B09F427
:1013400080E00E94AF6367E073E287E89EE00F945D
:10135000422381E02091011130910211232B09F4E5
:1013600080E00E94AF636EEF72E287E89EE00F9428
:1013700042238091AF090E94AF6387E89EE00F94FB
:10138000432269EF72E287E89EE00F9442230E94B5
:101390001633AB01BC0187E89EE00E9418AD87E8D8
:1013A0009EE00F94432281E08093FC0A84E59EE056
:1013B0000F949A36882351F084E59EE00F94BC3652
:1013C00084E090E09093FE108093FD108091FD10DA
:1013D0009091FE10079731F484E090E09093FE1016
:1013E0008093FD108091F91081508093F9108091C5
:1013F000FC0AAE960FB6F894DEBF0FBECDBFDF91EC
:10140000CF911F910F91FF90EF90DF90CF90BF9001
:101410009F908F90089580E0ECCFFCE0F91508F4E0
:101420003ACD5ECD5F926F927F928F929F92AF92F4
:10143000BF92CF92DF92EF92FF920F931F93CF93C1
:10144000DF93CDB7DEB7C157D1090FB6F894DEBF31
:101450000FBECDBF4C018B01F42E642F88E39FE0BB
:101460000E941BAD65ED7AE188E39FE00F94422373
:10147000B801CE0101965C010F94DA1FB50188E333
:101480009FE00F94342388E39FE00F944322C5012B
:101490000F94A41F92E0F912A4C263ED7AE1C50192
:1014A0000F94AC1FB501C8010F94121EF82EC50190
:1014B0000F94A41FFF2009F40DC320E04DE251E07A
:1014C000B40182E39EE00F94F427E090B009F0901D
:1014D000B1096CEC7AE1CE0184599F4F0F94AC1F97
:1014E00065EC7AE1CE018A599F4F0F94AC1FCE0173
:1014F000865A9F4F0F94E03CA0961FADA0976F9621
:101500000FAD6F976E96DFAC6E976D96CFAC6D9703
:101510006FE479E0CE0181960F94E31FBE016F5D09
:101520007F4FC5010F94DA1F6C2DC5010F94F51E76
:1015300060EA77E00F94261F6D2D0F94F51E60EA88
:1015400077E00F94261F602F0F94F51E60EA77E076
:101550000F94261F612F0F94F51EBC01CE01805AF7
:101560009F4F0F94DA1FC5010F94A41FCE018196DF
:101570000F94A41F60EC7AE1CE018C5A9F4F0F9418
:10158000AC1F6FE479E0CE01825B9F4F0F94E31FA5
:1015900003E61EE0D80118966C9170E084E0759522
:1015A00067958A95E1F7C5010E94DAAD4D815E81AC
:1015B00069817A81CE01825B9F4F0F94A31EC50182
:1015C0000F94A41FF80160856F7070E0C5010E9440
:1015D000DAAD4D815E8169817A81CE01825B9F4F58
:1015E0000F94A31EC5010F94A41F0F5F1F4FFEE0B1
:1015F00009361F0779F66AEB7AE1CE01885B9F4FC7
:101600000F94AC1F68EA7AE1CE0181960F94AC1F6B
:10161000BE016F5D7F4FCE01805C9F4F0F94DA1F3C
:1016200026960EAD1FAD2697085E1F4FB801CE015E
:10163000805C9F4F0F947B1E811184C0CE01805C23
:101640009F4F0F94E31EBE01685B7F4FCE01805C0D
:101650009F4F0F94401FBE01625B7F4F0F94401F4E
:10166000BE016C5A7F4F0F94401FBE01605A7F4FDE
:101670000F94401FBE016A597F4F0F94401F8C0189
:101680004AE0B50180E590E00F94C54DF501019069
:101690000020E9F73197AF014A195B09B501C8018C
:1016A0000F94A31E811103C0C8010F94E31EBE0155
:1016B00064597F4FC8010F94401FB7010F94261F34
:1016C000BC01C4010F943423C4010F944322CE0102
:1016D000805C9F4F0F94A41FCE0181960F94A41F8E
:1016E000CE01885B9F4F0F94A41FCE01825B9F4F5A
:1016F0000F94A41FCE018C5A9F4F0F94A41FCE01AC
:10170000805A9F4F0F94A41FCE018A599F4F0F9468
:10171000A41FCE0184599F4F0F94A41FC4010F949E
:10172000432264E670E080E090E00E9421BFD40193
:10173000ED91FC910488F589E02DC401199501E033
:1017400010E0ABC022962EAD3FAD229726968EAD0F
:101750009FAD26976FE87AE1820F931F0F94524D49
:1017600026961FAF0EAF26976ECF2A966EAD7FAD31
:101770002A97CE0181960E94F5B4892B09F464C1A1
:1017800024961CAE1DAE1EAE1FAE249728961CAE2E
:101790001DAE1EAE1FAE289722968FAD2297807F7A
:1017A00022968FAF229740E050E3BE016F5D7F4FDE
:1017B000CE01805C9F4F0E94326B00E020E030E35E
:1017C00040E250E0B501CE01805C9F4F0E940A6E5E
:1017D000BC01C6010F947E1F08EC10E137C1EE205A
:1017E00009F4FDC046E050E070E060E0C8010F94ED
:1017F0006E1D4091FF1050910011D8016D917C91A8
:10180000CE0181960E9463E8CE0181960E9484E415
:1018100000E911E08823E9F18BA5873061F4CE015E
:1018200081960E943CEA61E0892B09F462E0CE01D6
:1018300081960E94F8E724961CAE1DAE1EAE1FAE28
:10184000249728961CAE1DAE1EAE1FAE289722967A
:101850008FAD2297807F22968FAF229740E050E392
:10186000BE016F5D7F4FCE01805C9F4F0E94326B47
:1018700000E020E030E340E250E0B501CE01805CC2
:101880009F4F0E940A6EBC01C6010F947E1F08EC98
:1018900010E1CE0181960E9400E9C801CF58DF4FC8
:1018A0000FB6F894DEBF0FBECDBFDF91CF911F9171
:1018B0000F91FF90EF90DF90CF90BF90AF909F90EF
:1018C0008F907F906F905F900895F8016081718193
:1018D0000E9491AC7C01892B09F044C104E911E01C
:1018E000DCCFEE2009F47BC049E050E070E060E01E
:1018F000C8010F946E1D4AE0B401C5010F94C021C8
:1019000041E050E061E875E0C8010F94A31E4D81ED
:101910005E8169817A81C8010F94A31E6BE67AE12A
:1019200088E39FE00F944223B801CE0181960F9483
:10193000DA1FBE016F5D7F4F88E39FE00F94342371
:1019400088E39FE00F944322CE0181960F94A41F59
:1019500063E67AE1CE0181960F94AC1FF801848191
:1019600095812DA13EA182179307E1F4892BA1F166
:10197000E080F18069A07AA0D7018D917D01882354
:1019800059F1082E000C990B0F94F9586C01F301D2
:1019900081913F01082E000C990B0F94F958C8163D
:1019A000D90651F3CE0181960F94A41F552041F022
:1019B00021E048EC50E0B40182E39EE00F94F4276C
:1019C000D8018D919C910F947429009711F484E9AA
:1019D00091E08C01C50141C055245394E3CF01E946
:1019E0007ECFB1E0FB1274C068E87AE1C5010F94C4
:1019F000AC1FB501C8010F94E21D582EC5010F940C
:101A0000A41F552069F1EE2051F346E050E070E04C
:101A100060E0C8010F946E1D4AE0B401CE01885BFE
:101A20009F4F0F94C0214091FF1050910011F80179
:101A300060817181CE0181960E9463E8CE0181961A
:101A40000E9484E4811191CE00E911E0CE018196DB
:101A50000E9400E9CE01885B9F4F0F94A41F1DCF09
:101A600061E77AE1C5010F94AC1FB501C8010F947D
:101A7000E21DF82EC5010F94A41FF11032CF66E5C8
:101A80007AE1C5010F94AC1FB501C8010F94E21DA6
:101A9000182FC5010F94A41F00E0112309F4FDCEF7
:101AA00080E00E9418B16EE27AE187E89EE00F9430
:101AB000422387E89EE00F9443226FE479E0C5015A
:101AC0000F94E31FC5010E9491C9C5010F94A41F83
:101AD00000E036CE61E87AE1C5010F94AC1FB50194
:101AE000C8010F94E21DF82EC5010F94A41FF11038
:101AF00076CE6BE77AE1C5010F94AC1FB501C80142
:101B00000F94E21DF82EC5010F94A41FFF2001F3CE
:101B1000EE2009F464CF45E050E070E060E0C801D9
:101B20000F946E1D60EA77E0C8010F94FD1D8823B5
:101B300039F0E090FF10F0900011E114F10491F4FD
:101B40006FE479E0C8010F94FD1D811107C08091F9
:101B5000FF1090910011009709F0B7CEE090A8090E
:101B6000F090A90920E048EC50E2B40182E39EE045
:101B70000F94F427C4010F9443221C821B828DE230
:101B800092E09A8389839E828D828FEF9FEF988760
:101B90008F83B701C5010E9475B3C3CD8F929F9209
:101BA000AF92BF92CF92DF92EF92FF920F931F936B
:101BB000CF93DF93CDB7DEB7CF55D1090FB6F894E9
:101BC000DEBF0FBECDBF8C016B016115710519F031
:101BD0004115510579F564E47BE188E39FE00F94BA
:101BE00042236BE37BE188E39FE00F944223B8013B
:101BF00088E39FE00F94EB2269E37BE188E39FE0B9
:101C00000F94422388E39FE00F944322C15ADF4F91
